:020000040800F2
:10000000404C002001010008AF4A00089D4700084D
:10001000AD4A0008B1200008A968000800000000EF
:100020000000000000000000000000003151000846
:100030007F22000800000000394E000835510008FA
:100040001B0100081B0100081B0100081B01000820
:100050001B0100081B0100081B0100081B01000810
:100060001B0100081B0100081B01000825220008D5
:100070001B010008312200083D2200084922000827
:100080001B0100081B0100081B0100081B010008E0
:10009000456800081B0100081B0100081B0100083F
:1000A0001B0100081B0100081B0100081B010008C0
:1000B0001B0100081B0100081B0100081B010008B0
:1000C0001B0100081B0100081B0100081B010008A0
:1000D0001B0100088D5600081B0100081B010008C9
:1000E0001B0100081B0100081B010008DFF80CD0F1
:1000F00001F0E8FC004800470D710008404C00206A
:100100000648804706480047FEE7FEE7FEE7FEE7B1
:10011000FEE7FEE7FEE7FEE7FEE7FEE7FD5100082B
:10012000ED0000082DE9F04F4FF0000C4FF00003F8
:1001300001EB9C5EBEF90250BEF900400EF5806EE8
:10014000BEF90290BEF900800EF5806EBEF9027015
:10015000BEF900600EF5806EBEF902B0BEF900A0D7
:100160000EF5806ED044D944A8EB4A0AA9EB4B0B9C
:100170004FEAA4044FEAA50504EBA60405EBA70586
:10018000A4EB6606A5EB670704EBA80405EBA9053D
:10019000A4EB6808A5EB690906EBAB06A7EBAA0779
:1001A000A6EB6B0B07EB6A0A458020F8044B4780EF
:1001B00020F8046BA0F8029020F8048BA0F802A0AD
:1001C00020F804BB03F1010393FAA3FCB3F5807F8D
:1001D000AED1A0EB82014FF0100312090FF23410E0
:1001E00000F1000006B403EB430C6144A2F5803239
:1001F00002EB8332B1F90250B1F90040A1EB0301E7
:10020000B0F902B0B0F900A000F10400A5EB040EB3
:100210000EFB0BFC0AEB4B0E05FB0ACB04FB0ECAD4
:10022000B1F90250B1F90040A1EB0301B0F902901D
:10023000B0F9008000F10400A5EB040E0EFB09FCF0
:1002400008EB490E05FB08C904FB0EC8B1F90250C2
:10025000B1F90040A1EB0301B0F90270B0F9006000
:1002600000F10400A5EB040E0EFB07FC06EB470EA5
:1002700005FB06C704FB0EC6B1F90250B1F90040F8
:1002800001F10001D044D944A8EB4A0AA9EB4B0B79
:100290004FEAA4044FEAA50504EB264405EB2745E5
:1002A000A4EBE636A5EBE73704EB284405EB29453C
:1002B000A4EBE838A5EBE93906EB2B46A7EB2A4778
:1002C000A6EBEB3B07EBEA3A4D800C8019444F80DC
:1002D0000E801944A1F80290A1F800801944A1F8F9
:1002E00002A021F804BBB2F5803283DA03EB430CA1
:1002F0006144A2F101025FEA024E18BFA0EB0C00BC
:100300007FF476AF06BC4FEA830392087FF46AAFAE
:10031000BDE8F08F004000000040000000400000F9
:100320005DDD213BA3227E180000412D7EA5412DDD
:100330000000412D00C000405DDD82E75DDD213B16
:100340007EA5412D0040000000400000004000005C
:10035000AA2A94126B39460649327C0CA8118E23C6
:1003600049327C0CA3227E1821F77931AA2A9412F3
:10037000A8118E235DDD213BA3227E180000412DB4
:1003800095C6B13F461A2B1E58EE3735BEB4C53E52
:10039000A8118E235DDD213B63A97138DF089A28FF
:1003A000B7CDC53E7EA5412D0000412D00C00040C7
:1003B00063A92B1E21F77931BEB4C53EBEB47C0CB7
:1003C00058EE373561AC213B95C6BAF9BAE57138BC
:1003D0003BA737355DDD82E75DDD213B7EA5412D05
:1003E00021F766D756D53F3D3BA78E23A811C9CA32
:1003F000B7CDC53E61AC7E18AA2AC1C295C6B13F31
:10040000BEB47C0C00400000004000000040000032
:100410001E3BB504693E9201C83C2403EB356409D8
:10042000C83C24036B3946066C30060E1E3BB504EF
:10043000EB356409AA2A94126B39460649327C0CC2
:10044000AE240917AF37D607882E8D0F7E1E5D1B91
:10045000EB356409AA2A941224188C1F1E34F10A61
:10046000B3269015A8118E2349327C0CA3227E1846
:10047000140B60276C30060E7E1E5D1B7104FB2A78
:10048000882E8D0F461A2B1EC7FD5A2E9D2C121139
:10049000FE15E72021F77931AA2A9412A8118E239C
:1004A00087F05334B2281314480D202602EAE536AB
:1004B000B3269015DF089A289CE32B39AE24091740
:1004C0007104FB2A5DDD213BA3227E180000412D33
:1004D0004ED7C53C9320EF198FFB6C2F78D1153E7A
:1004E0007E1E5D1B21F77931E2CB0F3F641CC61CD9
:1004F000B8F2683395C6B13F461A2B1E58EE373511
:1005000097C1FB3F24188C1F02EAE536F0BCEC3F94
:10051000FE15E720BAE57138A6B8853FD5133D2210
:1005200082E1DB39BEB4C53EA8118E235DDD213BDF
:1005300040B1AF3D790FDA244DD9423C2EAE423C5A
:10054000480D202656D53F3D8EAB823A140B6027CE
:1005500078D1153E63A97138DF089A28B7CDC53E1A
:10056000B1A71236A906CE2915CA4F3F78A668331F
:100570007104FB2A95C6B13FBCA576303902212C07
:1005800038C3EC3F7EA5412D0000412D00C0004046
:10059000BCA5CE29C7FD5A2EF0BCEC3F78A620267C
:1005A0008FFB6C2F09BAB13FB1A73D2257F97630C6
:1005B0004DB74F3F63A92B1E21F77931BEB4C53E1D
:1005C0008EABEF19ECF474325EB2153E2EAE901580
:1005D000B8F268332DB03F3D40B1121187F053346B
:1005E0002EAE423CBEB47C0C58EE373561AC213B9C
:1005F000A6B8D6072BEC1236C8AADB39F0BC240308
:1006000002EAE53663A9713897C16EFEDCE7B037C0
:1006100034A8E53695C6BAF9BAE571383BA737353F
:10062000E2CB0FF59CE32B3978A6683378D173F0D1
:1006300082E1DB39EDA579314ED7EDEB6DDF823A02
:1006400099A56C2F5DDD82E75DDD213B7EA5412D07
:100650009CE33AE352DBB63B99A5FB2A02EA19DF99
:100660004DD9423CEDA59A2887F026DB4ED7C53CF4
:1006700078A6202621F766D756D53F3D3BA78E2387
:10068000C7FDDFD363D3AF3D34A8E720710494D016
:1006900078D1153E63A92B1E140B8CCD94CF723EDE
:1006A000C8AA5D1BA811C9CAB7CDC53E61AC7E18EA
:1006B000241850C8E2CB0F3F2EAE90157E1E25C6E3
:1006C00015CA4F3F2DB09412AE244AC451C8853F7D
:1006D0005EB28D0FAA2AC1C295C6B13FBEB47C0CD2
:1006E0006C308EC1E2C4D43F4DB76409EB35B1C064
:1006F00038C3EC3F09BA46061E3B2CC097C1FB3FEE
:10070000F0BC240300400000004000000040000056
:10071000D03E2E019B3F6500363FC9009A3D5B02EB
:10072000363FC900693E92015F3C8803D03E2E01EE
:100730009A3D5B021E3BB504693E9201C83C24030E
:10074000D939E205023EF701F43BED038E380E077E
:100750009A3D5B021E3BB5043F373908313DC0026C
:10076000463A7E05EB356409C83C24036B394606DE
:1007700092348E0A5F3C88038E380E073433B70BF1
:10078000F43BED03AF37D607D231DF0C8A3B51047F
:10079000CE369D086C30060E1E3BB504EB35640961
:1007A000022F2B0FB23A1A0505352B0A932D501044
:1007B000463A7E051E34F10A212C7311D939E2051F
:1007C0003433B70BAA2A94126B39460649327C0C93
:1007D0003129B413FD38AA065B31410DB327D21479
:1007E0008E380E076C30060E3226EE151F38720753
:1007F0007B2FCA0EAE240917AF37D607882E8D0F70
:10080000262321183F373908932D50109C21371982
:10081000CE369D089D2C12110E204B1A5D36010913
:10082000A42BD3117E1E5D1BEB356409AA2A9412FA
:10083000EB1C6C1C7835C709AF295413561B791D66
:1008400005352B0AB2281314BE19841E92348E0A61
:10085000B327D21424188C1F1E34F10AB326901526
:1008600088169120A933540BB1254C16EA14932114
:100870003433B70BAE2409174A139222BF321A0C35
:10088000A923C417A8118E2349327C0CA3227E18F9
:1008900005108824D231DF0C9C213719610E7E258A
:1008A0005B31410D9320EF19BB0C7126E430A40D90
:1008B000891FA71A140B60276C30060E7E1E5D1B65
:1008C0006D094C28F42F680E721D121CC4073529BF
:1008D0007B2FCA0E641CC61C1B061A2A022F2B0F64
:1008E000561B791D7104FB2A882E8D0F461A2B1E6C
:1008F000C702D82B0E2EEE0F3519DC1E1C01B22CB0
:10090000932D501024188C1F72FF882D182DB110B4
:1009100011173A20C7FD5A2E9D2C1211FE15E72003
:100920001DFC282F212C7311EA14932173FAF22F46
:10093000A42BD311D5133D22CAF8B830282B34127A
:10094000BF12E72221F77931AA2A9412A8118E2327
:1009500079F536322D2AF41291103524D2F3EF3284
:10096000AF295413790FDA242CF2A3333129B413AD
:10097000610E7E2587F05334B2281314480D2026CB
:10098000E3EEFF34332873142E0CC12641EDA53558
:10099000B327D214140B6027A1EB48363327311547
:1009A000FA09FE2702EAE536B3269015DF089A28F1
:1009B00065E87E373226EE15C4073529CBE61238B6
:1009C000B1254C16A906CE2932E5A1382F25AB1644
:1009D0008D05652A9CE32B39AE2409177104FB2A87
:1009E00008E2B0392B24661755038F2B77E0303A95
:1009F000A923C4173902212CE9DEAB3A262321189A
:100A00001C01B22C5DDD213BA3227E180000412D8C
:100A1000D5DB923B1F22DB18E4FECF2D4FDAFD3BE6
:100A20009C213719C7FD5A2ECDD8643C1721931944
:100A3000ABFCE42E4ED7C53C9320EF198FFB6C2FF7
:100A4000D3D5213D0E204B1A73FAF22F5CD4783D9A
:100A5000891FA71A57F97630E8D2C93D041F021B37
:100A60003CF8F93078D1153E7E1E5D1B21F77931B7
:100A70000CD05C3EF81DB81B06F6F831A5CE9D3EA5
:100A8000721D121CECF4743241CDD83EEB1C6C1C70
:100A9000D2F3EF32E2CB0F3F641CC61CB8F26833CE
:100AA00088CA403FDD1B201D9FF1DF3332C96B3FF9
:100AB000561B791D87F05334E1C7913FCE1AD31DE1
:100AC0006FEFC63495C6B13F461A2B1E58EE373528
:100AD0004EC5CC3FBE19841E41EDA5350CC4E13F87
:100AE0003519DC1E2BEC1236CFC2F13FAD18341F86
:100AF00016EB7D3697C1FB3F24188C1F02EAE536C2
:100B000065C000409B17E31FEFE84B3738BFFF3F3E
:100B100011173A20DCE7B03711BEF83F8816912054
:100B2000CBE61238F0BCEC3FFE15E720BAE5713891
:100B3000D4BBDB3F74153D21AAE4CF38BFBAC43F14
:100B4000EA1493219CE32B39AFB9A73F5F14E82146
:100B50008EE28439A6B8853FD5133D2282E1DB3988
:100B6000A2B75D3F4A13922277E0303AA5B6303FF4
:100B7000BF12E7226DDF823AAFB5FD3E34123B2350
:100B800064DED33ABEB4C53EA8118E235DDD213BA1
:100B9000D5B3883E1D11E22357DC6D3BF2B2453ED2
:100BA0009110352452DBB63B15B2FC3D051088246C
:100BB0004FDAFD3B40B1AF3D790FDA244DD9423CCD
:100BC00071B05B3DED0E2C254DD8853CA9AF033DA2
:100BD000610E7E254ED7C53CE8AEA53CD40DCF2591
:100BE00051D6033D2EAE423C480D202656D53F3D02
:100BF0007BADDA3BBB0C71265CD4783DD0AC6D3B51
:100C00002E0CC12663D3AF3D2BACFA3AA10B1127B2
:100C10006DD2E33D8EAB823A140B602778D1153E3E
:100C2000F8AA063A870AAF2785D0453E6AAA8439D2
:100C3000FA09FE2794CF723EE3A9FD386D094C28CE
:100C4000A5CE9D3E63A97138DF089A28B7CDC53E71
:100C5000EBA8E1375208E728CCCCEB3E7BA84B371A
:100C6000C4073529E2CB0F3F12A8B13636078129D8
:100C7000FBCA303FB1A71236A906CE2915CA4F3F8D
:100C800057A76E351B061A2A32C96B3F05A7C63413
:100C90008D05652A51C8853FBBA61934FF04B02ACB
:100CA00072C79C3F78A668337104FB2A95C6B13F92
:100CB0003EA6B232E303452BBAC5C43F0BA6F831BA
:100CC00055038F2BE2C4D43FE0A53931C702D82B9E
:100CD0000CC4E13FBCA576303902212C38C3EC3F6F
:100CE000A1A5AF2FAA016A2C66C2F53F8DA5E42EFF
:100CF0001C01B22C97C1FB3F81A5152E8E00FA2C4A
:100D0000CAC0FF3F7EA5412D0000412D00C000401C
:100D100081A56A2C72FF882D38BFFF3F8DA58F2BD0
:100D2000E4FECF2D73BEFB3FA1A5B02A56FE152EC3
:100D3000B0BDF53FBCA5CE29C7FD5A2EF0BCEC3F97
:100D4000E0A5E72839FD9F2E32BCE13F0BA6FE2728
:100D5000ABFCE42E77BBD43F3EA611271DFC282F09
:100D6000BFBAC43F78A620268FFB6C2F09BAB13FCB
:100D7000BBA62C2501FBAF2F56B99C3F05A73524F8
:100D800073FAF22FA6B8853F57A73B23E5F9343015
:100D9000F8B76B3FB1A73D2257F976304DB74F3FBB
:100DA00012A83D21CAF8B830A5B6303F7BA83A203A
:100DB0003CF8F93000B60F3FEBA8341FAEF73931DD
:100DC0005EB5EB3E63A92B1E21F77931BEB4C53E5B
:100DD000E3A9201D93F6B93122B49D3E6AAA121CE4
:100DE00006F6F83188B3723EF8AA021B79F536325E
:100DF000F2B2453E8EABEF19ECF474325EB2153EA2
:100E00002BACDB185FF4B232CDB1E33DD0ACC417EC
:100E1000D2F3EF3240B1AF3D7BADAB1645F32C338F
:100E2000B5B0783D2EAE9015B8F268332DB03F3D89
:100E3000E8AE73142CF2A333A9AF033DA9AF54134A
:100E40009FF1DF3328AFC53C71B0341213F1193470
:100E5000A9AE853C40B1121187F053342EAE423C0E
:100E600015B2EE0FFBEF8D34B6ADFD3BF2B2CA0EFC
:100E70006FEFC63441ADB63BD5B3A40DE3EEFF34FE
:100E8000D0AC6D3BBEB47C0C58EE373561AC213B29
:100E9000AFB5540BCCED6E35F6ABD33AA5B62B0AF5
:100EA00041EDA5358EAB823AA2B70109B6ECDC352F
:100EB00029AB303AA6B8D6072BEC1236C8AADB39D4
:100EC000AFB9AA06A1EB48366AAA8439BFBA7E0533
:100ED00016EB7D360FAA2B39D4BB51048CEAB13600
:100EE000B7A9CF38F0BC240302EAE53663A971380C
:100EF00011BEF70178E9183712A9123838BFC900B6
:100F0000EFE84B37C5A8B03765C09BFF65E87E3773
:100F10007BA84B3797C16EFEDCE7B03734A8E536C7
:100F2000CFC240FD53E7E137F1A77D360CC413FC77
:100F3000CBE61238B1A712364EC5E6FA42E6423881
:100F400074A7A53595C6BAF9BAE571383BA7373508
:100F5000E1C78EF832E5A13805A7C63432C963F778
:100F6000AAE4CF38D3A6533488CA39F623E4FD382F
:100F7000A4A6DF33E2CB0FF59CE32B3978A66833C8
:100F800041CDE6F315E3583950A6EF32A5CEBFF2B6
:100F90008EE284392CA674320CD098F108E2B03974
:100FA0000BA6F83178D173F082E1DB39EDA5793108
:100FB000E8D24FEFFCE0063AD3A5F9305CD42DEE31
:100FC00077E0303ABCA57630D3D50CEDF2DF593A54
:100FD000A9A5F22F4ED7EDEB6DDF823A99A56C2FC4
:100FE000CDD8CFEAE9DEAB3A8DA5E42E4FDAB4E9ED
:100FF00064DED33A85A55A2ED5DB9AE8E1DDFA3ACC
:101000007FA5CF2D5DDD82E75DDD213B7EA5412DF6
:10101000E9DE6DE6DADC473B7FA5B22C77E059E5E7
:1010200057DC6D3B85A5212C08E248E4D5DB923BDB
:101030008DA58F2B9CE33AE352DBB63B99A5FB2AA7
:1010400032E52DE2D1DADA3BA9A5652ACBE624E127
:101050004FDAFD3BBCA5CE2965E81DE0CED9203C8A
:10106000D3A5352902EA19DF4DD9423CEDA59A28CE
:10107000A1EB18DECDD8643C0BA6FE2741ED19DDAF
:101080004DD8853C2CA66027E3EE1EDCCDD7A53CD1
:1010900050A6C12687F026DB4ED7C53C78A6202671
:1010A0002CF231DACFD6E43CA4A67E25D2F33FD988
:1010B00051D6033DD3A6DA2479F551D8D3D5213DB5
:1010C00005A7352421F766D756D53F3D3BA78E238C
:1010D000CAF87FD6D8D45B3D74A7E72273FA9BD5B4
:1010E0005CD4783DB1A73D221DFCBBD4DFD3933D3A
:1010F000F1A79321C7FDDFD363D3AF3D34A8E72029
:1011000072FF06D3E8D2C93D7BA83A201C0131D238
:101110006DD2E33DC5A88C1FC70261D1F2D1FC3D61
:1011200012A9DC1E710494D078D1153E63A92B1E40
:101130001B06CCCFFED02D3EB7A9791DC40707CF23
:1011400085D0453E0FAAC61C6D0947CE0CD05C3E2B
:101150006AAA121C140B8CCD94CF723EC8AA5D1BD8
:10116000BB0CD4CC1CCF883E29ABA71A610E21CC76
:10117000A5CE9D3E8EABEF19051073CB2ECEB13EA2
:10118000F6AB3719A811C9CAB7CDC53E61AC7E18F8
:101190004A1324CA41CDD83ED0ACC417EA1483C93F
:1011A000CCCCEB3E41AD09178816E8C857CCFD3EC4
:1011B000B6AD4C16241850C8E2CB0F3F2EAE90159A
:1011C000BE19BEC76ECB203FA9AED214561B31C785
:1011D000FBCA303F28AF1314EB1CA8C688CA403F97
:1011E000A9AF54137E1E25C615CA4F3F2DB09412C9
:1011F0000E20A7C5A3C95D3FB5B0D3119C212DC555
:1012000032C96B3F40B112112623B9C4C1C8783F1F
:10121000CDB15010AE244AC451C8853F5EB28D0F87
:101220003226E0C3E1C7913FF2B2CA0EB3277BC3B7
:1012300072C79C3F88B3060E31291CC303C7A73F62
:1012400022B4410DAA2AC1C295C6B13FBEB47C0CDE
:10125000212C6DC227C6BB3F5EB5B70B932D1DC2B7
:10126000BAC5C43F00B6F10A022FD3C14EC5CC3F68
:10127000A5B62B0A6C308EC1E2C4D43F4DB76409C9
:10128000D2314FC176C4DB3FF8B79D08343315C166
:101290000CC4E13FA6B8D6079234E0C0A1C3E73F33
:1012A00056B90E07EB35B1C038C3EC3F09BA460654
:1012B0003F3788C0CFC2F13FBFBA7E058E3864C0C9
:1012C00066C2F53F77BBB504D93945C0FEC1F83FCA
:1012D00032BCED031E3B2CC097C1FB3FF0BC240386
:1012E0005F3C19C030C1FD3FB0BD5B029A3D0BC0F1
:1012F000CAC0FF3F73BE9201D03E03C065C000402C
:1013000038BFC900202A04DB203A21FA02F000216C
:10131000704721FA02F3D040C2F120029140084305
:10132000194670470649074A0868504343F2390294
:101330001044086040087047014908607047000089
:10134000C40100206D4EC64140EA01039B0703D053
:1013500009E008C9121F08C0042AFAD203E011F8F4
:10136000013B00F8013B521EF9D2704710B504460C
:1013700004E00B7800F8013B03B1491C521EF8D27F
:10138000204610BD80EA010210B502F00043400083
:1013900022D04A001FD0010E01EB1261C0F35600AB
:1013A000C2F3560240F4000042F40002A0FB022007
:1013B00000047F39140400D0401C50EA124001D4CC
:1013C0004000491EC2B20C0604EBD010401C40087D
:1013D000802A02D003E0002010BD20F00100002987
:1013E00000DA0020184310BD30B480EA010202F098
:1013F000004530F0004221F0004013D090B1C30D01
:10140000D40DC2F31601C0F31600E41A41F4000132
:1014100040F400027D34914201D3641C00E0490095
:10142000002C02DA30BC002070474FF4000000238B
:10143000914201D3891A034340084FEA4101F7D191
:1014400051B1914202D14FF0004105E002D24FF07C
:10145000010101E06FF0010103EBC450284430BCEE
:1014600000F010BA2DE9FE4F804681EA0300C00F5C
:101470000C46009021F0004123F00045B8EB02003B
:10148000A94105D24046214690461C460B460246DD
:1014900023F00040104347D0270DC7F30A00C3F3E1
:1014A0000A510290401A019040286BDAC3F31300EE
:1014B00040F4801B0098924620B10023D2EB030A2F
:1014C00063EB0B0B01985946C0F14002504600F007
:1014D000B8F906460D4650465946019A00F0C0F943
:1014E00010EB08006141002487EA115284EAE77397
:1014F0001A4340D0009A62B3019A012A4FEA075278
:1015000015DC001B61EB02014FF0004202EA0752BA
:10151000CDE90042001C41F5801132462B4600F017
:10152000F7F903B0BDE8F08F40462146F9E7001B0C
:1015300061EB0201001C41F5801300185B4120188B
:10154000A2F5001747EB030140EAD570B6196D41CB
:1015500011E06D084FEA360645EAC0754FEA0752BA
:10156000001B61EB0201001C41F5801149084FEAA4
:1015700030000019514132462B4603B0BDE8F04F10
:1015800000F0B7B90098012240000023D0EB02021E
:1015900063EBE073009821464FEAE074B8EB00007B
:1015A00061EB0401E9E783F000435BE781F0004170
:1015B00058E72DE9FE4F81EA030404F0004421F0CE
:1015C000004100944FF0000B23F0004350EA010467
:1015D0005ED052EA03045BD0C3F30A54C1F30A5548
:1015E0002C44A4F2F3340194A0FB0254C1F3130180
:1015F00041F48011C3F3130343F4801301FB02444D
:1016000000FB034E840A970A44EA815447EA835751
:10161000A4FB076802958D0A05FB07854FEA932C0A
:1016200004FB0C542705029D4FEA065847EA16377B
:10163000B5EB08056EEB070C870E920E47EA811793
:1016400042EA8312A7FB0201B6EB0B0164EB000434
:101650002B0D43EA0C335E1844EB1C50DA4651461E
:10166000E7FB0201C5F313044FEA0B3343EA1453BB
:101670004FEA0432019C43EA0603A4F10C040294ED
:10168000009CCDE900B400F043F903B0BDE8F08F51
:1016900000200146F9E72DE9F04D81EA030404F04A
:1016A000004B21F0004514464FF0000A23F00041A2
:1016B00050EA050220D054EA01021DD0C5F30A57B2
:1016C0000246C5F31303C1F31300C1F30A5640F4F5
:1016D000801543F48013A7EB0608101BD64608F2CA
:1016E000FD3873EB050002D308F1010801E0921800
:1016F0005B41B8F1000F03DA00200146BDE8F08D30
:1017000000204FF48011064684460EE0171B73EB51
:10171000050705D3121B63EB050306434CEA010CD6
:1017200049084FEA300092185B4150EA0107EDD1B9
:1017300052EA030012D082EA040083EA050108435A
:1017400005D0101BAB4106D20122002306E0002287
:101750004FF0004302E06FF0010253101AEB060055
:101760004CEB085110EB0A0041EB0B01BDE8F04DCA
:1017700000F0BFB8C10F80EAE0700844CA079623A2
:10178000002100F088B896230022114600F083B8AB
:101790000EB5C10F80EAE0700844CA07002140F28C
:1017A00033438DE80E000A460B4600F0B1F803B053
:1017B00000BDC1F30A5210B5C1F3130140F2FF336B
:1017C00041F480119A4201DA002010BD40F2334307
:1017D0009A42A2F2334203DC5242FFF793FD10BD5E
:1017E000904010BD00F0004230F000400AD0C10D22
:1017F00001F56071C0F3160042EA0151C2084007CA
:101800001143704700200146704701F0004330B497
:1018100021F0004150EA010206D00A0DA2F56072E3
:10182000C1F31301002A02DC30BC00207047440FD2
:1018300044EAC104C100E01830BC00EBC25000F023
:1018400021B8202A04DB203A00FA02F10020704778
:101850009140C2F1200320FA03F3194390407047EE
:10186000202A06DBCB17203A41FA02F043EAE07364
:1018700006E041FA02F3D040C2F120029140084351
:10188000194670470029A8BF7047401C490008BF8F
:1018900020F00100704710B4B0FA80FC00FA0CF0A0
:1018A00050EA010404BF10BC704749B1CCF12004D8
:1018B00021FA04F411FA0CF118BF01212143084365
:1018C000A3EB0C01CB1D4FEA00614FEA102042BF91
:1018D000002010BC704700EBC35010440029A4BF87
:1018E00010BC7047401C490008BF20F0010010BC2C
:1018F000704710B5141E73F1000408DA401C41F162
:10190000000192185B411A4301D120F0010010BD83
:101910002DE9F04D92469B4611B1B1FA81F202E0F9
:10192000B0FA80F220329046FFF78BFF04460F4654
:1019300040EA0A0041EA0B0153465A46084313D0D5
:10194000114653EA010019D0C8F140025046FFF792
:10195000D9FC05460E46504659464246FFF771FFF0
:10196000084305D0012004E020463946BDE8F08D4B
:101970000020054346EAE0762C4337430A98630586
:10198000E40AA0EB08000022FD0A44EA47540A30AA
:1019900002D500200146E9E7010510196941DDE99A
:1019A000084500196941BDE8F04DA2E770B521F086
:1019B000004303430CD0C1F30A550024D5EB0405C2
:1019C00064EB0403D617AD1AB34102DB00200146D5
:1019D00070BD201841EB025170BD00002DE9F041AF
:1019E000054621F000400C46284309D0C4F30A50B4
:1019F00040F23341884205DD28462146BDE8F081AA
:101A00002846FBE740F2FE31884210DC0CDB4FEA4F
:101A1000043040EA155050EA053105D0104804F072
:101A2000004101430020E9E700200146E6E7A0F27B
:101A300033404642C6F1400228462146FFF701FFE7
:101A400007468846284621463246FFF75BFC434658
:101A50003A46FFF74EFF3246BDE8F041FFF7F1BED0
:101A60000000F03F30B5041E71F1000404DB4FF0BC
:101A70000044404264EB0101141E73F1000405DBD5
:101A80001C464FF00043524263EB04038B4208BFF5
:101A9000824230BD30B5041E71F1000404DB4FF00A
:101AA0000044404264EB0101141E73F1000405DBA5
:101AB0001C464FF00043524263EB0403994208BFB7
:101AC000904230BD064C074D06E0E06840F001034F
:101AD00094E8070098471034AC42F6D3FEF70AFBAF
:101AE00040CB000860CB00082DE9F04D00231A46DA
:101AF0001B1A8A4103DB00200146BDE8F08DC1F3CB
:101B00000A52C1F3130141F480154FF0000BD107C5
:101B100002D100186D41521E0027044640F2FF1109
:101B2000384601EB620A3E468046024600204FF4EA
:101B30008011FFF7E7FBC2197141BB1846EB0100AA
:101B4000B4EB030C75EB000C04D3E41A65EB000551
:101B500017460E46241908F101006D4180463428CD
:101B6000E3DDF91946EB0600091BA84103D24FF04B
:101B7000FF32134601E0002213461BEB070046EB41
:101B80000A51BDE8F04DFFF7B4BE70B58C1810F8DF
:101B9000015B15F0070301D110F8013B2A1106D1B2
:101BA00010F8012B03E010F8016B01F8016B5B1ECC
:101BB000F9D12B0705D40023521E0DD401F8013BA7
:101BC000FAE710F8013BCB1A921C03E013F8015B13
:101BD00001F8015B521EF9D5A142D8D3002070BD97
:101BE00070B5044600688168C943C9071BD1816884
:101BF00021F00101816001F0FFF905460EE001F0DE
:101C0000FBF9401B022809D9A06A40F01000A0622D
:101C1000E06A40F00100E062012070BD2068806849
:101C2000C043C007EBD0002070BD10B50146406A2C
:101C3000826A12F0500F05D0006A026BBDE81040B6
:101C400008461047816A41F4007181620168896821
:101C5000C1F3424107290CD1C16851B9816A21F40D
:101C600080718162816AC90403D4816A41F00101F3
:101C7000816200F08FFC10BD10B5406A816A41F0AE
:101C800040018162C16A41F00401C16200F055FD6A
:101C900010BD10B5406A00F04FFD10BDF8B500262C
:101CA0000446009600688168C943C90727D0816847
:101CB00041F001018160134813490068B0FBF1F065
:101CC00000E0401E00900028FBD101F095F9054688
:101CD00010E001F091F9401B02280BD9A06A40F0F6
:101CE0001000A062E06A40F00100E06284F8246025
:101CF0000120F8BD20688068C043C007E9D10020FA
:101D0000F8BD0000A800002040420F002DE9FC5F54
:101D1000DC4EF08E401C80B2F086DFF86C9340F20F
:101D20007F31A9F1300809F1180A09F1300B08F1E7
:101D30007807884230D30025F586F07807287DD0D3
:101D40007078401CC0B27070012800D9757008F01E
:101D500085FE0024F18E4AF824104FF07E50CA49C7
:101D600048F82400183927F81450C84841F82400CE
:101D700049F824502046FFF70BFD0022C44BFFF723
:101D80008AFCC44AC44BFFF711FCFFF73EFD4BF839
:101D90002400641C062CDDDB7079C04D00287CD04B
:101DA00001287BD002287AD00428FCD00024328D70
:101DB00037F82400BA49D1F8FC1107F0EFFA07EB25
:101DC0008400B18C4088328D081A401E80B2E96FC1
:101DD00007F0E4FA641C032CE9DB0024B0465AF84F
:101DE0002400B8F836104646081AFFF7C3FCDFF89F
:101DF0009892054649F82400B08C4000FFF7C3FCD8
:101E000001462846FFF7F0FAFFF7ECFC00224FF0FE
:101E1000804306F09BF94FF0C042A24BFFF7C9FB8D
:101E2000B68C05460F467000FFF7ADFC019059F8DF
:101E30002410A9F1180959F8240000E051E000909D
:101E4000FFF7A0FA0199FFF7CFFAFFF7CBFC2A467C
:101E50003B46FFF707FBFFF7D8FCA9F1180510F187
:101E6000FF4F45F8240014D3002045F824004F46C6
:101E70005BF824000099FFF785FA47F82400B8F8CA
:101E8000362089494AF82420884202DC7F4847F8F6
:101E90002400701EFFF76EFC02E031E03DE04DE0F3
:101EA00055F82410FFF76EFAFFF79CFC07F068F96D
:101EB000FFF77FFC744F483727F81400641C062C8A
:101EC0008DDB98F80110D8F83C004646405C98F845
:101ED0000510734D05297DD2DFE801F04755667F77
:101EE00097003079401CC0B23071062800D9357196
:101EF00030796E4900EB400001EB4000F06326E7CB
:101F00000024328D37F814006549D1F8FC1107F030
:101F100045FA641C032CF4DB5FE70024B18C37F82E
:101F20001400328D081A401E80B25D49D1F8FC11B0
:101F300007F034FA641C032CF0DB4EE70024328DEA
:101F400037F814005649D1F8FC1107F027FA37F892
:101F50001400B18C328D081A401E80B2E96F07F070
:101F60001DFA641C032CEADB37E7002405EB80052F
:101F700037F81400328D296807F010FA641C032C1E
:101F8000F6DBBDE8FC9F002405EB800537F8140064
:101F9000B18C328D081A401E80B2296807F0FEF914
:101FA000641C032CF2DBECE7002405EB800537F81A
:101FB0001400328D296807F0F1F937F81400B18C5C
:101FC000328D081A401E80B2296807F0E7F9641CB8
:101FD000032C00E037E0EADBD3E7002405EB8005C3
:101FE00037F82400328D296807F0D8F907EB840010
:101FF000B18C4088328D081A401E80B2296807F0E3
:10200000CDF9641C032CEBDBBBE70024F06B328DB5
:10201000005D05EB800137F81400096807F0BEF990
:10202000F06BB28C2044C07805EB800137F81400C7
:10203000101A401E328D80B2096807F0AFF9641C97
:10204000032CE3DB9DE70024F06B328D005D05EB94
:10205000800137F82400096807F0A0F9F06BB28C12
:102060002044C07805EB800107EB84004088101AFB
:10207000401E328D80B2096807F090F9641C032C71
:10208000E2DB7EE70C000020443800208FC28D4048
:1020900000004240CDCCCCCCCCCCEC3F80E9000859
:1020A00000E80008B89E13C00AD7233C6C03002048
:1020B000FEE70020704700207047000010B50022A6
:1020C0000449054803F0B8FB0449034803F0AEFB9C
:1020D000002010BD1845002018460020184400209C
:1020E00070B50A6800260B4C0D46182A06D2014628
:1020F0002046FFF73BF92868265405E0452020706C
:1021000072206070A070E670034803F073FB00203B
:1021100070BD000054030020184600200A460949FB
:1021200010B5D1F81812D1F8141209B1012010BD60
:102130000146044803F080FBBDE81040014803F06D
:10214000BBBB0000184600202DE9F041224E02469C
:10215000204C00213046B51430F8113024F81130ED
:10216000491CA942F8DB12B31C491D4A002031F872
:10217000023B977C00EB071704EB4707401CA7F8CE
:1021800000311028F3DB304602F057FE00F036FE37
:10219000002734F8022B06EB47010023012000F052
:1021A000EBFD78B100F0DEFD0020BDE8F0810B49C9
:1021B0003039002031F8022B24F81020401C182858
:1021C000F8DBE0E77F1CBFB2AF42E2D300F0CAFD0C
:1021D0000120EAE7C80B002000F400089C0300205F
:1021E0000C00002070B50E4E0546304602F025FE6C
:1021F00000F004FE002404CD06EB8401002302203D
:1022000000F0BAFD18B100F0ADFD002070BD641CF7
:10221000A4B2802CEFD300F0A5FD012070BD00001A
:1022200000E80008014800F033BC0000883A0020B4
:10223000014800F02DBC0000CC3A0020014800F01D
:1022400027BC0000543B0020014800F021BC0000E6
:10225000103B002030B590F840500124AC40C56BD5
:102260006C60046863604368102B036803D0996056
:102270000068C26030BD9A600068C16030BD7047C0
:1022800006490020C8610648016941F00401016166
:10229000016941F04001016170470000D001002058
:1022A00000200240064A0021D16106490A6942F035
:1022B00002020A614861086940F040000861704705
:1022C000D001002000200240044B0022DA61044AC1
:1022D000136943F00103136101807047D0010020AE
:1022E0000020024014490020CA68D306134A04D5CE
:1022F000D06940F00200D0611020CB685B0705D5A3
:10230000D36943F00103D36140F00400CB69DB07DC
:1023100007D0D36943F00403D361CA6922F00102F4
:10232000CA61A0F58072013A01D0C8607047C869DF
:1023300020F00100C861704700200240D001002059
:1023400070B5044600F058FE0546114E09E0601CC9
:1023500007D024B100F050FE401BA04201D9032059
:1023600070BDF068C007F2D1F068800601D520206A
:10237000F060F068C00605D4F069C00702D1F068CB
:10238000400703D5FFF7AEFF012070BD002070BDF0
:10239000002002402DE9F04100243D4D2646052055
:1023A00006F028FD35F81410814202DA25F8146091
:1023B00002E0081A25F81400641CF02CEFDBEF2073
:1023C000032205EB400131F8023C31F8041C0B44B8
:1023D0001944B1FBF2F125F81010401E0228F0DA82
:1023E000FF2006F007FDFF27782812D20E2006F006
:1023F00001FD0446FF21A02006F0EEFC35F8142074
:1024000029461044FF2802DD21F8147001E021F86C
:1024100014000024DFF87C8030E0C4EB04100001DD
:1024200090FBFCF035F81000C0EB801202EBC010FE
:10243000B0FBF7F0C2B29006000E802A06D967F30F
:10244000070167F30F2160F317410CE0402A04D91C
:1024500067F3070160F30F2103E060F3070166F300
:102460000F2166F317415879C0070ED0ACEB04007A
:10247000401E80B21A8D06F091FF641CB8F824C08B
:1024800043466445C9DBBDE8F081A0B2F2E7000035
:102490003A3400200C000020F8B50023009390F897
:1024A00024201C46012A12D0012280F824204A68E8
:1024B0001F26072A0DD205686F6B521E02EB82029F
:1024C0009640B7430E68964037436F6319E0022089
:1024D000F8BD05680D2A0AD22F6BD21F02EB8202CB
:1024E0009640B7430E68964037432F6309E0EF6A82
:1024F0000D3A02EB82029640B7430E68964037438E
:10250000EF620A68072605680A2A0AD3EF680A3AC2
:1025100002EB42029640B7438E6896403743EF6025
:1025200008E02F6902EB42029640B7438E6896405E
:1025300037432F610A68102A01D0112A20D1124D89
:102540000268AA4217D195682D0219D4956845F4FE
:10255000000595600968102912D10C490C4A0968D8
:10256000B1FBF2F101EB8101490000E0491E00914D
:102570000029FBD104E0816A41F02001816201233E
:1025800080F824401846F8BD00240140A80000202F
:1025900040420F0070B55E4A0168914204D15D4926
:1025A000CA6882F40042CA6000685B4988427CD1F4
:1025B0005A4CA0785A4E1E2808D0207E40F00200C7
:1025C0002076607D4A15012835D093E055490020DA
:1025D0004FF4806536F81020A2F2AA5292B241F868
:1025E0002020401CA842F5DB4E492A4601F58050C8
:1025F000FDF798FD29464C4804F00AFD48492A4653
:10260000A1F5CD7000F072F9E078012810D0A17C1E
:10261000607C06F087FA04F017FB207E20F00200B1
:102620002076E28CBDE870404049414801F070BB23
:1026300001210620EDE700210D46084636F810304E
:10264000A3F5A063B43B00D55B42401C19440828A5
:10265000F4DB15E08D4200DA0D4606EB400333F85B
:10266000103CA3F5A063B43B00D55B42C91A36F811
:102670001030A3F5A063B43B00D55B421944401C65
:102680009042E7DB8D4200DA0D46E81705EB50700B
:10269000C3100021274D084635F82060401C314406
:1026A00089B24028F8DB880900E030E0B3F5FA7F12
:1026B00003DDC82801D2207B60B1217B002029B135
:1026C000217B202910D2217B491C2173E17A4029EA
:1026D0001BD202E0207B401C0BE0E07A05EB80017E
:1026E000401CE0720B6005E0218E51B1218E2185E6
:1026F00020862073BDE870400949A1F5CD7000F037
:10270000F5B8218D21862085F3E7E072E5E770BDFD
:102710000028014000100140002401400C0000206E
:10272000C6030020C80B0020C81B0020C82B0020B7
:102730005C02002098380020704770472DE9F04176
:102740004FF00006040035467DD0A06A002728B966
:10275000E76284F82470204600F07EF82046FFF7F8
:102760003FFAA16AC90600D420B1A06A40F0100067
:10277000A06268E0A16A21F4885141F00201A162DF
:102780006268E169E3680A4346EA43010A43A168D3
:102790004FF48076B14208D0012906D00021D4F848
:1027A00014C0BCF1010F02D00AE03146F7E7F3B1E3
:1027B000A36A43F02003A362E36A43F00103E362E8
:1027C0002368D3F804C02CF4694C4CEA010CC3F81C
:1027D00004C021688B68DFF874C003EA0C0313435C
:1027E0008B60A168B1420BD0012909D00CE0DFF861
:1027F00060C0A3690CEB43330B4343F40061DFE794
:10280000218A0D05A5F580152168CB6A23F4700394
:102810002B43CB62216889680E4B1940914208D145
:10282000E762A16A21F0020141F00101A162BDE865
:10283000F081A06A20F0020040F01000A062E06A7F
:1028400040F00100E0620120F1E70000FDF7E1FF48
:1028500000E0FFFFFE0E1FFF30B505460068174978
:1028600085B0884227D11648816941F400718161A1
:102870008069694600F40070049003200090019084
:10288000104800F0CFFA114C0F4880212060002042
:102890006060C4E90201490021618900C4E90510B2
:1028A000E061204600F0A0F918B1862108A004F0EC
:1028B0002BF82C62656205B030BD00000024014099
:1028C000001002400008014008000240883A002041
:1028D0002E2E2F5372632F73746D333266317878D6
:1028E0005F68616C5F6D73702E6300002DE9F047C7
:1028F000894604463B4900683B4F0E1D904688427E
:1029000001D0B84207D1306810F4702F03D00125F0
:102910002846BDE8F08794F8240001280CD0012057
:1029200084F824002046FFF7B9F905004FF00001B4
:1029300004D084F82410EBE70220EAE7A06A40F60E
:102940000162904340F48070A0622068B84218D1C0
:10295000326812F4702F14D0A06A40F48010A06284
:102960003068400505D5A06A20F4005040F480503E
:10297000A062A06AC0040AD5E06A20F00600E06206
:1029800006E0A26A22F48012A2624068E9E7E162EE
:1029900084F82410216A15488862216A1448C862A4
:1029A000216A1448086321686FF0020008602068FB
:1029B000816841F480718160216843464A464C3108
:1029C000206A00F043F920688168C1F34241072979
:1029D000816803D041F48011816099E741F4A0013E
:1029E000FAE7000000240140002801402B1C0008E9
:1029F000931C0008791C000810B590F821100024E1
:102A0000022903D00421816301243DE001680A68A2
:102A100022F00E020A6001680A6822F001020A60D0
:102A20001A4A0168914201D1012121E0174A14326A
:102A3000914201D110211BE0144A2832914201D168
:102A4000891515E0114A3C32914201D189140FE0F9
:102A50000E4A5032914202D14FF4803108E00B4AC5
:102A60006432914202D14FF4801101E04FF0807145
:102A7000064A083A5160012180F82110002180F8AF
:102A80002010416B01B18847204610BD080002406C
:102A90002DE9F05FC16B0B6801680A68046C4FF0A8
:102AA000040C0CFA04FC4A4DDFF828A14A4E4B4FA7
:102AB000DFF82CB1DFF82CE11CEA030F2DD05FEA20
:102AC000427C2AD50A68920603D40A6822F00402DE
:102AD0000A600168A94201D1042119E0514501D1E0
:102AE000402115E0B14202D14FF4806110E0B942BB
:102AF00002D14FF480410BE0594502D14FF48021BF
:102B000006E0714502D14FF4800101E04FF0806191
:102B10002F4A083A5160C16A3BE04FF0020808FAB8
:102B200004F818EA030F4FF000094FF0010C35D0FC
:102B30005FEA827832D50A68920605D40A6822F0E4
:102B40000A020A6080F821C00168A94201D102216D
:102B500019E0514501D1202115E0B14202D14FF4D5
:102B6000007110E0B94202D14FF400510BE0594519
:102B700002D14FF4003106E0714502D14FF400114B
:102B800001E04FF00071124A083A516080F820903D
:102B9000816A00291AD0BDE8F05F08470825A540E2
:102BA0001D4213D0120711D50A6822F00E020A60E6
:102BB00090F84010C26B0CFA01F15160C0F838C0B7
:102BC00080F821C080F82090016BE2E7BDE8F09F1B
:102BD000080002401C000240300002404400024055
:102BE000580002406C00024030B548B302C8154A94
:102BF00014230A44B2FBF3F29200C263124A8263C6
:102C0000022242770B6843F6F0729343D0E9002426
:102C10002243D0E902452C432243046922434469FC
:102C20002243846922431A430A600021416281627F
:102C3000C16201634163012242770177084630BDDA
:102C4000012030BDF8FFFDBF0000024070B5044612
:102C500090F82000002501280CD0012084F82000E5
:102C600094F821600020012E06D084F8200002256F
:102C7000284670BD022070BD022684F82160A06342
:102C80002068066826F0010606602046FFF7E2FA93
:102C9000E06A00282068016802D041F00E0106E0D9
:102CA00021F0040101602068016841F00A0101601F
:102CB0002068016841F001010160D9E72DE9F04782
:102CC000054626480F460126017E01290FD0012125
:102CD000814601762868DFF888804CF2503402285B
:102CE00008D0A2462046FFF72BFBA8B131E0022016
:102CF000BDE8F0872046FFF723FB08BB0120FFF764
:102D0000BFFA2046FFF71CFBD8F81010064621F04A
:102D10000401C8F810101CE04FF0FF303860AC68B8
:102D200011E02046FFF7BEFA5046FFF709FBD8F83E
:102D30001010060021F00201C8F8101001D03C600C
:102D400007E004F58064D5E9020100EB8120A04290
:102D5000E7D8002189F818103046C9E7D0010020D3
:102D6000002002400348016941F080010161002018
:102D700070470000002002402DE9F05F05461D4825
:102D800088460024017E16461F46012909D00121EC
:102D9000814601764CF2503A5046FFF7D1FA18B10D
:102DA00023E00220BDE8F09F012D02D0022D00D0CB
:102DB0000425D346DFF840A015E02201304639460D
:102DC000FEF7A0FA81B208EB4400FFF77DFA5846FF
:102DD000FFF7B6FADAF8102022F00102CAF8102044
:102DE00018B9641CE4B2AC42E7D3002289F8182079
:102DF000D8E70000D0010020002002400649002052
:102E00000A69120607D5054A4A60054A4A600969F7
:102E1000090600D5012070470020024023016745C4
:102E2000AB89EFCD2DE9F84FDFF8A091002309F130
:102E3000040A0AF1040B1C464FF00F080BF1040EB4
:102E400001270A68A7403A40BA4272D1DFF880C130
:102E50004D68A5EB0C0665452BD00DDC032D34D059
:102E600005DC35B3012D19D0022D2FD11BE0112D1A
:102E700016D0122D2AD119E0B6F5881F19D006DC1C
:102E8000B6F5803F15D0B6F5801F1FD111E0B6F51D
:102E9000001F0ED0B6F5041F18D10AE0CB6815E06C
:102EA000CB681B1D12E0CB6808330FE0CB680C33F6
:102EB0000CE08B682BB1012B4FF0080303D0476166
:102EC00004E0042302E0076100E00023FF2A01D8A8
:102ED000064601E000F104064FEA840501D9A5F198
:102EE0002005376808FA05FC27EA0C0703FA05F500
:102EF00047EA050737604D68ED0060D5354DAE698E
:102F000046F00106AE61AD6924F0030605F0010547
:102F10000095314D7719BE68A5072D0F08FA05FCFD
:102F200026EA0C06DFF8B4C0604503D14FF0000C70
:102F300017E044E0DFF8A8C0604502D14FF0010C73
:102F40000FE0DFF8A0C0604502D14FF0020C08E0AE
:102F5000DFF894C0604502D14FF0030C01E04FF060
:102F6000040C0CFA05FC4CEA060CC7F808C04D68C6
:102F7000D9F80060ED034D4601D5164300E09643B5
:102F80002E604D68DAF80060AD03554601D5164352
:102F900000E096432E604D68DBF80060ED025D4670
:102FA00001D5164300E096432E604D68DEF80060C0
:102FB000AD02754601D5164300E096432E60641CB1
:102FC000102CFFF43DAFBDE8F88F00000004014075
:102FD00000001110001002400000014000080140F4
:102FE000000C014000100140001401400AB10161D1
:102FF00070470904FBE70000014880687047000043
:103000000000002002488168027811448160704706
:1030100000000020074810B5016841F01001016070
:10302000032000F095F8002000F006F800F024F8E6
:10303000002010BD0020024070B50D4D04464FF435
:103040007A712878B1FBF0F00A490968B1FBF0F019
:1030500000F0C9FE48B9102C07D200222146501EAC
:1030600000F056F800206C6070BD012070BD0000BB
:1030700000000020A80000201D4808B5816941F02B
:1030800001018161806900F001000090032000F0DF
:103090005FF8002211466FF00B0000F039F80022B3
:1030A00011466FF00A0000F033F8002211466FF06D
:1030B000090000F02DF800221146501F00F028F8FA
:1030C00000221146101F00F023F800221146901E26
:1030D00000F01EF800221146501E00F019F80549B4
:1030E000486820F0E06040F00070486008BD0000D3
:1030F000001002400000014000F01F020121914039
:103100004009800000F1E020C0F800117047000085
:10311000F0B40E4B1B68C3F30223C3F10704042C65
:1031200000D904241D1D072D01D2002300E0DB1E61
:10313000012606FA04F56D1E0D409D409E40761E48
:10314000164045EA0601F0BC01F0B2BC0CED00E00F
:10315000064A00F0070110684FF6FF03184040EAE6
:103160000120034908431060704700000CED00E0A7
:103170000000FA0510B50C0605D501F07F0100EB43
:103180004110283003E000EB411000F50A7099B2BD
:1031900032B101228272C180190C0181002010BD60
:1031A000002282728180F9E7704700EB4112D0F86B
:1031B0005C04D26B02F01EBD00EB4112D0F85C043F
:1031C000D2F83C2202F06BBD10B504460A460B064D
:1031D00001F07F0004EB401101D5283101E001F539
:1031E0000A710870D009487094F82804012809D0A1
:1031F000012084F82804206803F04BF9002084F8AB
:10320000280410BD022010BD70B50A460446090608
:1032100002F07F0003D504EB4011283103E004EBFA
:10322000421101F50A7100258D700870D0094870AF
:1032300094F82804012809D0012084F82804206883
:1032400003F0CBF984F82854002070BD022070BD33
:1032500001F00F0100EB4110B0F8440280B270475A
:1032600070B504460D460E0601F07F0004EB4011D8
:1032700001D5283101E001F50A710870E8094870AC
:103280000A61CB7094F82804012809D0012084F841
:103290002804206802F0D2FF002084F8280470BDC2
:1032A000022070BD70B50D4601F07F0400EB4411A3
:1032B000C1E98F230022C1F8442281F8292281F834
:1032C000284201F50A716A06006803F0E0F900205F
:1032D00070BD70B50D460446090605F07F0003D5A4
:1032E00004EB4011283103E004EB451101F50A71AC
:1032F00001228A700870E809487094F828040128AF
:1033000007D084F82824206803F09CF9680602D0CE
:1033100006E0022070BD04F22C41206803F05BF946
:10332000002084F8280470BD70B50D4601F07F04BC
:1033300000EB4411C1E90F2300224A64012281F805
:10334000292001F8284F6A06006803F0A0F9002040
:1033500070BD10B50446006803F07AFA000402D587
:10336000204601F0B5FB206803F072FA40050CD549
:10337000206830F8441F21F480610180204600F06D
:10338000EBF80021204600F0FCF8206803F060FA1A
:10339000400405D5206830F8441F21F480410180A5
:1033A000206803F055FA800405D5206830F8441FE2
:1033B00021F400510180206803F04AFAC00414D5BA
:1033C000206830F8401F21F004010180206830F8A7
:1033D000401F21F008010180204600F0CAF8206853
:1033E00030F8441F21F480510180206803F030FA46
:1033F00000051AD5206830F8401F41F0080101800F
:10340000206830F8441F21F400610180206830F802
:10341000401F41F004010180206803F019FAC04305
:10342000C00402D5204600F0E1F8206803F010FA4D
:10343000800508D5206830F8441F21F40071018010
:10344000204600F09AF8206803F002FAC00505D57E
:10345000206830F8441F21F48071018010BD2DE9EF
:10346000F04186B004004FF0000504D094F8290420
:10347000002620B108E0012006B0BDE8F08184F804
:103480002864204600F04AF8032084F829042068C4
:1034900003F09AF804F11001142288466846FDF7FB
:1034A00053FF94E80F0002F0F2FF0021206803F0C0
:1034B000E0F9012704EB451080F8297000F8285F37
:1034C0008581C670066146616D1C86610F2DF1D342
:1034D000002104EB411080F8296280F828128186CF
:1034E00080F82B62C0F83862C0F83C62491CC0F812
:1034F00040620F29EDD3142241466846FDF724FFB0
:1035000094E80F0003F051F884F8246084F82974DB
:10351000206803F048F80020AEE7000008B5006816
:103520000B49884212D10B48C16941F40001C161C5
:10353000C069002200F40000009011461420FFF73B
:10354000E7FDBDE808401420FFF7D6BD08BD000028
:10355000005C00400010024010B504460121D0F884
:103560005C0402F085FCD4F85C04BDE8104002F075
:103570004EBCD0F85C0402F069BCD0F85C0402F0E8
:103580006BBC10B5044690F8280401280BD001202C
:1035900084F8280484F82410206803F06CF90020D3
:1035A00084F8280410BD022010BDD0F85C2400F27D
:1035B0002C41104602F06FBC10B5044690F8280468
:1035C000012810D0012084F8280401462046FFF786
:1035D000EBFD206802F0E5FF206803F02BF90020E6
:1035E00084F8280410BD022010BD000010B5044668
:1035F000D0F85C0402F09CFCA069002804D00348C9
:10360000016841F00601016010BD000010ED00E00E
:103610002DE9F84304460078344FC00752D0F869CA
:103620000025C00008D4F86940F08050F861F869BE
:10363000012500F0805000902D480168C90511D483
:103640000168804641F480710160FFF7D5FC0646B1
:1036500004E0FFF7D1FC801B642822D8D8F80000D2
:10366000C005F6D5386A10F4407020D0A18801F466
:10367000407181421BD0386A1E49012220F44070FB
:103680000A6000220A603862C00710D0FFF7B4FC5D
:10369000064641F2883807E0FFF7AEFC811B414542
:1036A00002D90320BDE8F883386A8007F4D5386A68
:1036B000616820F44070084338621DB1F86920F059
:1036C0008050F8612078800705D57868A16820F4DB
:1036D0004040084378602078C00605D57868E168E6
:1036E00020F48000084378600020DBE700100240EF
:1036F00000700040400442422DE9F047DFF8348179
:1037000004460E46D8F8000000F00700B0420CD284
:10371000D8F8001021F007013143C8F80010D8F89C
:10372000000000F00700B04260D12078424F8007CF
:1037300005D57868A16820F0F0000843786020780B
:10374000C00742D06068012816D03968022816D018
:10375000890700294ADA796821F003010143796079
:10376000FFF74AFC0546606841F2883101280ED017
:103770000228894617D024E039688903E9E78901DE
:10378000E7E7FFF739FC411B494501D916E08946B7
:103790007868C0F381000128F3D116E0FFF72CFC14
:1037A000411B49450AD87868C0F381000228F5D149
:1037B0000BE0FFF721FC411B494502D90320BDE87E
:1037C000F087786810F00C0FF3D1D8F8001040465D
:1037D00001F00701B1420BD9016821F00701314323
:1037E0000160006800F00700B04201D00120E6E768
:1037F0002078400705D57868E16820F4E060084348
:1038000078602078000706D57868216920F4605038
:1038100040EAC100786000F03BF87968074AC1F3DC
:103820000311515CC840064908600020FFF704FC02
:103830000020C4E7002002400010024092CA0008A5
:10384000A80000200148006870470000A800002080
:103850000448054900684968044AC1F30221515CE3
:10386000C8407047A800002000100240A2CA00080B
:103870000448054900684968044AC1F3C221515C03
:10388000C8407047A800002000100240A2CA0008EB
:1038900012A085B00FC88DE80F0014A0144B00686B
:1038A00004905968134801F00C02042A10D0082A29
:1038B0000ED1C1F38342C9031DF802000AD559682D
:1038C00004AAC1F34041515C0A4A5043B0FBF1F0F5
:1038D00005B0704708494843FAE7000002030405B1
:1038E000060708090A0B0C0D0E0F1010010200004C
:1038F0000010024000127A0000093D002DE9F84F47
:1039000004460078B64DC00747D06868C0F3810010
:10391000012807D06868C0F38100022809D16868CF
:10392000C00306D52868800337D5606800286ED0AC
:1039300033E06068B0F5803F0BD010B1B0F5A02F38
:1039400011D0286820F480302860286820F4802076
:1039500002E0286840F480302860606888B1FFF792
:103960004BFB064609E0286840F480202860F0E719
:10397000FFF742FB801B642873D828688003F7D5C3
:103980000BE0FFF739FB064604E0FFF735FB801B31
:103990006428F1D828688003F7D42078DFF84482BF
:1039A00080074FF0010A4FF0000939D5686810F020
:1039B0000C0F07D06868C0F38100022809D168683D
:1039C000C00306D42868800713D5206901281ED1BA
:1039D0000FE02069A8B1C8F800A0FFF70DFB06466C
:1039E00004E0FFF709FB801B0228C5D82868800780
:1039F000F7D52868616920F0F80040EAC100286026
:103A00000EE0C8F80090FFF7F7FA064605E0E5E09B
:103A1000FFF7F2FA801B022823D828688007F7D422
:103A2000207800072CD57049A069D8B1C1F800A052
:103A3000FFF7E2FA064604E0FFF7DEFA801B0228F1
:103A40000FD8686A8007F7D568484FF4FA510068C4
:103A5000B0FBF1F0009000BF0098411E0091FAD237
:103A60000EE07CE0C1F80090FFF7C6FA064604E0DD
:103A7000FFF7C2FA801B022871D8686A8007F7D462
:103A8000207840075BD5E8690027C00008D4E869C2
:103A900040F08050E861E869012700F08050009014
:103AA00053480168C90511D40168834641F4807107
:103AB0000160FFF7A1FA064604E0FFF79DFA801BBC
:103AC00064284CD8DBF80000C005F6D5E068012872
:103AD0000AD008B1052813D0286A20F00100286216
:103AE000286A20F0040002E0286A40F00100286201
:103AF000E06841F2883B88B1FFF77EFA064609E0AC
:103B0000286A40F004002862EEE7FFF775FA811B8F
:103B100059455BD8286A8007F7D50BE0FFF76CFAA8
:103B2000064604E0FFF768FA811B59454ED8286A1B
:103B30008007F7D41FB1E86920F08050E861E069A0
:103B4000A8B36968C1F38101022947D00228484619
:103B500006D0C8F86000FFF74FFA044639E035E0B8
:103B60004746C8F86000FFF747FA064604E0FFF74B
:103B700043FA801B022829D828688001F7D4206ADC
:103B8000B0F5803F05D16868A16820F40030084393
:103B90006860D4E908010843696821F47411084396
:103BA0006860C7F860A0FFF727FA044605E013E055
:103BB000FFF722FA001B022808D828688001F7D5F1
:103BC0000AE0FFF719FA001B022802D90320BDE81A
:103BD000F88F28688001F4D40020F8E70120F6E788
:103BE000001002400000424280044242A80000202F
:103BF00000700040704770B5040005D00025A56234
:103C000094F8510010B104E0012070BD204600F08E
:103C100033F8022084F851002068016821F0400147
:103C20000160D4E901010843D4E9031211430843B8
:103C300061690843218B01F400710843E16908437D
:103C4000216A0843A16A084321680860A069042129
:103C500001EA1040616A0843216848602168E06A0F
:103C600008612068C16921F40061C16165650120B6
:103C700084F85100002070BD30B505460068184931
:103C800085B0884229D11748816941F4805181610A
:103C90008069694600F480500490A02000900220C2
:103CA0000190032003901048FFF7BCF8104C0F4818
:103CB000002120601020C4E901018020C4E9030133
:103CC0006161A1612046E161FEF78EFF18B1CD214F
:103CD00008A002F019FEAC64656205B030BD0000BA
:103CE0000030014000100240000801403000024056
:103CF000CC3A00202E2E2F5372632F73746D333203
:103D0000663178785F68616C5F6D73702E63000058
:103D100070B5044690F850000026012809D0012013
:103D200084F8500094F851000025012803D00226A1
:103D30003FE0022070BD89B182B1032084F85100B8
:103D400065652163A286E286A56365642564A5870F
:103D5000E587A068B0F5004F02D006E0012628E014
:103D60002068016841F480410160A16C1348C86279
:103D7000A16C13488862A16C12480863A06C45636B
:103D8000E38E2268216B0C32A06CFEF75FFF206887
:103D90000168490603D4016841F0400101602068D0
:103DA000416841F0200141602068416841F0020112
:103DB000416084F85050304670BD00003750000814
:103DC0004150000815500008704770474FF0E0213F
:103DD0000428086903D020F004000861704740F00F
:103DE0000400FAE7704710B5401EB0F1807F01D3A0
:103DF000012010BD4FF0E02460610F21601700F03A
:103E000057FE0020A06107202061002010BD10B5E2
:103E1000FFF7E8FF10BD30B590F83C20012A20D014
:103E2000012380F83C30022280F83D20026854686B
:103E300024F070045460026854680D682C43546088
:103E40000268946824F08004946002689468496869
:103E50000C43946080F83D30002180F83C10084607
:103E600030BD022030BD10B5040003D094F83D00F1
:103E700010B107E0012010BD002084F83C0020466E
:103E800000F00CF8022084F83D00211D206801F0AC
:103E9000D9F9012084F83D00002010BD08B5006864
:103EA0000649884208D10648C16941F00201C16152
:103EB000C06900F00200009008BD0000000400404E
:103EC00000100240022180F83D1001680A6842F0AB
:103ED00001020A60012180F83D100020704701684E
:103EE000CA6842F00102CA600068016841F001013D
:103EF000016000207047022180F83D1001680A6AC5
:103F000041F211131A4207D10A6A9B101A4203D1D7
:103F10000A6822F001020A60012180F83D100020A9
:103F2000704770B5044690F83C00012817D0012571
:103F300084F83C50022084F83D002068826822F01A
:103F4000770222F47F4282600868502836D00DDC68
:103F5000202858D005DC80B3102840D150E0022042
:103F600070BD302852D0402839D13EE060282DD095
:103F700070280BD0B0F5805F03D0B0F5005F2ED174
:103F800010E02068816821F0070109E0CB68D1E9E1
:103F90000121206801F08CF92068816841F07701E7
:103FA00081601CE0CB68D1E90121206801F080F933
:103FB0002068816841F48041F2E71EE0CA684968E0
:103FC000206801F087F95021206806E0CA68496836
:103FD000206801F090F96021206801F073F984F8FD
:103FE0003D50002084F83C0070BDCA6849682068D4
:103FF00001F070F940212068EFE700212068ECE72C
:1040000010212068E9E720212068E6E730212068B8
:10401000E3E7704770B5026804461068D1685369D9
:1040200010F00F0F50D003F0010501F490763543E6
:104030005DD0C20705D0CA0503D5E26B42F001028C
:10404000E263420705D5DA0703D0E26B42F00202D1
:10405000E263820705D5DA0703D0E26B42F004027F
:10406000E263020705D5DA0703D0E26B42F00802EB
:10407000E263E26B002A33D0800604D5880602D5BD
:10408000204601F0CDF920684069E16BC0F3801053
:10409000090700D428B3204601F0ABF92068416934
:1040A00049061AD5416921F040014161606BA0B118
:1040B0001B494163606BFEF79FFC002810D0606BCA
:1040C000416BBDE870400847830610D58B060ED5BE
:1040D0002046BDE8704001F0A3B92046FFF799FFE4
:1040E00070BD2046FFF795FF0020E06370BD03061A
:1040F00006D50B0604D52046BDE8704001F094BA01
:104100004006F3D54806F1D5D168204621F040019C
:10411000D160202184F8391000F03EFB70BD000012
:104120001B53000870B5040004D094F83900002532
:1041300010B106E0012070BD84F83850204600F030
:1041400023F8242084F839002068C16821F4005144
:10415000C160204601F0B0F92068016921F4904166
:1041600001612068416921F02A0141612068C1682C
:1041700041F40051C160E563202084F8390084F8DF
:104180003A00002070BD0000F0B5044600682C49DC
:1041900085B0884252D12B48816941F480418161C8
:1041A0008069294E00F4804004904FF40070009024
:1041B000022001900320039069463046FEF732FE4C
:1041C00030150025CDE900050120029069463046F2
:1041D000FEF728FE1E4E1D488027C6E90005C6E9E9
:1041E000025735617561B5613046F561FEF7FCFC3B
:1041F00020B140F23B1117A002F086FB66637462A7
:1042000012481B4E143801C61020A1C6184846F8A3
:1042100010597561B561F561FEF7E6FC20B140F219
:104220004B110CA002F070FB2663002211462520E2
:104230007462FEF76DFF2520FEF75EFF05B0F0BD4E
:1042400000380140001002400008014058000240C0
:10425000103B00202E2E2F5372632F73746D333258
:10426000663178785F68616C5F6D73702E630000F3
:10427000543B002037B5044690F83A0082B013460C
:1042800020283AD1039AAAB3A3B394F8380001289E
:1042900033D0012084F83800A262A3850025E563AD
:1042A000222084F83A00616B15488862616B1548DA
:1042B000C862616B14480863606B45632168606B7A
:1042C000091DFEF7C3FC206801684168009184F86D
:1042D0003850C16841F48071C1602068416941F083
:1042E000010141612068416941F0400141610020C4
:1042F00005B030BDFFE70120FAE70220F8E7000033
:1043000075530008B15300082B5300082DE9F05FE6
:10431000DFF8CC93002609F1180A09F5B67835467E
:10432000F04FB9E1F048805DF04AB97E5054491C25
:10433000C9B2B9762E2804D0002858D00A28FCD05B
:10434000A9E1092953D35018093802F0A9FCE6481D
:104350000222E749C83800F0DFF9F87E0028ECD0E7
:104360000A2844D2DFE800F043F1F0E0C6B8A744E1
:1043700005EF788E20F4004078861E20B87097F8FC
:104380003800F870B88D20B9388E10B1388EB885E5
:104390003D86B87A000903F011FCDFF844B300242D
:1043A0000BF1300BF98E4BF82410CD494FF07E50B5
:1043B000183941F8240001F1780020F8145049F828
:1043C00024504AF824502046FDF7E2F90022C94B58
:1043D000FDF761F9C84AC94BFDF7E8F8FDF715FA92
:1043E000BF49483141F82400641C062CDADB51E156
:1043F000788E20F400407886388F0A21B0FBF1F2E5
:1044000001FB1202FA70B0FBF1F0B870FD86F8788B
:104410003871F878B44900EB4000503901EB4000A6
:10442000F863B878152802D0B878162802D14FF46E
:104430000060F886388D10B1B88D28B106E0388E4E
:1044400040B1388E388505E0388EB885788D08B94A
:10445000388E78853D86022003F0B0FB06F0FEFA28
:10446000DFF87CB200240BF1300BF98E4BF82410EE
:104470009B494FF07E50183941F8240001F1780033
:1044800020F8145049F824504AF824502046FDF7EB
:104490007FF90022974BFDF7FEF8974A974BFDF7FF
:1044A00085F8FDF7B2F98E49483141F82400641CC3
:1044B000062CDADBEEE0B8781F2807D0B8781E2883
:1044C000388F4FEA900005D23885E3E0388F8008B6
:1044D000B88550E07885DDE0B8781E2805D097F8DB
:1044E0003800874909300870D4E0388FC0F1FA00ED
:1044F000F885CFE0788E20F4004078861F20B870D1
:10450000388F602800D38020F871387E40F0010099
:104510003876B88D20B9388E10B1388EB8853D8682
:10452000022003F04BFBB5E0388F0B280AD2DFE8FE
:1045300000F0B1060D113756585B64667200FD86B7
:1045400002F030FBA6E08FE075E08AE0FD8600F027
:1045500057F99FE0B8781F2808D0B8781E28388E01
:1045600012D0C8B1388E38853D8693E0388E38B188
:10457000388EB8853D86387E40F00100387689E077
:10458000B88D3886BD85F6E710B1388E7885EBE7B3
:10459000788D38867D857DE0388D38863D8579E05B
:1045A000B8781E2876D20020414600E0401C00EB7F
:1045B00040028A5CFF2A02D05028F7DB6AE05028CC
:1045C00068DAFA78BB7800EB400002EBC3020A54C9
:1045D0004B4A127840444270797981705AE07D7577
:1045E00058E00120787555E0788E20F400407886F8
:1045F0001F20B8708020F871BDE7424818E042489B
:10460000FFF779FC04F086FF404800F0D9F83E48F7
:10461000FFF765FC3EE00020FF22434600EB40012F
:10462000401C5A54194450284A708A70F6DB3848A6
:1046300000F003FC2EE0388F0028788E0ED040F476
:1046400000407886BD8698F80000C208BA7000F075
:104650000700F87098F8020078711BE020F4004021
:1046600012E097F83800F7E7B8781E280ED01F2818
:1046700026D0788E00F400407886388F798EC0EB93
:10468000001001EB0010F030788603E097F8380056
:10469000801C7872BD76761C787E8642FFF642AE2C
:1046A000B87E092190B1092800D9BD76B87EB0FB4B
:1046B000F1F201FB120038B1C0F10900787606E092
:1046C00097F83800387256E7797600E079767A7E86
:1046D000BDE8F05F0449A1F1C800FFF7CBBD0000C1
:1046E0002C3800200C000020BC0300201A360020CB
:1046F000F4C5000800004240CDCCCCCCCCCCEC3F83
:104700006100002000FC0008B4020020983900205D
:1047100000F8000870470000F7B5044690F839002B
:10472000202831D1019969B362B394F83800012887
:104730002AD0012084F838002162A284E284002576
:10474000E563212084F83900236B10489862236BBD
:104750000F48D862236B0F481863206B13464563DC
:104760002668206B321DFEF771FA21686FF0400059
:10477000086084F838502068416941F08001416147
:104780000020FEBD0120FEBD0220FEBDBB5300087F
:10479000E95300082B53000870477047FEE70000FC
:1047A000064A002102EB8103D3F8003840F821309B
:1047B000491C89B23C29F5D30120704700F000085C
:1047C00070B50E4E0546304600F037FBFEF716FB7F
:1047D000002404CD06EB840100230220FEF7CCFA6E
:1047E00018B1FEF7BFFA002070BD641CA4B23C2CC7
:1047F000EFD3FEF7B7FA012070BD000000F8000803
:1048000030B500202F4A014622F81010401C06281F
:10481000FADB2D4C0F211222A08C1E2378282FD0DA
:1048200010DC4FF00A05482820D006DC1E2817D0DF
:10483000322817D03C2811D116E05A281AD0642803
:104840000CD11BE0B42823D004DC90281CD096287F
:1048500004D11BE0C82820D0D82820D0A38407E0AA
:10486000322008E03C2002E048200AE05A20A084E0
:10487000617417E06420A084657413E078200FE071
:104880009020A08462740DE09620F0E7B420F8E751
:10489000C820A0841420607404E0D820F1E7F02040
:1048A000A0846374607C04F0B5FCA08C617CB0FBD8
:1048B000F1F1E1740621B0FBF1F12175BDE8304062
:1048C00006F004BF8C3800200C000020FEB5124911
:1048D000002405468C60CC600E484C6108600126BF
:1048E0000E614FF400204C60C8610846FDF726FFBA
:1048F00000B1FEE7012D09D00094CDE901646946BD
:104900000548FDF7C9FD002802D0FEE70096F4E750
:10491000FEBD0000002401402C020020F0B5074637
:104920002B4885B0816941F010018161816901F0F6
:1049300010010491816941F020018161816901F0D8
:1049400020010491816941F004018161816901F0D4
:1049500004010491816941F00801816180691D4C65
:1049600000F008004FF460450490002229462046DC
:10497000FEF73CFB0095012502266946204603967A
:104980000195FEF74FFAE80300248DE831006946EF
:104990001148FEF747FA40F20120CDE90004012F4B
:1049A00011D0022F11D002940C4E69463046FEF70A
:1049B00039FA40F2FA508DE8310069463046FEF788
:1049C00031FA05B0F0BD0296EEE70295ECE7000083
:1049D000001002400010014000080140000C01409E
:1049E0000E4810B50C4901604FF4827141600021FE
:1049F0008160C1604FF400720161C0E905121022AC
:104A0000C0E90721416281620A21C162FFF7F3F820
:104A1000002800D0FEE710BD003001405C020020FD
:104A200010B5134886B011490024C0E9001440F2C3
:104A30006161C0E9024104618461FFF714FA00B1C9
:104A4000FEE74FF48050009069460948FFF769FA85
:104A500000B1FEE72020CDE9040404A90448FFF7D3
:104A6000DAF9002800D0FEE706B010BD00040040CF
:104A7000B402002010B500220849094801F085F869
:104A80000849074801F081FA0749054800F0C6FEC9
:104A9000BDE81040024801F0C5BA000064000020E3
:104AA000184600208801002098000020FEE770478B
:104AB0000907090E002806DA00F00F0000F1E020D7
:104AC00080F8141D704700F1E02080F80014704752
:104AD0002DE9FC5F04460020ADF80000ADF80400AD
:104AE00040F68F7B4FF006094FF0020A4FF48068C2
:104AF00084E1BDF8001011F00F0628D030F8261020
:104B0000ADF80410BDF80410090475D530F826106E
:104B100001EA0B0120F8261004EB461595F8320245
:104B200005F50A750028206867D0297830F821201B
:104B3000B0F8503052047CD50AEBC1015A1808EB8A
:104B40004201415A8F05BF0D74D0EA88C7E0BDF815
:104B50000010C9062CD4018848F60F72114001805C
:104B6000206804F12805B0F850202B780AEBC30127
:104B70000A4408EB4201405AC0F309006064E16B4B
:104B80000844E06300212046FEF70FFB94F8240060
:104B90000028ADD0A8690028AAD194F82400216883
:104BA00040F08000A1F84C00002084F8240025E1AA
:104BB000018804F50A75ADF80410BDF80410090564
:104BC0001CD5B0F850202B7809EBC3010A4408EB40
:104BD0004201405A04F22C41C0F30903EB61AA8858
:104BE000206801F038FE2068018801EA0B0101808D
:104BF0002046FEF7DAFC01E195E054E0BDF8041030
:104C00000904D4D5018801EA0B0101802068B0F8BD
:104C100050202B78464609EBC301114408EB4101B3
:104C2000405A83059B0DEB610BD0AA886969206807
:104C300001E04AE057E001F00EFEE96968690844C6
:104C4000686100212046FEF7B7FA2068B0F85010DE
:104C5000891D06EB4101421828693E280CD9C0F392
:104C60004F11C00601D1491E89B24FF6FF7000EA0C
:104C7000812040F4004009E0C0F34F01C00701D09B
:104C8000491C89B24FF6FF7000EA8120106020684D
:104C900001884BF68F72114081F4405148F2800236
:104CA00011430180AAE0B0F850202B7809EBC30132
:104CB0000A4408EB4201415A8F05BF0D1FD0AA8854
:104CC0003B46696901F0C7FD19E009EBC1015A18BB
:104CD00008EB4201415A8F05BF0D04D02A893B469B
:104CE000696901F0B8FD2978206830F8212048F67C
:104CF0008F731A4048F2C0031A4320F82120E86954
:104D00003844E8616869C2196A61AB6913B12869FE
:104D1000B84204D929782046FEF74EFA03E02978F4
:104D20002046FEF7BFFABDF80400000666D52068ED
:104D300004EB461530F8261048F60F72114020F8A3
:104D4000261095F8320028350028206812D02978DE
:104D500030F82120B0F8503052061ED50AEBC101C0
:104D60005A1808EB4201405A83059B0DEB6123D092
:104D7000EA881DE0B0F850202B780AEBC3010A4402
:104D800008EB4201405A83059B0DEB6120D0AA88B5
:104D90006969206801F075FD1AE009EBC1015A1834
:104DA00008EB4201405A83059B0DEB6104D02A8930
:104DB0006969206801F065FD2978206830F82120B4
:104DC00048F68F731A404CF280031A4320F82120D2
:104DD0002068B0F850202B780AEBC3010A4408EB96
:104DE0004201405AC0F30900E86169690A186A6122
:104DF0002978AB69204663B1FEF796FA2068B0F8CF
:104E00004410ADF8001009043FF573AE0020BDE872
:104E1000FC9FFEF7CAF9F1E7054A0649002032F87F
:104E2000023B401C21F8023B1828F8DB70470000C9
:104E300000F400086C030020704710B586B00446EB
:104E4000FDF7DCFF0121002003918DE8130004A988
:104E50006846FDF733FF10B1FDF784FF04E0FDF76E
:104E600081FF0498401C02D0002006B010BD012034
:104E7000FBE7000000B588B0684600F043F8002862
:104E80003AD0BDF800000DF10201A0F50742653AE5
:104E900032D11A48BDF8022082849DF80420827025
:104EA0009DF80520C2709DF8062002719DF807202C
:104EB0004271134BBDF808201A70BDF80A204286D3
:104EC000BDF80C200285BDF80E2042859DF810200B
:104ED000C2719DF8112002729DF8122042749DF853
:104EE000132042758A7C4272CA7C82728A8AC28589
:104EF000CA8A8285097E817108B000BD0C0000203D
:104F00006100002010B51021164C0A4604EB411335
:104F10005208D3F8003C5B1C01D0114400E0891A10
:104F200089B2002AF2D104EB4112D2F8002C521CB3
:104F300001D1491E89B2202901D3002010BD0022D1
:104F4000490101EB82032344D3F8003C40F82230AE
:104F5000521C92B2082AF4D30068401CEED0012003
:104F600010BD000000F000082DE9F04106461024B5
:104F70001E48214600EB44124908D2F8002C521C6E
:104F800024D0621894B20029F4D100EB4410D0F878
:104F9000000C401C01D0641CA4B2154F202C03D37C
:104FA0003846FFF74AFF0024FDF728FF002564017B
:104FB00004EB850004CEC11900230220FDF7DCFEBE
:104FC00058B1FDF7CFFE0020BDE8F08111B1621AA3
:104FD00094B2CFE7641EA4B2D7E76D1CADB2082D22
:104FE000E6D3FDF7BFFE0120EEE7000000F0000869
:104FF00000FC000838B50B460092044600228021D0
:1050000000F04BF8002804D0606D40F0200060658F
:10501000032038BD10B5406A01684A6822F00302D7
:105020004A60416D41F010014165012180F8511045
:10503000FEF7E0FD10BD10B5406AFEF7C6FE10BDDC
:1050400038B50546446AFDF7D7FF02462868006870
:1050500080061ED42068416821F00201416064216D
:105060002046FFF7C7FF18B1606D40F02000606573
:10507000A068002118B92068C26880680090E186A5
:10508000012084F85100606D18B12046FEF7B2FD92
:1050900038BD2046FEF798FE38BD2DE9F0411D468B
:1050A00017460E460446DDF8188035E0681C33D0FC
:1050B0002DB1FDF7A1FFA0EB0800A8422CD320687A
:1050C000416821F0E00141606068B0F5827F0BD15A
:1050D000A068B0F5004F02D0B0F5806F04D1206811
:1050E000016821F040010160A06AB0F5005F0AD1BB
:1050F000206801684DF6FF72114001602068016868
:1051000041F400510160012084F85100002084F82E
:1051100050000320BDE8F0812068806836EA000076
:1051200004D00020B842C1D10020F3E70120F9E704
:105130007047000010B5FDF765FFFEF768FE0D49EA
:105140000878401CC0B20870CB780022984204D97D
:105150000A70887840F0010088704878401CC0B21E
:105160004870122804D94A70887840F0020088708C
:1051700010BD00005E00002030B593B0012108048E
:10518000CDE900100024029402250491CDE90750D6
:105190004FF4E01009906846FEF7B0FB00B1FEE75F
:1051A0000F20CDE90A054FF48060CDE90C404FF4A3
:1051B000A0600E9002210AA8FEF79EFA00B1FEE759
:1051C00012200F904FF48040CDE911040FA8FEF794
:1051D0001FFA00B1FEE7FEF735FB4FF47A71B0FB22
:1051E000F1F0FEF700FE0420FEF7F0FD002211466C
:1051F000501EFDF78DFF13B030BD00000D48016853
:1052000041F00101016041680B4A114041600168B1
:105210000A4A11400160016821F48021016041685F
:1052200021F4FE0141604FF41F0181600449C00375
:1052300008607047001002400000FFF8FFFFF6FE14
:1052400008ED00E0F0B50268164C174D174E4FF010
:105250008047A04205D0B84203D0A84201D0B04256
:1052600003D122F070034A681A43A04205D0B84225
:1052700003D0A84201D0B04203D122F44073CA68DF
:105280001A434B6922F08002134303608A68C262AA
:105290000A688262A04201D109690163012141616A
:1052A000F0BD0000002C0140000400400008004058
:1052B00010B5846842EA032224F47F440A4322435F
:1052C000826010BD826822F070020A4342F007013A
:1052D0008160704710B5046A036A23F0010303621A
:1052E000836923F0F00343EA021324F00A020A431D
:1052F0008361026210BD10B5036A23F010030362DC
:105300008469036A24F4704444EA023223F0A0035F
:1053100043EA01118261016210BD10B5406A0021AB
:10532000C185C184FEF775FE10BD70B5446A206862
:10533000406994F83910C0F3C0100025212904D128
:1053400018B1E584204600F062F82068406994F8BE
:105350003A10C0F38010222904D118B1E585204607
:1053600000F047F8E06B40F01000E0632046FEF7E5
:1053700050FE70BD10B50146406A0968096889068B
:1053800013D40021C1850168CA6822F48072CA6002
:1053900001684A6922F001024A6101684A6922F003
:1053A00040024A61202180F83A10FEF7AFFF10BD9D
:1053B00010B5406AFFF7AEF910BD10B50146406A5E
:1053C0000968096889060CD40021C18401684A690A
:1053D00022F080024A610068C16841F04001C1606A
:1053E00010BDFFF7D9F910BD10B5406AFFF7D5F928
:1053F00010BD0168CA6822F49072CA6001684A69E7
:1054000022F001024A61202180F83A1070470168B9
:10541000CA6822F0C002CA60202180F839107047A3
:1054200010B590F83A10222901D0022010BD8168F1
:10543000B1F5805F11D00169002901681FD049686A
:1054400001F07F03816A4A1C82620B70C18D491E84
:105450000904090CC18518D02BE00269816A002A71
:105460000268526805D0D2B20A80816A491C816202
:10547000ECE7C2F308020A80816A891CF7E74A68F0
:10548000816A4B1C83620A70E0E70168CA6822F0F7
:105490002002CA600168CA6822F48072CA6001688A
:1054A0004A6922F001024A61202180F83A10FEF791
:1054B0002DFF002010BD00002DE9F04104460068DA
:1054C0000169E26821F4405111430161A16820693A
:1054D0000143606901432068C26841F20C639A434A
:1054E0000A43C26020684169A26921F440711143F6
:1054F00041614C4920686426322788423CD1FEF73E
:10550000B7F900EBC00101EB001061688900B0FB46
:10551000F1F5FEF7ADF900EBC00101EB0010616899
:10552000B8468900B0FBF1F0B0FBF6F06FF018015F
:10553000484305EB800107EB0110B0FBF6F000F0EB
:10554000F005FEF795F900EBC00101EB0010616872
:105550008900B0FBF1F0B0FBF6F005EB0015FEF7AB
:1055600087F900EBC00101EB001061688900B0FB16
:10557000F1F7FEF77DF93BE0FEF76AF900EBC001B9
:1055800001EB001061688900B0FBF1F5FEF760F9EE
:1055900000EBC00101EB00106168B8468900B0FB68
:1055A000F1F0B0FBF6F06FF01801484305EB800115
:1055B00007EB0110B0FBF6F000F0F005FEF748F93C
:1055C00000EBC00101EB001061688900B0FBF1F055
:1055D000B0FBF6F005EB0015FEF73AF900EBC00161
:1055E00001EB001061688900B0FBF1F7FEF730F9BC
:1055F00000EBC00101EB001061688900B0FBF1F025
:10560000B0FBF6F06FF01801484307EB800108EBA0
:105610000110B0FBF6F0216800F00F00284488600C
:10562000BDE8F0810038014090F83910212901D0FF
:10563000022070478168B1F5805F016A0BD04A1C77
:105640000262026809785160C18C491E0904090C84
:10565000C1840ED017E009880268C1F308015160C7
:1056600001690029016A02D0491C0162ECE7891C2A
:10567000FBE70168CA6822F08002CA600068C1685E
:1056800041F04001C1600020704700000148FEF772
:10569000C1BC0000F4020020D0F8180220B10021A3
:1056A000C0F81412084670470220704770B50546CE
:1056B000D0F8184200F028FBC4F80C02D5F8180204
:1056C00048B1D5F81C12D4F80402CA6804F5037175
:1056D0009047002070BD022070BD70B504460025C3
:1056E000812100F077FA0121204600F073FA82212F
:1056F000204600F06FFAD4F8180250B1D4F81C021A
:1057000004F5067440688047206800F091FD002091
:105710002060284670BD10B5D0E9864159B194F893
:105720000002FF2807D08B6894F801222146984791
:10573000FF2084F80002002010BD00000A21018033
:1057400000487047B00000204321018000487047A6
:10575000000100204321018000487047BC00002068
:105760004321018000487047440100202DE9F041A9
:105770000546007C00264FF4007770B340230222D8
:105780008121284600F020FB4023022201212846E7
:1057900000F01AFB082303228221284600F014FBA4
:1057A0004FF4077000F046FDC5F81802F0B104464A
:1057B000D5F81C02006880470021C4F81412C4F810
:1057C0001812287CD4F8042290B1402301212846E5
:1057D00000F00DFB3046BDE8F081FFE73B460222BA
:1057E0008121284600F0F0FA3B46CEE70126F1E79A
:1057F0003B46EBE710B5D0F8181269B1027C002ADD
:10580000D1F8042205D04023012100F0F0FA002055
:1058100010BD4FF40073F7E7022010BD02460220CE
:10582000002902D00020C2F81C127047D0F81802DC
:10583000C0F8041200207047D0F81802C0F81022F7
:10584000C0F808120020704770B50646D0F818520C
:1058500008780C4610F0600121D0202927D1E28879
:10586000AAB10006607807D5D6F81C128B682946C5
:105870009847E288294617E085F80002A07985F864
:105880000102E2882946304600F050F80FE0D6F8D1
:105890001C12607800228B682146984707E06078E8
:1058A0000A2804D103490122304600F059F80020AB
:1058B00070BD0000AC00002010B5D0F8181289B1FE
:1058C000D1F814220AB1012010BD0122C1F814221E
:1058D000B1F8102293B2D1F80822812100F031FBF7
:1058E000002010BD022010BD10B5D0F8142252685F
:1058F0009047002010BD134610B50A46002100F065
:1059000076FA002010BD134610B50A46002100F0BB
:1059100018FB002010BD10B50446802100F0E8FA05
:105920002046BDE81040002100F0E2BA10B5032384
:10593000C0F80821C0F8F431C0F80C2113460A461B
:10594000002100F054FA002010BD10B505210023FD
:10595000C0F8F4111A46194600F049FA002010BDAB
:1059600010B502238261C0F8F431C26113460A46C1
:10597000002100F0E6FA002010BD10B5042100233C
:10598000C0F8F4111A46194600F0DBFA002010BDE9
:1059900010B50A46024903A000F0D4F8004810BD33
:1059A000983B002043444320436F6E6669670000C4
:1059B00012200880004870478400002010B50A4675
:1059C000024903A000F0BEF8004810BD983B00203B
:1059D00043444320496E746572666163650000004C
:1059E00004200880004870478000002010B50A4657
:1059F000024903A000F0A6F8004810BD983B002023
:105A000053544D6963726F656C656374726F6E6930
:105A10006373000010B50A46024903A000F092F833
:105A2000004810BD983B002053544D333220566936
:105A3000727475616C20436F6D506F72740000005A
:105A400010B50A46024903A000F07CF8004810BDDA
:105A5000983B002030303030303030303030314101
:105A600000000000F8B5044648880D46010A0829E0
:105A70004BD2DFE801F04A0409174A4A4048D4F8FB
:105A80001012207C0A6832E0207C02260028D4F81C
:105A9000140205D0C16A684688470146467041E055
:105AA000816AF8E7C0B206282FD2DFE800F00308C9
:105AB0000D12171CD4F81012207C4A6817E0D4F895
:105AC0001012207C8A6812E0D4F81012207CCA6878
:105AD0000DE0D4F81012207C0A6908E0D4F8101206
:105AE000207C4A6903E0D4F81012207C8A69694658
:105AF0009047014616E0207C38B9D4F81402416B77
:105B000068468847F5E7207C20B129462046FFF704
:105B100002FFF8BDD4F81402016B684688470146BD
:105B200007204870BDF800000028F2D0EA88002A5B
:105B3000EFD0824200D90246ADF800202046FFF7A0
:105B40000FFFF8BD70B5002300281DD004460025C6
:105B500002E06D1CEDB2641C2678002EF9D10224FF
:105B600004EB45041480CC545B1C0322CA5400246B
:105B70005B1C06E0CA545B1CDAB28C54521CD3B2D4
:105B8000401C0278002AF5D170BD10B580B1D0F864
:105B9000143213B10023C0F8143209B1C0F8101246
:105BA000012180F8FC11027000F0B2F8002010BD55
:105BB000022010BD10B50024D0F82002FDF724FB10
:105BC00030B1012801D0022801D0022400E00124D4
:105BD000204610BD10B50024D0F82002FDF7F4FADD
:105BE00030B1012801D0022801D0022400E00124B4
:105BF000204610BD2DE9F0411746044641B1D4F8C6
:105C0000140242698AB394F8FC01032842D043E0AD
:105C1000D4F8F411002504F11400022933D1D0E99D
:105C200002639E4207D9F31A83609AB2394620462E
:105C3000FFF769FE12E04068B0FBF3F103FB1101CE
:105C4000A1B9984212D3D4F8F81188420ED200229A
:105C500011462046FFF757FEC4F8F85100231A46B4
:105C60001946204600F0C3F80DE012E0D4F8140203
:105C7000C16829B194F8FC01032801D12046884766
:105C80002046FFF762FE94F80002012804D184F850
:105C9000005201E0204690470020BDE8F08170B539
:105CA0001546044641B1D4F8140282693AB394F817
:105CB000FC01032824D025E0D4F8F41104F5827007
:105CC00003291FD1D0E902318B420BD95B1A8360C3
:105CD0000846834200D303469AB229462046FFF77E
:105CE0000AFE0FE0D4F81402016929B194F8FC010E
:105CF000032801D1204688472046FFF73EFE01E0F9
:105D000020469047002070BDD0F82002FDF7A0BAD1
:105D100010B504461E481F49C0F85C44C4F8200270
:105D2000016008214160022181600021C160816120
:105D3000C1610162FDF793FB20B14FF4977116A08A
:105D400000F0E2FD0022D4F820021823114604F5E9
:105D50000874FDF70FFA5823002280212068FDF710
:105D600009FAC023002281212068FDF703FA4FF4CD
:105D70008873002201212068FDF7FCF94FF480733D
:105D8000002282212068FDF7F5F9002010BD0000F7
:105D9000B83F0020005C00402E2E2F5372632F75F9
:105DA0007362645F636F6E662E6300000A06D0F84C
:105DB000200201F07F0100EB411002D590F82A008B
:105DC000704790F82A02704770B51D4613460024AC
:105DD000D0F820022A46FDF743FA30B1012801D05D
:105DE000022801D0022400E00124204670BD10B535
:105DF0000024D0F82002FDF755FA30B1012801D077
:105E0000022801D0022400E00124204610BD70B514
:105E10000022044640231146FFF7D6FF40252B46BB
:105E2000002280212046C4F81051FFF7CDFF012049
:105E3000256284F8FC01D4F8180228B1D4F81402C1
:105E40002179426820469047002070BD90F8FD11EE
:105E500080F8FC110020704710B590F8FC11032960
:105E600004D1D0F81412C96901B18847002010BDCF
:105E700001740020704710B50024D0F82002FDF70F
:105E800080FB30B1012801D0022801D0022400E0BB
:105E90000124204610BD70B5044600F50270054689
:105EA00000F05FF80120C4F8F401B4F80E02C4F861
:105EB000F80194F8082212F01F000AD001280DD032
:105EC000022810D002F08001204600F011F80020D6
:105ED00070BD2946204600F0AAF8F8E7294620467A
:105EE00000F08CF9F3E72946204600F019F9EEE7B7
:105EF00010B50024D0F82002FDF7EBF930B10128ED
:105F000001D0022801D0022400E00124204610BD67
:105F100010B50024D0F82002FDF74EFB30B1012867
:105F200001D0022801D0022400E00124204610BD47
:105F300090F8FC1180F8FD11042180F8FC1100207C
:105F4000704710B50024D0F82002FDF7EDF930B10C
:105F5000012801D0022801D0022400E001242046BB
:105F600010BD0A7802704A7842708A78CB7802EBCA
:105F7000032242800A794B7902EB032282808A79DC
:105F8000C97902EB0121C18070470246002011B19E
:105F9000C2F8141270470220704710B5D0F81422CE
:105FA00002241AB11268904700B90024204610BD9F
:105FB00070B50D461A4E897804463170012928D8EB
:105FC00094F8FC01022802D0032822D105E099B1FF
:105FD0000320616084F8FC0109E091B160688842A7
:105FE0000AD0C1B22046FFF77FFC317861602046BD
:105FF000FFF7D3FF02280CD02046BDE87040FFF722
:10600000BCBC022084F8FC0120466160FFF76CFCF8
:10601000F2E729462046BDE87040FFF77CBC00004F
:10602000C001002010B5FFF773FF002010BD2DE95F
:10603000F04100274A7801263B460A2A43D2DFE88E
:1060400002F03C584251420805422A27FFF70AFD58
:1060500063E004468888C8B9C888B8B9887800F071
:106060007F0594F8FC01032810D084F8FE512946DE
:106070002046FFF700FF2046FFF77FFC1DB10220FE
:1060800084F8FC0149E084F8FC6146E020461AE00F
:10609000FFF78EFF41E0CA88012A14D190F8FC2155
:1060A000022A02D0032A0ED104E0012200F10801E5
:1060B000836014E00122011D11E090F8FC21022A06
:1060C00004D0032A02D0FFF726FC26E0C660D0F8F1
:1060D000041209B10321C160022200F10C01FFF793
:1060E0003FFC1AE004464888012816D1C4F804622F
:1060F0000BE0044690F8FC01022801D00328C5D12A
:106100004888012809D1C4F80432D4F814028268FE
:10611000204690472046FFF730FC3846BDE8F08126
:1061200070B50D460446287800260979C0F3411061
:10613000012806D06878A0B301281FD003283FD1DA
:1061400007E0D4F8140229468268204690470020D0
:1061500070BD94F8FC01022817D003282CD1688860
:1061600028B921B1802902D02046FFF7C1FED4F81A
:106170001402294682682046904713E094F8FC01F7
:10618000022802D0032817D103E0C9B180291BD10E
:1061900016E06888A0B9480604D02046FFF70AFD3B
:1061A000E5E703E02046FFF7E8FB09E094F8FC018F
:1061B000022807D003280BD029462046FFF7ABFB67
:1061C000304670BD4806FBD02046FFF791FEF7E74A
:1061D000080601F07F0004EB001501D5143501E03D
:1061E00005F582752046FFF7E1FD00B1012028602A
:1061F000022229462046FFF7B3FBE1E770B50546CA
:1062000090F8FC010C4603280DD1207901280AD80A
:10621000D5F81402826828469047E08830B92846AD
:10622000FFF7ABFB02E02846FFF775FB002070BDCF
:106230007047000000487047983D00202DE9F04766
:10624000CB780A7848F68F1433B1012B67D0022B34
:1062500008D0032B0BD17FE030F82230234043F4E9
:10626000007302E030F82230234020F822300A7810
:1062700030F8224048F68F731C4048F280052C43CA
:10628000144320F822408A7A48F6BF794FF0040C74
:106290004BF68F7A48F2C0044CF28007F2B30A78CA
:1062A00030F8226048F280181E4046EA080620F8BE
:1062B0002260CA88B0F8506022F0010291F8008094
:1062C00006EBC80600EB4606C6F800240A89B0F8BB
:1062D000506022F0010291F800800CEBC80C66447B
:1062E00000EB4606C6F800244A78002A0A7830F8FF
:1062F00022604FEA46467DD0002E05DA30F8226053
:106300001E403E4320F822600A7830F8226076066C
:1063100008D530F822601E40264301E028E021E045
:1063200020F822600A7830F822401C403C4320F8D4
:1063300022400A7830F8223003EA09032B4320F880
:106340002230097830F8212002EA0A022A4320F894
:1063500021200020BDE8F08730F82230234043F4AC
:10636000C06382E730F82230234043F480637CE747
:106370004A78002A8A8822F001021BD0B0F85060C7
:106380000F7806EBC70600EB4606C6F800240A782D
:1063900030F82260760605D530F822601E4026438C
:1063A00020F82260097830F8212002EA090282F000
:1063B0002002CBE7B0F850400E780CEBC606344410
:1063C00000EB4404C4F80024B0F850200C780626F2
:1063D00006EBC404224400EB42060A694FF6FF7C38
:1063E00006F580663E2A0CD9C2F34F14D20603D1BB
:1063F000641E00E021E0A4B20CEA842242F40042D0
:1064000007E0C2F34F04D20701D0641CA4B20CEA27
:10641000842232600A7830F82240640405D530F8CE
:1064200022401C403C4320F82240097830F82120CB
:1064300002EA0A0282F4405288E7002E05DA30F8B8
:1064400022601E403E4320F822600A7830F8226025
:10645000760605D530F822601E40264320F82260DB
:106460000A7830F822601E40264320F822600A781D
:1064700030F8223003EA0A0383F440532B4320F818
:106480002230097830F8212002EA09025EE7002074
:1064900070472DE9F04391F80A804C780A7848F665
:1064A000BF794BF68F7748F2800548F2C0064CF270
:1064B000800C48F68F73B8F1000F2AD0002C30F80A
:1064C00022404FEA444449D0002C06DA30F82240FA
:1064D0001C4044EA0C0420F822400A7830F822409C
:1064E000640605D530F822401C40344320F8224091
:1064F0000A7830F822401C4044EA0C0420F822407C
:106500000A7830F8223003EA09032B4320F82230BE
:106510001AE0002C30F822400DD0640605D530F882
:1065200022401C40344320F82240097830F82120D2
:1065300002EA09020CE0640406D530F822401C404F
:1065400044EA0C0420F82240097830F821203A402F
:106550002A4320F821200020BDE8F083002C06DA31
:1065600030F822401C4044EA0C0420F822400A780B
:1065700030F82240640605D530F822401C403443F0
:1065800020F822400A7830F822401C40344320F89A
:1065900022400A7830F822303B402B4320F822304A
:1065A000C3E7002070470020704700B50121A0F824
:1065B00040100021A0F84010A0F84410A0F850109E
:1065C00000F038F9002000BD30F8401F21F43D41B3
:1065D0000180002070470020704730B54C780A7861
:1065E000002C48F68F7530F8224048F2800312D014
:1065F000640607D530F822402C4048F2C0052C43F1
:1066000020F82240097830F8212048F6BF74224053
:1066100082F0300211E0640407D530F822402C40AB
:106620004CF280052C4320F82240097830F82120D4
:106630004BF68F74224082F440521A4320F82120F6
:10664000002030BD10B50A7848F2800352B1497875
:10665000002930F8221010D048F6BF74214081F094
:1066600010010FE001884BF6BF72114081F4805198
:1066700081F010011943018007E04BF68F7421402F
:1066800081F48051194320F82210002010BD2DE91B
:10669000F0410D460646896995F801C00023AA7AA3
:1066A000022728690C4648F28008BCF1010F05D08A
:1066B000814252D90446081AA8614FE0814203D9A9
:1066C0000446081AA86100E0AB617AB1287836F870
:1066D00020104906B6F8501007EBC000084406EB3E
:1066E0004000C0F8004412D52A8911E0A3B2AA885C
:1066F0003046696900F0C5F8B6F85000297807EB14
:10670000C101084406EB4000C0F800441CE0EA88E0
:10671000A3B23046696900F0B4F8687848F68F7221
:1067200010B1012807D00FE0287836F8201011406A
:1067300048F2C00205E0287836F8201011404CF2EB
:106740008002114326F82010287836F8201048F6E9
:10675000BF72114081F0300165E0AB6106234FF656
:10676000FF711AB1BCF1000F19D054E0B6F8500017
:106770002A783E2C03EBC202104406EB400202F5DD
:10678000806237D9C4F34F10E30630D001EA80208D
:1067900040F4004001E001EA802010603BE0B6F8E0
:1067A00050002A783E2C07EBC202104406EB400250
:1067B00002F580620BD9C4F34F105FEAC46C01D1BB
:1067C000401E80B201EA802040F4004008E0C4F39B
:1067D0004F005FEAC47C01D0401C80B201EA8020F7
:1067E000106068780028C1D001280AD013E0401E4C
:1067F00080B2CBE7C4F34F00E307CCD0401C80B29B
:10680000C9E7B6F85000297807EBC101084406EB48
:106810004000C0F80044287836F820104BF68F72FC
:10682000114081F4405141EA080126F8201000206F
:10683000BDE8F08130F8401F41F43F410180002065
:10684000704700000148FCF784BD0000B83F0020FD
:10685000B0F8440070475B1C00EB42005B0800F599
:10686000806005D030F8042B21F8022B5B1EF9D193
:1068700070470020704711B98021A0F84C1000200B
:10688000704710B55B1C00EB42005B0800F58060B0
:1068900009D011F8012B5B1E11F8014B42EA0422CA
:1068A00020F8042BF5D110BDFEE710B5C0F1FF01B3
:1068B000002355290AD2A1EB81041046641E64F31B
:1068C000070063F30F2001EB41010CE0AA290DD270
:1068D0001046553901EB410263F30700A1EB81013A
:1068E00062F30F20491E61F3174010BDAA3901EB76
:1068F00041041046A1EB810164F30700491E61F3D6
:106900000F2063F3174010BDFEE7490050EAC12095
:1069100018BF04204A0D18BF40F0010040F2FF727A
:10692000B2EB515F08BF40F00200012808BF05200C
:1069300070472DE9F0414F1E00EBC7010446D1E935
:10694000000115461E4637F006020DD02A46334692
:10695000FAF72FFE7F1E04EBC703D3E90023FAF7F3
:1069600081FD37F00602F1D1022F25D0042F13D07C
:10697000062F18BFBDE8F0812A463346FAF719FE04
:10698000D4E90A23FAF76EFD2A463346FAF711FED8
:10699000D4E90823FAF766FD2A463346FAF709FEDA
:1069A000D4E90623FAF75EFD2A463346FAF701FEDC
:1069B000D4E90423FAF756FD2A463346FAF7F9FDDF
:1069C000D4E90223FAF74EFD2A463346FAF7F1FDE1
:1069D000D4E90023BDE8F041FAF744BD0022134694
:1069E00010460149FAF757BE0000F03FFAF73ABDEA
:1069F0000022134610461146FAF74DBE40F201320E
:106A000000204FF0E041FAF7D1BF0000024A002019
:106A10001107FAF7CBBF000001FDFFFF02E008C835
:106A2000121F08C1002AFAD170477047002001E008
:106A300001C1121F002AFBD1704700000149086004
:106A400070470000C80100207FB5002405461D23C3
:106A5000224601A900F0D4F8002820DB2E18651E7C
:106A600016F8010B2C2819D107230022694630465D
:106A700000F0C6F8002812DB064416F8010B2C289B
:106A80000CD10523002203A9304600F0B9F80028F4
:106A900005DB304410F8011B2C2902D0284604B035
:106AA00070BDF023002202A900F0AAF811490028C5
:106AB000F5DB01E0641CA4B204EB4400085CFF2891
:106AC00001D0502CF6D3502C11D0BDF80000BDF8E9
:106AD000042000EBC20204EB44000A540844BDF851
:106AE00008204270BDF80C1081700020D7E76FF0CD
:106AF0000500D4E79839002000224FF0804100E0E3
:106B000089108142FCDC0CE05318834202DCC01A7D
:106B100002EB410202EBD272CB17521001EB9371E0
:106B200089100029F0D190B27047000030B50D49AE
:106B30000D4B0E4C31F8101033F81020657AB2EB83
:106B4000C51F03D9647AA2EBC41200E0002223F827
:106B5000102092B28A4202D223F8101000E01146AF
:106B6000084630BD3A340020F00100200C0000201F
:106B700018B51E230522694600F042F800280EDBF6
:106B8000074CBDF800006074607C02F043FBA08CF1
:106B9000617CB0FBF1F1E17404F098FD002018BDB8
:106BA0000C00002010B5154C607C0F281FD006DCAF
:106BB00005280AD006280AD00A2804D115E0122890
:106BC00017D0142817D0052002E0062000E00A2084
:106BD0006074607C02F01EFBA08C617CB0FBF1F164
:106BE000E174BDE8104004F071BD0F20F0E7122001
:106BF000EEE71420ECE71E20EAE700000C0000207E
:106C0000F0B5002425466FF02F0706E004EB84045E
:106C100007EB4404401C34446D1C0678A6F1300C8C
:106C2000BCF1090FF2D925B1944205DA6FF00200E8
:106C3000F0BD6FF00100F0BD9C4202DD6FF003007B
:106C4000F0BD0C8028B2F0BD1448C0784FF47061DC
:106C50000C2821D2DFE800F02006080A0D0F1214DC
:106C600017191B1E05F0D0BA7E2000E07F2005F02A
:106C700085B97E2000E07F2005F084BC7E2000E006
:106C80007F2004F05BBE05F0A7B804F0ADBE7F2006
:106C900004F024BE05F0CABB05F09CB90C0000202E
:106CA00010B501794279303901EB81036FF02F0182
:106CB00001EB43031A4402EB8202837901EB4202A7
:106CC0001A4402EB8202C37901EB42021A4402EB3E
:106CD0008202037801EB42021A4402EB82024378FB
:106CE00001EB42021A4402EB8202837801EB42027A
:106CF0001A4402EB8202C07801EB420108444FF4CF
:106D00007A7100F2134090FBF1F2642392FBF3F4EA
:106D100003FB14230A4A90FBF1F490FBF2F201FB0F
:106D200014004A43104490FBF3F090FBF1F3054A42
:106D3000D37690FBF1F301FB1300108710BD000028
:106D4000A08601000C00002008B54F2300226946F0
:106D5000FFF756FF0F4A00281BDB07E0B1F80330AE
:106D60000B804B798B70401CADF80000BDF8000023
:106D70004F2805D200EB40011144CB78FF2BEDD119
:106D800080B200EB4000FF2111541044417081702B
:106D9000002008BD983900202DE9F041644EA6F18D
:106DA000220530782A8D634901F5C074D1F8FC11B1
:106DB00002F0F4FA70782A8DE16F02F0EFFA687948
:106DC000002867D05B4F01287CD0022879D0287C2E
:106DD000411C2974802801D900202874287C60284F
:106DE0003ED9702002F006F807EB8008A88C401E00
:106DF00080B201F0FFFF298D8A08D8F8001002F058
:106E0000CDFA702001F0F6FF07EB8008A88C401E39
:106E100080B201F0EFFF298D8A08D8F8001002F047
:106E2000BDFA702001F0E6FF07EB8008A88C401E39
:106E300080B201F0DFFF298D8A08D8F8001002F037
:106E4000ADFA702001F0D6FF07EB8007A88C401E3A
:106E500080B201F0CFFF298D8A08396802F09EFACE
:106E6000A88C401E80B201F0C5FF3249C0B230701C
:106E7000FF22D1F8C01102F091FAA88C401E80B216
:106E800001F0B8FFC0B27070FF22216CBDE8F04184
:106E900002F084BAA88C401E80B201F0ABFF3070C3
:106EA000A88C401E80B201F0A5FF707030782A8D4A
:106EB0002049D1F8C01102F071FA70782A8DE4E708
:106EC00000E01EE0A88C401E80B201F093FF3070FD
:106ED000A88C401E80B201F08DFF70706F2001F011
:106EE00089FF07EB800130782A8D096802F056FA95
:106EF0006F2001F07FFF07EB800170782A8D096811
:106F0000C4E7702001F076FFB84607EB8007A88C35
:106F1000401E80B201F06EFF298D8A08396802F0A8
:106F20003DFA702001F066FF08EB80078EE7000055
:106F30002E00002000E8000808B5FF230022694663
:106F4000FFF75EFE002804DB0249BDF800008871EF
:106F5000002008BD0C0000201CB504461048437CEE
:106F60000022694620465B1EFFF74AFE002806DB2A
:106F7000204410F8011B2C2902D04FF0FF301CBD1B
:106F8000FF23002201A9FFF73BFE0028F7DB05499C
:106F9000BDF80020BDF80400885400201CBD00008E
:106FA0000C0000209C0300200D4AD18E491C89B2A0
:106FB000D186814212D30021D186D078072806D10C
:106FC0001079401CC0B21071062800D911711079D7
:106FD000044900EB400001EB4000D0637047000023
:106FE0000C0000206C030020084AD18E491C89B295
:106FF000D186814208D30021D1861079401CC0B2CD
:107000001071062800D91171704700000C00002093
:1070100070B50E46054600240BE055F8240001B279
:107020000014494300FB0010FFF766FD45F82400FB
:10703000641CB442F1DB701E012209E055F82210F5
:1070400055F82030401E1944491145F82210521CB1
:10705000B2EB560FF2DB70BD30B585B004464F235E
:10706000002202A9FFF7CCFD00282EDB25184FF0E7
:10707000FF3415F8010B2C2826D11D23002201A96D
:107080002846FFF7BDFD00281FDB054415F8010B5E
:107090002C2819D10723002269462846FFF7B0FDA6
:1070A000002812DB054415F8010B2C280CD1052310
:1070B000002204A92846FFF7A3FD002805DB284489
:1070C00010F8011B2C2902D0204605B030BDF0235A
:1070D000002203A9FFF794FD0028F6DBBDF80000AD
:1070E000BDF80410084A00EBC101BDF8080000EB30
:1070F000400011541044BDF80C104170BDF8101040
:1071000081700020E1E700009839002008B5FBF706
:1071100081FFFEF731F8FDF7ADFEF74EB08C717CC4
:10712000B0FBF1F1F1740621B0FBF1F03075707C29
:1071300002F070F8B08C04F0C9FAB0781F2803D1BF
:10714000307E40F001003076FDF766FEB07A00092F
:10715000FDF7E4FBE948416941F001014161406903
:10716000002200F00100009011460B20FBF7D0FF39
:107170000B20FBF7C1FF002211460D20FBF7C8FFD3
:107180000D20FBF7B9FF002211460E20FBF7C0FFD0
:107190000E20FBF7B1FF002211460F20FBF7B8FFCE
:1071A0000F20FBF7A9FFB07A00F00F00FDF78EFB70
:1071B000FDF716FCD348D249002701604FF4165161
:1071C000C0E901170C21C760C0E904718761C7617C
:1071D000FCF7A8FF00B1FEE7FDF722FCFDF74AFC33
:1071E000DFF8209309F1600989F80070F07809F15F
:1071F000180A00EB40010AEB41000024C24DF06385
:1072000009E005EB4400C82147700A2001F0E4FDC5
:1072100005F81400641CB08C8442F2DBBB48FDF717
:10722000BFFA90B1B9480178FF290ED1042101704D
:107230005821417087700E22C270017147710F2270
:107240008271C1710772FDF7BBFAAE494FF48062DB
:10725000D231A1F5CD70FBF749FB727EA949A9484F
:10726000C831FDF707F8A7484038FCF738FECB4691
:10727000DFF89C924FF0FF389BF80000002872D096
:10728000A04DADF800706035002415F8010B4128C1
:107290006AD115F8010B542866D115F8010B2B287B
:1072A00073D115F8010B41381A285DD2DFE800F0E0
:1072B0000D6E1554F8BEBEF711BEBED17BC0BEB177
:1072C000F6D98CC4DDBEBE88BED52846FFF7BCFB10
:1072D000AAE02846FFF7C0FEA6E02878532807D08A
:1072E000284604F0ADFA04B2002C7DDBF4700EE009
:1072F000681C072300226946FFF782FC041E05DD97
:10730000BDF80000F0701F20B07000E0EDDBF078F9
:10731000002500EB40010AEB4100F0630FE005EBB4
:1073200045014900B1FBF0F0F16B328D095C794801
:1073300050F82110284602F031F86D1CEDB2B08CE7
:107340008542ECD3B1781F2905D16E48F28C724981
:107350009838FCF7DDFCC0E02878412805D02846A5
:10736000FFF7F2FC60E00AE160E00020674BFF22DB
:1073700000EB4001401C5A54194450284A708A704E
:10738000F6DB6648FDF759FDA7E0D5E04FF48073C2
:10739000002269462846FFF733FC041E28DDBDF8AD
:1073A00000003085C8E04FF480730022694628460B
:1073B000FFF726FC041E1BDDBDF800007085BBE056
:1073C0002878312815D077754E484038FCF793FD62
:1073D0002878532810D0502811D0432813D0512892
:1073E00013D04446474800E079E04038FCF76AFD96
:1073F00073E001207075E7E702F08CF8F2E743488C
:10740000FDF7DEF9EEE7002000E00120FAF79CFE30
:10741000E8E72878502802D0432803D006E001F09E
:1074200025FC01E001F0B4FB04B256E0444656E00E
:10743000284601F0EDFFF7E7F0230A2269462846C7
:10744000FFF7DEFB041E48DDBDF8000089F80000F0
:1074500072E0284601F00EFF3EE0284604F026FACE
:10746000E2E7284601F024FDDEE7287830380728D7
:107470000DD2DFE800F004080C0C161B2000B07AD7
:1074800000F0F00002E0B07A40F00100B072B07895
:107490001E2814D0022000F091FB4DE012E043E0E2
:1074A00045E0B07A00F00F002030EFE7B07A00F04E
:1074B0000F001030EAE7B07A00F00F00E6E7B07A8C
:1074C0000009E8E728784E2811D0472828D0462818
:1074D000ACD1681CFFF730FD0446002C2CDAA41D4B
:1074E000062C4AD2DFE804F0443F3A35302B681CC2
:1074F000FFF73EFBF0E700000C0000200010024008
:1075000000380140F40200203A340020983900206D
:107510006100002000E80008C82B002000F80008E7
:10752000681CFFF719FDD7E704F0E4F87CE71022A8
:10753000F949FA48FDF7F0F80421F9481BE0F6484C
:107540002F21FC38FAF7EAFDF3481E21CB38FAF771
:10755000E5FDF1482021AC38FAF7E0FDEE481E21A8
:107560008B38FAF7DBFDEC481E216C38FAF7D6FDB4
:10757000E9484C214D38FAF7D1FD8BF80070E94805
:107580000178C907017875D021F001010170B07848
:107590001F280CD1307E032809D1F07901F088FF33
:1075A000DE48F28CE0499838FCF7B2FB3776B078C9
:1075B0001E28BFF461AEDD494FF480400861B07809
:1075C0001E2836D2DFE800F00F294A6C6F727478FB
:1075D0007B7E8184878A8D909396999B9FA1A3A699
:1075E000A9353535ACAFF078072813D2DFE800F0C5
:1075F00004040407090B0F0002F0C6F895E001200F
:1076000002E0022000E0032001F000FC8DE002F027
:10761000F1F88AE002F0D8F887E0F07807281AD26B
:10762000DFE800F004070A0D10131600FFF7B4FBA3
:107630007BE002F0FFF878E002F068F975E002F014
:10764000D9F972E002F0BEFA6FE002F0A9FB6CE03B
:1076500002F090FC69E001F003FC66E0F078072896
:107660001BD2DFE800F004080B0E1114170002F023
:10767000D1FD5AE060E002F051FE56E002F0FEFE5D
:1076800053E002F0A5FF50E003F0F2FF4DE001F0FF
:1076900083FB4AE001F064FB47E0FAF77BFE44E03D
:1076A000FAF734FB41E000F047F93EE0002000E04B
:1076B000012000F001FB38E003F01CFA35E003F094
:1076C00077FB32E003F04AFE2FE003F087FE2CE068
:1076D00003F0C4FE29E003F0DFFE26E003F040FFE4
:1076E00023E003F0FFFE20E003F028F81DE003F0A4
:1076F00021FA1AE003F0CCFA17E0112000E00F2085
:1077000003F03AFB11E00D20FAE70B20F8E703F055
:1077100063FB0AE003F044FC07E003F041FD04E0F2
:1077200003F0EEFD01E003F0B5F97C48F28C7E49F0
:107730009838FCF7EDFA9FE58907FCD5017821F030
:1077400002010170708E00042AD5B08E401CB086F4
:10775000708EB18EC0F30E00884221D2B786B06C15
:10776000C01CB0640078FF2804D17148B064007870
:10777000FF2841D0B06C0178C908B170017801F0E0
:107780000701F170427889F8002080787071F078F4
:107790003071307900EB40010AEB4100F063F7866D
:1077A000B08B401E0004000CB083C4D10520B08310
:1077B0006048016840F2FA508843002874DDF18B7C
:1077C000491C89B2F1830229B5D90121F18320280E
:1077D0005DD018DC022820D008286FD01028AAD14C
:1077E000B0781E28308C57D00028308D6AD02328DE
:1077F00072D9308D203870E0B770F770082089F8A2
:1078000000007771C3E740280AD0802819D0B0F56E
:10781000807F90D1FCF7F4FF2EE501F07BFE2BE595
:107820001E20B0707079401CC0B270710528F3D969
:107830007771F078401CF070F07800F00700F0707D
:107840001AE5B0781D2803D9B770F770777115E085
:107850007079401CC0B2707105280FD97771F0782B
:10786000401CC0B2F070072808D9F770B078401CEF
:10787000C0B2B0701D2800D9B770F786F0783071AB
:10788000307900EB40010AEB4100F063F4E4708EC4
:1078900080F400407086EFE40028708D05D0232826
:1078A0000ED9708D203807E02EE0E02802D2708DCE
:1078B000203001E04FF480707085DDE40FE001E0DE
:1078C0000320F9E7B0F5687F02D2308D203004E064
:1078D0004FF4707001E0FFE703203085CCE4308C7A
:1078E00099F800100028484604D00E2909D90178DB
:1078F000083907E0E82902D20178083102E0F021D6
:1079000000E008210170B7E4F08B10B1308CC04367
:107910003084F783B0E4000081CA0008F40200203C
:10792000F4C5000860000020C82B002000100140B2
:1079300098390020080C01402DE9F0479B4FF88E44
:10794000401C80B2F886B98C2331884220D30021B4
:10795000F986387858B13970F87807280AD07878DD
:10796000401CC0B27870012812D9797021E0012042
:107970003870F1E73879401CC0B23871062800D958
:10798000397138798A4900EB400001EB4000F86317
:10799000787870B1F86B45787879DFF81882864E80
:1079A000012809D0387810B17879022804D0002451
:1079B0003FE0F86B0578EFE700241CE00A2001F0B7
:1079C00019FA052816D938F814000A2801D8002019
:1079D00001E0A0EB900080B228F81400398D4843F4
:1079E000C0F30F22B88C56F82510001B401E80B241
:1079F00001F0D4FC641CB88C8442DFDB1CE00A205C
:107A000001F0F8F9052813D938F814000A2801D82C
:107A1000002001E0A0EB900080B228F81400398D1E
:107A20004843C0F30F22A0B256F8251001F0B6FC6F
:107A3000641CB88C8442E2DB78794FF0FF0930B1E6
:107A4000012825D002284FF0000475D142E000241F
:107A5000F88EB98C001B884215DAF88E001B12D400
:107A6000F88E021B28F81290F98E091B38F81100C5
:107A7000398D4843C0F30F22F88E56F82510001BAD
:107A800080B201F08BFC641C0A2CE1DBBDE8F087BE
:107A90000024F88E011BB88C814217DAF98E091B7D
:107AA00014D4FA8E131B28F81390F98E3A8D091B03
:107AB00038F81110FB8E5143C1F30F221B1BC01A63
:107AC000401E80B256F8251001F068FC641C0A2C98
:107AD000DFDBDBE7F88E011BB88C81421ADAF98E06
:107AE000091B17D4F98E0B1B28F813903A78AAB10A
:107AF000FA8E121B38F812103A8DFB8E5143C1F3E7
:107B00000F2206EB85011B1BC01A401E80B20968BC
:107B100001F044FC641C0A2CDCDBB7E7F88E398DDD
:107B2000001B38F810004843C0F30F22F88E06EB14
:107B30008501001BEAE7FFE7F88E011BB88C814244
:107B400030DAF98E091B2DD4FA8E131B28F8139006
:107B5000FA8E121B821A08EB420020F8029CF88E63
:107B6000011B38F81100398D06EB850A4843C0F334
:107B70000F22F88EDAF80010001B80B201F00EFC24
:107B8000F88E011B38F81100398D4843C0F30F22DD
:107B9000F88EBB8C001B181A401E80B2DAF8001059
:107BA00001F0FCFB641C0A2CC6DB6FE70C00002014
:107BB0006C0300203A34002000E800081FB540F2B2
:107BC0000121009100210191012807D0022807D04E
:107BD000029169460448FBF725F91FBD022000E029
:107BE00001200290F5E70000000C0140F0B5314D96
:107BF0000C46074669794FF0FF36062956D2DFE872
:107C000001F055030916193701F092FDA2B2394669
:107C1000002047E001F0CAFCA88CA2B24008394617
:107C200001F0BCFBA88CA2B206EB500038E001F0DA
:107C30001BFD2DE001F0E4FCA88CA2B280083946BF
:107C400001F0ACFBA88CA2B206EB900080B23946E2
:107C500001F0A4FBA88CA2B2800800EB40003946DA
:107C600001F09CFBA88CA2B2800800EB400016E05B
:107C700001F02AFDA88CA2B24008394601F08EFB23
:107C8000A88CA2B206EB500080B2394601F086FB08
:107C9000A2B23946002001F081FBA88CA2B2401E9E
:107CA00080B23946BDE8F04001F078BB01F058FDE4
:107CB000F3E700000C0000202DE9F041DFF8E88335
:107CC00098F80530424600245178F84D491C042BA1
:107CD000928CB8F83630C9B2C3F1000398F80F603F
:107CE00002EB83032ED2B3423CDC88F80F40B8F895
:107CF00036305B1C9BB2A8F83630B3EB920F31D311
:107D0000A8F8364088F80F4098F80330072B06D0C3
:107D100088F80110012925D988F801402BE098F84E
:107D20000410491CC9B288F80410062901D988F842
:107D3000044098F8041001EB410105EB4101C8F83B
:107D40003C100FE0B3420DDCB8F836309B0088F8E9
:107D50000F30B8F836305B1C9BB2A8F83630B3EB66
:107D6000D20FCDD298F8011029B1D8F83C104C7838
:107D7000097828B105E0D8F83C100C784978F8E784
:107D80007F2498F80500CA4E052876D2DFE800F077
:107D9000034685CBF9003746002506EB810607E050
:107DA000B8F828202846316801F0F8FA6D1CEDB2C9
:107DB000B8F83600B5EB800FF2D3B8F8360007EB11
:107DC00084048006050E07E0B8F8282028462168BC
:107DD00001F0E4FA6D1CEDB2B8F824008542F3D34B
:107DE00098F8240098F80F10401A401EC4B209E019
:107DF000844205D2B8F828202046316801F0CEFA36
:107E0000641CE4B2B8F8240098F80F10411AC91C99
:107E1000A142EDDC98F80F00401C80E0B8F8360075
:107E20003746404202EB8000C5B206EB810607E010
:107E3000B8F828202846316801F0B0FA6D1CEDB280
:107E4000B8F824008542F3D3002507EB840407E04B
:107E5000B8F828202846216801F0A0FA6D1CEDB280
:107E6000B8F83600B8F82410404201EB8000A84270
:107E7000EEDC98F80F40E41E09E0F9E0002C05DB89
:107E8000B8F82820A0B2316801F088FA641C98F88C
:107E90000F00401C8442F1DBBCE73746002506EBAF
:107EA000810607E0B8F828202846316801F076FA04
:107EB0006D1CEDB2B8F83600B5EB800FF2D3B8F810
:107EC000360007EB84048006050E07E0B8F828208A
:107ED0002846216801F062FA6D1CEDB2B8F8240062
:107EE0008542F3D398F8240098F80F10401A401EEA
:107EF000C4B209E0844205D2B8F82820204631688F
:107F000001F04CFA641CE4B2B8F8240098F80F10A1
:107F1000411AC91CA142EDDC98F80F00001D88F839
:107F20000F00BDE8F081B8F8360006EB810740424B
:107F300002EB8000C5B207E0B8F82820284639686F
:107F400001F02CFA6D1CEDB2B8F824008542F3D391
:107F5000002506EB840407E0B8F8282028462168AD
:107F600001F01CFA6D1CEDB2B8F83600B8F8241018
:107F7000404201EB8000A842EEDC98F80F40E41E7E
:107F800009E00EE0002C05DBB8F82820A0B2396823
:107F900001F004FA641C98F80F00401C8442F1DBE5
:107FA000BAE73746002506EB810607E0B8F8282037
:107FB0002846316801F0F2F96D1CEDB2B8F83600D0
:107FC000B5EB800FF2D3B8F8360098F82410404291
:107FD00001EB8000C5B207E0B8F8282028463168D8
:107FE00001F0DCF96D1CEDB2B8F824008542F3D342
:107FF000B8F8360007EB84048006050E07E0B8F8F1
:1080000028202846216801F0C9F96D1CEDB2B8F8A6
:108010003600B8F82410404201EB8000A842EEDCA4
:1080200098F80F4007E0B8F828202046316801F0A2
:10803000B5F9641CE4B298F80F00001D8442F2D335
:1080400098F8241098F80F00081A001FC4B207E02F
:10805000B8F828202046316801F0A0F9641CE4B289
:10806000B8F8240098F80F10401AA042F0DCD1E6CE
:108070003746002506EB810607E0B8F82820284699
:10808000316801F08BF96D1CEDB2B8F83600B5EB34
:10809000800FF2D3B8F8360098F82410404201EB74
:1080A0008000C5B20EE000000C0000206C03002030
:1080B00000E80008B8F828202846316801F06EF979
:1080C0006D1CEDB2B8F824008542F3D3B8F8360041
:1080D00007EB84048006050E07E0B8F82820284640
:1080E000216801F05BF96D1CEDB2B8F83600B8F804
:1080F0002410404201EB8000A842EEDC98F80F40CB
:1081000007E0B8F828202046316801F047F9641CE0
:10811000E4B298F80F00001D8442F2D398F82400CE
:1081200098F80F10401A001FC4B207E0B8F82820D2
:108130002046316801F032F9641CE4B2B8F824003A
:1081400098F80F10401AA042F0DCE5E62DE9F04D5A
:108150001D460C4698B0174621F0004123F000431D
:10816000002814BF4FF0010C4FF0000C0CEB440C36
:10817000FE4A0CEB02064FEA620C66452BD33E002A
:1081800018BF012606EB45061644F94A964222D34B
:10819000F84A53EA070C02D0944205D148B918B006
:1081A00000201146BDE8F08D002808BF4FF0000CFC
:1081B00001D04FF0010C0CEB440212F5001F0AD85D
:1081C000002F14BF4FF0010C4FF0000C0CEB4502D8
:1081D00012F5001F07D918B03A462B462146BDE8D4
:1081E000F04DFEF703BC0022DFF88CA3002CB8BFD3
:1081F000534526DADFF884C36345A8BF022220DA9C
:10820000DFF870C39C451CDCDFF874C30CEB235C07
:10821000BCF1140F08DDCCF1340627FA06FC0CFA89
:1082200006F6BE420DD108E05FB9CCF1140623FA80
:1082300006FC0CFA06F69E4203D10CF00102C2F1D4
:10824000020251EA000C19D1002D17DA002C18BFD8
:10825000022A01D0012A07D00220FEF7EFFB18B056
:10826000BDE8F04DFEF7BABB0220FEF7E7FBFEF7D4
:10827000B5FB18B081F00041BDE8F08DB7F1000CFE
:108280006CD1534525D104F1804212F5801201BF13
:1082900000280020B74918B008BFBDE8F08DB548E8
:1082A000884207DC002DA1BF6046294618B0BDE812
:1082B000F08D07E0281E05DA80F0004118B0604616
:1082C000BDE8F08DAF497944D1E9000118B0BDE8AF
:1082D000F08DDFF8A0C2634525D1002D1FDA19B15A
:1082E000514512D1D8B909E0002840F0EC82A24AE9
:1082F000214618B062F31E01BDE8F08D0020214632
:1083000018B060F31E01BDE8F08D08DA18B02346FE
:10831000BDE8F04D024600206146F9F7BCB918B03F
:108320002146BDE8F08D514518DAB5F1804F0DD0EA
:10833000A5F1005CBCF1FF5C10D1B4F1000C0DDBC9
:1083400018B06146BDE8F04D02F062BB234618B09C
:108350000246BDE8F04D1946F9F72BB9060024F0A6
:10836000004C3BD1D9B1514533D1002C06DD002D55
:10837000A1BF0020514618B0BDE8F08D002C01DDF2
:10838000002D1BDB002C13DA002D11DB012A4FF02E
:10839000000014BF78497C4918B0BDE8F08D022A6E
:1083A00018BF002C0AD0012A08D1002C06DA0AE0F6
:1083B000002CB8BF002D11DA012A04D0002018B01B
:1083C0000146BDE8F08D18B000204FF00041BDE837
:1083D000F08DA1F14050B0F17F601AD0012000EB88
:1083E000E47050EA020421D0624C521E4FF0000BA0
:1083F000104304BF4FF0000B644C654883427CDDA2
:10840000644A654893421FDD884217DB002D25DB57
:1084100037E0002C00DA4AB1022A0CBF01204FF0ED
:10842000FF3018B0BDE8F04DF9F7B2B90120FEF702
:1084300005FB18B0BDE8F04DFEF7DABA4D4A8A42A6
:1084400002DC002D0ADC1CE0814202DA002D18DA81
:1084500004E0484B994220DD002D12DD0220FEF79A
:10846000EDFAFEF7CBFA05460E4600225346584673
:108470002146F9F79EF818B066F31E012846BDE8BC
:10848000F08D0220FEF7DAFAFEF7C0FA0A4621461E
:1084900018B062F31E01BDE8F08D0022304661463F
:1084A000F9F781F880460E466FF00102F9F77EFA7F
:1084B0004FF05532394BF9F779F842463346F9F720
:1084C00078F80022364BF9F771F882464246334677
:1084D000049110461946F9F76CF85246049BF9F7D7
:1084E00068F88A4600904FF0C0422E4B4046314615
:1084F000F9F75FF82C4A2B4B00E027E0CDE90601A5
:1085000051460098F9F755F882460191274A284BC1
:1085100040463146F9F74DF85246019BF9F743F8CA
:1085200082460B4602460591DDE90601F8F79AFFFF
:10853000DDE90623002688463046F9F734F852462E
:10854000059BF9F733F8024600F07EB90020B1F53B
:10855000801F07DA352230466146F9F727FA0646CA
:108560006FF0340000EB215024E00000FFFF1F00FB
:10857000FFFF0F000000F03F0000F07F00004043CD
:1085800001FCFFFF6E4800000000F0FF0000F0BF9C
:108590000000E0410000F043FFFFEF3F5555D53F9D
:1085A0000000E03F4715F73FFE822B6544DF5DF892
:1085B0000BAE543EA0F2FF300190C1F3130040F027
:1085C0007F6141F040510291FE498842D8BF0020AE
:1085D00004DDFD498142C8BF012001DD0D9008E0A6
:1085E00000200D900198401C01900298A0F5801089
:1085F00002900299F54878440B910D9900EBC10067
:10860000D0E900230F9330460A920B99F8F7CBFF7D
:10861000CDE90601DDE90A2130460F9BF8F722FF7C
:1086200002460B460020EA49F9F735F80591024663
:108630000B460090DDE90601F8F7BBFF1490E54812
:108640008A464FF0000878440299006812904FF073
:10865000005040EA61010D980F9B01EB804000F54E
:10866000002109910A9A1298F8F79DFF32460B9B58
:10867000F8F79CFF42465346F8F79BFF06460291E7
:1086800040465146099B129AF8F793FFDDE906230D
:10869000F8F78CFF3246029BF8F785FF059B009A9E
:1086A000F8F787FF0091149A049053461046194634
:1086B000F8F77FFF06460246C7480B46029106219F
:1086C0007844FEF736F9CDE90510029B3246104694
:1086D0001946F8F76EFFDDE90532F8F76AFF0591F4
:1086E0000646534640461946149AF8F7BBFE009BCF
:1086F000049AF8F75EFF3246059BF8F7B3FECDE922
:1087000005104246534610461946F8F752FF00221C
:10871000B24B02910A90F8F7A5FEDDE90532F8F7B1
:10872000A1FE0E464246AD4B4046F8F73CFF029B89
:108730000A9AF8F738FFDDE90532F8F737FF4246C5
:1087400002910A90334610465146F8F732FFCDE9C0
:1087500006015346149A02990A98F8F72AFF8A46A6
:1087600002903346424600990498F8F722FF534698
:10877000029AF8F777FE82460B4602460591DDE93C
:108780000601F8F76FFEDDE906230020884606465D
:10879000F8F709FF5246059BF8F708FF8246099152
:1087A0004FF060428E4B30464146F8F702FF04908E
:1087B00006918C4A8A4B50460999F8F7FAFE824690
:1087C0000291894A894B30464146F8F7F2FE5246FB
:1087D000029BF8F747FE864B7B440D9A03EBC203DE
:1087E000D3E90023F8F73EFE0E9007910198F8F7C1
:1087F000CFFF0591DDE9061382460E9A0498F8F73B
:1088000031FE7C4A7A440D9B02EBC303D3E900237B
:1088100000930292F8F726FE5246059BF8F722FED7
:108820000026884652463046059BF8F7BCFE009B62
:10883000029AF8F7B8FE069B049AF8F7B4FE079B75
:108840000E9AF8F7B3FE024600200B460290384617
:108850002946F8F7AEFE824601912B463846194666
:10886000029AF8F7A0FE32464346F8F7A2FE5246B7
:10887000019BF8F7F7FD07468A46324643462946EC
:108880000298F8F796FE05460E463A465346F8F724
:10889000E9FD594A8846914221DBA8EB020353EADD
:1088A000000210D12A463346F8F77DFECDE90401D7
:1088B000524A534B38465146F8F7D4FDDDE90423BC
:1088C000F9F7E8F821D20220FEF7B8F8FEF796F89B
:1088D0000A46214618B062F31E01BDE8F08D494BEF
:1088E00028F000429A4210D3474A08EB020353EAA9
:1088F00000027FF4C6AD2A463346F8F754FE3A46E6
:108900005346F9F7C7F87FF6BCAD0022019228F074
:1089100000403E493E4A01EB2051824223DA481C86
:108920004FF4801121FA00F040443A4AC0F30A5152
:108930007A44394BA1F2FF31CB4020EA0303C0F364
:10894000130040F48010C1F11401C8401268019076
:10895000B8F1000FBCBF4042019028463146F8F7FD
:1089600022FE05460E462A46334638465146F8F75B
:1089700079FD4FF000084246284B40460591F8F734
:1089800018FECDE90601264A264B40460599F8F720
:1089900010FE009102902A46334640460599F8F7AA
:1089A00002FE3A465346F8F701FE1F4A1F4BF8F7FE
:1089B00000FE009B029AF8F755FD074688460246DE
:1089C0000B4635E08E9803007AB60B00B6440000E3
:1089D0000000F03FEE4400001C440000000008408E
:1089E00009C7EE3FFD033ADCF5015B14E02F3EBE04
:1089F000F4420000B842000000009040FE822B6567
:108A00004715973C00CC904000346F3F01FCFFFFBE
:108A10000000E03F04420000FFFF0F00432EE63F4E
:108A2000396CA80C615C20BEEF39FAFE422EE63F9D
:108A3000DDE90601F8F716FDDDE9062305460E46D9
:108A4000F8F7B1FD3A464346F8F7B0FD0F462A461F
:108A50003346009010461946F8F7ABFD82460246B1
:108A60002E4888460B4605217844FDF762FF5246A2
:108A70004346F8F79EFD2A463346F8F797FD8046B1
:108A80008A463B4628463146009AF8F792FD3B4617
:108A9000009AF8F7E7FC0691009000224FF080431F
:108AA00040465146F8F77FFD0F460C90424653462C
:108AB00028463146F8F77DFD3B460C9AF8F7EBFD6A
:108AC000069B009AF8F76FFD2A463346F8F76BFDD0
:108AD0000022134BF8F76AFD054601980E4601EB9C
:108AE00000510815002810DC28463146019AF8F795
:108AF0005DFFFDF70AFF042808BFFDF787FF284642
:108B00003146019AF8F752FF05460B4618B02A463F
:108B100058462146BDE8F04DF8F74BBDA440000093
:108B20000000F03F2DE9F047144A012402EB411CFC
:108B30000021134FDFF84C80DFF84C90DFF84CA099
:108B400018E000231A461CF8016006E057F824508C
:108B5000641C521C2B44A4B2D2B29642F6D8B8F888
:108B60002E20534319F80120521C53432AF8113088
:108B7000491CC9B28142E4D3BDE8F08700EC00088B
:108B8000C81B00200C0000209C0300203A34002069
:108B90002DE9F05F16211E48F9F7C0FA00274FF0C3
:108BA0003A0B1C4C3846214600F036F8194904446B
:108BB0000646002507EB470038314FF02C094FF0EF
:108BC000090A01EB40081FE0F5B104F8019B04F825
:108BD00001AB18F80500214600F01EF806446D1C94
:108BE000B61C0444062DEFDB0D2020700A206070B7
:108BF000B61CB1B20748F9F791FA0028F9D17F1CE9
:108C0000082FCEDBBDE8F09F04F801BBDFE70000D2
:108C10002CC600083403002010B5002263280DDDA7
:108C2000642290FBF2F390FBF2F2303301F8013B47
:108C30006FF018035A4300EB820001220A2309282F
:108C40000CDD90FBF3F4303401F8014B90FBF3F4AE
:108C5000644204EB840400EB4400521C90FBF3F4E8
:108C600003FB140030300870501C10BD2DE9F05F7C
:108C7000002412213748F9F751FADFF8DCB0354803
:108C80001A211330F9F74AFA0028F8D156E0334E8A
:108C900020463146FFF7C0FF0246B0183A2100F8DF
:108CA000011B092600F8016B8046785D02F1020A7B
:108CB000C0084146FFF7B0FF014608EB01004FF046
:108CC0002C0800F8018B00F8016B81460AEB0100CB
:108CD00000F1020A785D494600F00700FFF79CFFAB
:108CE000014609EB01003D4400F8018B00F8016BDF
:108CF00081460AEB010000F1020A68784946FFF755
:108D00008BFF014609EB010707F8018B07F8016BA0
:108D10000AEB0006A8783946B61CFFF77DFF01462E
:108D200078180D2202700A2275184270AD1CA9B283
:108D30000A48F9F7F3F90028F9D1641C502C06DA37
:108D400004EB44055F461BF80500FF289FD1002077
:108D5000BDE8F09FFEC500089839002034030020CC
:108D600030B50C4DE88E401CE886E88EC0B2E8862F
:108D700000240AE0E88EC0B2FDF797FD2A8D014677
:108D8000204600F00BFB641CA4B2A88C8442F1D3F3
:108D900030BD00000C00002030B50E4DE88E401CA8
:108DA000E886E88EC0B2E88600240EE02102B1FB1E
:108DB000F0F0E98E0844C0B2FDF777FD2A8D014638
:108DC000204600F0EBFA641CA4B2A88C8442EDD3D8
:108DD00030BD00000C00002070B50D460446F8F7C9
:108DE000A1FA291B491C90FBF1F201FB120020445F
:108DF00000B270BD10B50446F8F794FA641C90FBFD
:108E0000F4F104FB110080B210BD000070B5124DEA
:108E10007F24E97B11B1E97B491EE973E97B0E4EA2
:108E20004C3659B1E97B814200DA34780B48298D00
:108E300050F82400BDE87040FEF7D8BE00F10A01EA
:108E4000401C09B200B2FFF7C7FFE8733478632013
:108E5000FFF7D0FF3070E9E70C00002000E80008C1
:108E600070B5114CE07B0A2801D90120E073E07B4A
:108E7000401E10F0FF00E0730B4D05F14C0508D1CA
:108E80000A210320FFF7A8FFE0737320FFF7B2FF6A
:108E900028702878054901EB8000218D0068BDE825
:108EA0007040FEF7A3BE00000C00002000E80008A0
:108EB0002DE9F0410446AE48FBF71DF820784FF04D
:108EC000FF14AC49AC4F2504261231384FF6FF7C15
:108ED00005286ED2DFE800F0D4A16E360300FF2231
:108EE000002004C1401C02F580121028F9DB00208C
:108EF00010C1401C103C1028FADB002020C1401C8F
:108F000005F580551028F9DB002080C1401CA7F52D
:108F100080171028F9DB002040C1401C10361028B3
:108F2000FADB002041F804CB401CACF5805C102833
:108F3000F8DBFF22002004C1401C02F5801210283B
:108F4000F9DB02E13546002220C1521C05F58015EF
:108F5000102AF9DB002080C1401CA7F5805710289B
:108F6000F9DB4FF47F22002004C1401C103210288E
:108F7000FADB002010C1401CA4F580141028F9DB96
:108F8000FF22002004C1401C02F580521028F9DBAA
:108F9000002041F804CB401CACF1100C1028F8DB89
:108FA0003046002201C1521C00F58030102AF9DB46
:108FB000CBE097E02A46002004C1401C1032102864
:108FC000FADB002010C1401CA4F580141028F9DB46
:108FD000FF22002004C1401C02F580521028F9DB5A
:108FE000002041F804CB401CACF1100C1028F8DB39
:108FF000002040C1401C06F580161028F9DB002037
:1090000080C1401CA7F580571028F9DB002020C143
:10901000401C10351028FADB97E02B46002008C1D1
:10902000401C03F580531028F9DB002080C1401C50
:10903000A7F580171028F9DB002040C1401C10362E
:109040001028FADB002041F804CB401CACF5805C12
:109050001028F8DBFF22002004C1401C02F580121A
:109060001028F9DB002010C1401C103C1028FADB4E
:10907000002020C1401C05F580551028F9DB64E074
:109080003046002201C11030521C102AFADB0020A9
:1090900041F804CB401CACF5805C1028F8DBFF22C3
:1090A000002004C1401C02F580121028F9DB0020CA
:1090B00010C1401C103C1028FADB002020C1401CCD
:1090C00005F580551028F9DB002080C1401CA7F56C
:1090D00080171028F9DB002040C1401C10361028F2
:1090E000FADB32E0FF22002004C1401C02F580526E
:1090F0001028F9DB002041F804CB401CACF1100C27
:109100001028F8DB002040C1401C06F5801610280E
:10911000F9DB002080C1401CA7F580571028F9DB3F
:10912000002020C1401C10351028FADB002010C19F
:10913000401CA4F580141028F9DBFF22002004C194
:10914000401C02F580521028F9DB0C4B6FF07F4277
:10915000002004C1401C1A441028FADB0548F9F726
:1091600041F80348FAF7AEFE0020BDE8F0810000A8
:10917000B4020020C80B002000FFFF00EFEEEEFF5E
:109180002DE9F04D07460E46F8F728FC04460D463B
:109190003A463346F8F70AFADFF86CA0DFF86CB00D
:1091A0001B4B0746884616F0004F4FF000020AD0CE
:1091B000F8F758FC0AD900225B4638464146F8F7D2
:1091C00069FC1BD212E0F8F74DFC08D2002253468E
:1091D00020462946F8F7E7F904460D460EE000223E
:1091E0005B4638464146F8F755FC07D800225346FF
:1091F00020462946F8F736F904460D463146204602
:1092000065F31E01BDE8F08D0000F03F0000E03F77
:109210000000E0BF10B514490F281FD006DC052858
:109220000AD006280AD00A2804D115E0122817D03F
:10923000142817D0062002E0002000E001208874E6
:109240000A4A0B4B00208C7C02EB4414245C1C5417
:10925000401C1E28F7DB10BD0220F0E70320EEE7DC
:109260000420ECE70520EAE70C00002000F50008E8
:109270009C0300203CB50446F0231E226946FDF7FE
:10928000BFFC00286BDB2044062510F8011B424C74
:109290002C2965D0BDF800001E22B0FBF2F102FBC4
:1092A000110139B9B0FBF2F109B2CB0702D16274F6
:1092B00000295FDA1422B0FBF2F102FB110139B987
:1092C000B0FBF2F109B2CB0702D16274002951DA86
:1092D0001222B0FBF2F102FB110139B9B0FBF2F13D
:1092E00009B2CB0702D16274002943DA0F22B0FB26
:1092F000F2F102FB110139B9B0FBF2F109B2CB076F
:1093000002D16274002935DAB0FBF5F105FB1101D9
:1093100039B9B0FBF5F109B2CA0702D16574002969
:1093200028DA0A22B0FBF2F102FB110139B9B0FBD5
:10933000F2F109B2CB0702D1627400291ADA0521D1
:10934000B0FBF1F201FB12023AB9B0FBF1F000B24E
:10935000C20702D1617400280CDA6FF004003CBD32
:109360000723002201A9FDF74BFC0028F7DBBDF81D
:1093700004006074BDF80000A084607CFFF74AFF21
:10938000A08C617CB0FBF1F1E174B0FBF5F12175CB
:1093900002F09CF900203CBD0C00002030B54FF4D9
:1093A00080739A4200D91A46174B184C03EBC0033E
:1093B0001844C1F307235343C3F3072304EB4305C6
:1093C0002B441D7845705D7885709B78C370CBB257
:1093D0005343C3F3072304EB43052B44C1F3074175
:1093E0001D78057151435D78C1F30721457104EB88
:1093F00041029B78114483710A78C2714A780272E3
:109400008978417230BD0000C82B002000E00008C0
:109410003FB505461D2300226946FDF7F1FB0028F4
:109420003DDB204CBDF80010A170054415F8010B80
:109430002C2833D10723002201A92846FDF7E0FBA1
:1094400000282CDBBDF80410E170E178217121794E
:10945000154A01EB410102EB41010544E16315F8B6
:10946000010B2C281AD10523002202A92846FDF75A
:10947000C7FB002813DBBDF808106171284410F801
:10948000011B2C290AD1F023002203A9FDF7B8FB08
:10949000002804DB0549BDF80C000870002004B06A
:1094A00030BD00000C0000206C0300206100002093
:1094B00070B5164D802803D2154951F8206019E087
:1094C000287A4FF0E236C0F12001C6F30740401A77
:1094D00001D5002002E0FF2800DDFF2060F31746E1
:1094E000F0B2401801D5002002E0FF2800DDFF2087
:1094F00060F30706002405E0AA8DA0B23146FFF70D
:109500004DFF641CA88C8442F6DB70BD0C0000206B
:1095100000E8000800B589B048F26570ADF80000B9
:1095200020486946828CADF8022082788DF80420AC
:10953000C2788DF8052002798DF8062042798DF8E1
:109540000720194A1278ADF80820428EADF80A209B
:10955000028DADF80C20428DADF80E20C2798DF849
:109560001020027A8DF81120427C8DF81220427D65
:109570008DF81320427A0A75827A4A75C28DCA82A2
:10958000828D0A83807988760020C87640F2012097
:10959000888340F20340C8836846FBF7E5FC09B0C6
:1095A00000BD00000C0000206100002030B5124D0D
:1095B0000021681C114C4B1E03E0427A00F8012B7D
:1095C000491CA28C03EB520202EBC2028A42F4DC79
:1095D000A08C002100EBC000284404E010F8092C06
:1095E00000F80129491CA28C03EB520202EBC202D3
:1095F0008A42F3DC30BD0000C82B00200C000020A4
:1096000030B51748174D808C800800EBC001681CEE
:10961000002203E0437A00F8013B521C8A42F9DB46
:1096200005EB4102531C002403E0587A03F8010BB8
:10963000641C8C42F9DB002304E012F8090C02F8E8
:1096400001095B1C8B42F8DB05EB8100002204E082
:1096500010F8093C00F80139521C8A42F8DB30BD91
:109660000C000020C82B002030B5154C154D0021F2
:10967000A08C4B1E00EBC00005EB5000401C03E02B
:10968000427A00F8012B491CA28C03EB520202EB38
:10969000C2028A42F4DCA08C002100EBC00005EB82
:1096A000500004E010F8092C00F80129491CA28C94
:1096B00003EB520202EBC2028A42F3DC30BD00002F
:1096C0000C000020C82B002030B51748174C808CA8
:1096D000800800EBC00163185A1C002003E0557A93
:1096E00002F8015B401C8842F9DB01EB41000444B5
:1096F000601C002503E0427A00F8012B6D1C8D42AE
:10970000F9DB002004E013F8092C03F80129401CC0
:109710008842F8DB002004E014F8092C04F8012941
:10972000401C8842F8DB30BD0C000020C82B002014
:109730000A4B0949988C01EBC0010844002104E060
:1097400010F8092C00F80129491C9A8C521E02EBD2
:10975000C2028A42F4DC7047C82B00200C000020B3
:1097600007480021074B03E0427A00F8012B491C0F
:109770009A8C521E02EBC2028A42F5DC704700004E
:10978000C92B00200C00002010B50D4CE08E88B1D4
:109790007F200C4901EB8000218D0068FEF726FA3E
:1097A000E08E401C80B2E086E178884201D900203A
:1097B000E08610BD7020FFF71DFBC0B2E9E7000096
:1097C0000C00002000E80008084900B508790001F5
:1097D0005F2800DD1030064A098D52F82000FEF7A0
:1097E00005FA08205DF804EBFDF7FEBB0C00002035
:1097F00000E800080D49C88E401C80B2C8860828C1
:1098000001D90020C886C88E072807D2C88E000755
:10981000000E5F2803D91030C0B200E07F20044A58
:10982000098D52F82000FEF7E1B900000C0000207D
:1098300000E8000870B5334E314CF08E401C80B209
:10984000F086B18CB0EB910F08D90021F186B07D84
:10985000401CC0B2B0755F2800D9B175002534E056
:10986000607868B18108002902DD401A60701EE04E
:10987000401E10F0FF00607019D1F021282013E085
:109880002078401E10F0FF00207010D1F0217820C9
:10989000FFF7A2FA6070707901281AD002281CD054
:1098A000032822D05F210020FFF796FA207060780D
:1098B000318D4843020A2078134901EB8001A8B298
:1098C0000968FFF76BFDA41C6D1CB08C8542C7DBDB
:1098D00070BDB17DB07D1031E6E7C5EB4510B18CB0
:1098E00000EB851090FBF1F0E0E7C5EB4510B18C83
:1098F00000EB851090FBF1F0C0F15F00D6E70000AF
:109900003A3400200C00002000E800082DE9F04166
:10991000354FF88E401C80B2F886B98CB0EB910FB1
:1099200008D90021F986B87D401CC0B2B8755F28FF
:1099300000D9B97500242D4E50E006EB4405697836
:10994000A9B1491EC8B26870398D4843020A16F899
:109950001400274901EB8001A0B20968FFF71EFD42
:10996000687858BBF0215020FFF736FA33E016F83C
:10997000141069B3491E11F0FF0106F814102CD120
:109980007979012907D002290BD0032917D05F204C
:10999000FFF730FA0BE0B97DB87D1031FFF71CFA04
:1099A00005E0C4EB441101EB841191FBF0F006F8E3
:1099B00014007820FFF71EFA783068700DE0C4EBD1
:1099C000441101EB841191FBF0F0C0F15F00EEE770
:1099D0007320FFF70FFA06F81400641CB88C844259
:1099E000ABDBBDE8F08100000C0000203A34002021
:1099F00000E800082DE9F05F6F4E7279DFF8BCA136
:109A0000DFF8BC814FF01E096FF0010B0025D2B1C9
:109A10003046022A818C504600EB410002D0032AD6
:109A200047D135E0F27B521CF273F27B082A0AD947
:109A3000F573801E02E030F8022D4280491E002995
:109A4000F9DC20F8025C5D4C00271DE0617879B1FB
:109A5000B0FBF9F0C0F10E0001B25846FFF7BCF9B7
:109A6000617840B2814202DD081A607000E06570E2
:109A70006078318D48432178020AB8B258F8211035
:109A8000FFF78CFCA41C7F1CB08C8742DEDB37E028
:109A9000F27B521CF273F27B082A0AD9F573801EFE
:109AA00002E030F8022D4280491E0029F9DC20F83E
:109AB000025C424C002720E0617879B1B0FBF9F0FC
:109AC000C0F10E0001B25846FFF786F9617840B246
:109AD000814202DD081A607000E065706078318DA7
:109AE0004843020AB08C2178C01B401E80B258F84F
:109AF0002110FFF753FCA41C7F1CB08C8742DBDBDA
:109B0000F18E64200AEB4104FFF774F9142809D29E
:109B1000F0217820FFF760F960705F210020FFF7E7
:109B20005BF92070707950B3022828D06078318DAD
:109B3000F38E4843020A2078444608EB8001B08C3B
:109B40000968C01A401E80B2FFF728FCF08E401C46
:109B500080B2F086B18C884200D3F58680217020D7
:109B6000FFF73AF904EB8001B08CF28E801A401EA8
:109B7000328D80B20968BDE8F05FFFF70FBC6078F6
:109B8000318D4843020A2078444658F82010F08E60
:109B9000FFF704FCF08E401C80B2F086B18C884246
:109BA00000D3F58680217020FFF716F9328D54F826
:109BB0002010F08EDFE700000C0000203A34002077
:109BC00000E800082DE9F05F724E7279DFF8C8A155
:109BD000DFF8C8814FF01E096FF0010B0025D2B1EC
:109BE0003046022A818C504600EB410002D0032A05
:109BF00047D135E0F27B521CF273F27B082A0AD976
:109C0000F573801E02E030F8022D4280491E0029C3
:109C1000F9DC20F8025C604C00271DE0617879B126
:109C2000B0FBF9F0C0F10E0001B25846FFF7D4F8CE
:109C3000617840B2814202DD081A607000E0657010
:109C40006078318D48432178020AB8B258F8211063
:109C5000FFF7A4FBA41C7F1CB08C8742DEDB37E03F
:109C6000F27B521CF273F27B082A0AD9F573801E2C
:109C700002E030F8022D4280491E0029F9DC20F86C
:109C8000025C454C002720E0617879B1B0FBF9F027
:109C9000C0F10E0001B25846FFF79EF8617840B25D
:109CA000814202DD081A607000E065706078318DD5
:109CB0004843020AB08C2178C01B401E80B258F87D
:109CC0002110FFF76BFBA41C7F1CB08C8742DBDBF1
:109CD000F18E64200AEB4104FFF78CF8142804D2BB
:109CE000F0217820FFF778F86070707980B302284F
:109CF0002ED0F08EC0EB401101EB8010B18CB0FB88
:109D0000F1F0C0F15F00C0B220706178328DF38E47
:109D100051430A0A08EB8001B08C4746C01A401E26
:109D200080B20968FFF73AFBF08E401C81B2F186E1
:109D3000B08C814200D3F5862178F28E801A401EC5
:109D4000328D80B257F82110BDE8F05FFFF726BBD7
:109D5000F08EC0EB401101EB8010B18CB0FBF1F044
:109D6000C0B220706178328D474651430A0A58F8D4
:109D70002010F08EFFF712FBF08E401C80B2F086B0
:109D8000B18C884200D3F5862078328D57F82010A8
:109D9000F08ED9E70C0000203A34002000E80008DB
:109DA0002DE9F05F704E7279DFF8C0A1DFF8C08155
:109DB0004FF01E096FF0010B0025D2B13046022A88
:109DC000818C504600EB410002D0032A47D135E098
:109DD000F27B521CF273F27B082A0AD9F573801EBB
:109DE00002E030F8022D4280491E0029F9DC20F8FB
:109DF000025C5E4C00271DE0617879B1B0FBF9F0A0
:109E0000C0F10E0001B25846FEF7E6FF617840B29D
:109E1000814202DD081A607000E065706078318D63
:109E200048432178020AB8B258F82110FFF7B6FA71
:109E3000A41C7F1CB08C8742DEDB37E0F27B521C17
:109E4000F273F27B082A0AD9F573801E02E030F81B
:109E5000022D4280491E0029F9DC20F8025C434CA7
:109E6000002720E0617879B1B0FBF9F0C0F10E0075
:109E700001B25846FEF7B0FF617840B2814202DD80
:109E8000081A607000E065706078318D4843020AFE
:109E9000B08C2178C01B401E80B258F82110FFF70B
:109EA0007DFAA41C7F1CB08C8742DBDBF18E78200E
:109EB0000AEB4104F021FEF78FFF6070707980B3E8
:109EC00002282ED0F08EC0EB401101EB8010B18C37
:109ED000B0FBF1F0C0F15F00C0B220706178328D4C
:109EE000F38E51430A0A08EB8001B08C4746C01A32
:109EF000401E80B20968FFF751FAF08E401C81B213
:109F0000F186B08C814200D3F5862178F28E801ADA
:109F1000401E328D80B257F82110BDE8F05FFFF788
:109F20003DBAF08EC0EB401101EB8010B18CB0FB5C
:109F3000F1F0C0B220706178328D474651430A0A71
:109F400058F82010F08EFFF729FAF08E401C80B2EE
:109F5000F086B18C884200D3F5862078328D57F890
:109F60002010F08ED9E700000C0000203A340020C9
:109F700000E800082DE9F05FDFF88CA2BAF82410A1
:109F80009AF805204C08DFF884B24FF0000802B3BD
:109F900050469F4B808C022A03EB400002D0032ADC
:109FA00069D151E09AF80F205346521C8AF80F20CD
:109FB0009AF80F20082A0CD9424683F80F80801E99
:109FC00002E030F8023D4380491E0029F9DC20F808
:109FD000022C8F4D00265F46D14632E06878A8B14A
:109FE000B9F824101E20B1FBF0F0C0F10E0001B250
:109FF0006FF00100FEF7F0FE697840B2814202DDA9
:10A00000081A687002E0404685F80180B9F8281007
:10A01000C0B24843020A287807EB8001B0B2096851
:10A02000FFF7BCF96878B9F828104843020A287885
:10A0300007EB8001A01980B20968FFF7AFF9AD1CEA
:10A04000761CA642CADB4FE09AF80F205346521CFA
:10A050008AF80F209AF80F20082A0CD9424683F874
:10A060000F80801E02E030F8023D4380491E002927
:10A07000F9DC20F8022C664D0026D946574631E01F
:10A080006878A0B1B98C1E20B1FBF0F0C0F10E00D1
:10A0900001B26FF00100FEF79FFE697840B2814285
:10A0A00002DD081A687002E0404685F80180398DAB
:10A0B000C0B24843020AB88C2978801B401E80B287
:10A0C00059F82110FFF76AF96878398D4843020A78
:10A0D0002978A01B401E80B259F82110FFF75EF9C5
:10A0E000AD1C761CA642CBDB4948BAF83610564662
:10A0F00000EB4105F0217820FEF76EFE6870707964
:10A10000F0B302284AD0F08EC0EB401101EB801072
:10A11000B0FBF4F0C0F15F00C0B228706978328DF6
:10A12000F38E51430A0A0BEB8001B08C5F46C01AD4
:10A13000401E80B20968FFF731F96878318D4843D5
:10A14000020A287807EB8001F08E0968201A401E69
:10A1500080B2FFF723F9F08E401C80B2F086A04257
:10A1600001D3A6F836802878F28E07EB8001B08CF8
:10A17000801A401E328D80B20968FFF70FF900E0A7
:10A180000CE0287807EB8001F08E201A401E328DFB
:10A1900080B20968BDE8F05FFFF700B9F08EC0EB50
:10A1A000401101EB8010B0FBF4F0C0B22870697868
:10A1B000328D5F4651430A0A5BF82010F08EFFF79C
:10A1C000EDF86878318D4843020A287807EB800162
:10A1D000F08E0968204480B2FFF7E0F8F08E401C52
:10A1E00080B2F086A04201D3A6F836802878328D5E
:10A1F00057F82010F08EFFF7D1F8287807EB800190
:10A20000F08E2044C3E700000C00002000E80008A6
:10A210003A3400202DE9F0473D4E7079DFF8F49094
:10A220004FF00008012802D0707902280CD1B18CBF
:10A2300009EB4100801E02E030F8022D4280491EE9
:10A240000029F9DC20F8028C324C0025324F1AE04C
:10A25000607818B1810841D0401A60707079318DF2
:10A260000128607800FB01F04FEA1022207807EB0C
:10A27000800135D0B08C401B401E80B20968FFF7CA
:10A280008DF8A41C6D1CB08C8542E1DBF08E401C67
:10A2900080B2F086022838D9A6F836805F210020E7
:10A2A000FEF79AFD0446F021A020FEF795FD074633
:10A2B000B08C81080009FEF78FFD054610210220B1
:10A2C000FEF78AFD8046B08C0209401E01B210469E
:10A2D000FEF782FD81B209EB410012E0401EBCE7AF
:10A2E000A8B2CBE70470A41C24B247705F2C00DD39
:10A2F0000024491E6D1EA7EB080217B289B22DB2C9
:10A30000801E002901D0002DECDCBDE8F0870000A4
:10A310000C0000203A34002000E800082DE9F04746
:10A32000524F7879DFF848A14FF00009012815D97C
:10A33000F87B401CF873F87B08280FD94A4687F849
:10A340000F90B98C0AEB4100801E02E030F8023D0C
:10A350004380491E0029F9DC20F8022CDFF8148123
:10A36000002408F13006B98C36F8140088420BD16D
:10A3700058F82410002903DC401C26F8140032E0B1
:10A38000491E48F824102EE007D926F814904808F2
:10A39000FEF730FD48F8240002E0401C26F81400C7
:10A3A00036F8141078200AEB4105F021FEF714FD71
:10A3B0006870787968B102280BD036F81400C0EBC9
:10A3C000401101EB8010B98CB0FBF1F0C0F15F00DF
:10A3D00008E036F81400C0EB401101EB8010B98C96
:10A3E000B0FBF1F02870641C032CBCDB204C7879A6
:10A3F000214E18B1022801D0002531E0002512E0DD
:10A40000607818B1010913D0401A6070398DC0B25C
:10A410004843020A207806EB8001A8B20968FEF7DB
:10A42000BDFFA41C6D1CB88C8542E9DBBDE8F0873C
:10A43000401EEAE7607818B1010915D0401A607033
:10A44000398DC0B24843020A207806EB8001B88CEF
:10A450000968401B401E80B2FEF7A0FFA41C6D1CC3
:10A46000B88C8542E6DBE1E7401EE8E70C000020FF
:10A470003A3400205C38002000E800082DE9F05F45
:10A480004F4E7079DFF83CA14FF00009012815D933
:10A49000F07B401CF073F07B08280FD94A4686F801
:10A4A0000F90B18C0AEB4100801E02E030F8023DB3
:10A4B0004380491E0029F9DC20F8022C424FDFF8C6
:10A4C0000081002407F1300B08F14C083BF8140020
:10A4D000B18C5D4688420BD157F82410002903DC6B
:10A4E000401C2BF8140021E0491E47F824101DE001
:10A4F0000DD925F814904F20FEF77CFC08F80400D5
:10A50000B08C4008FEF776FC47F8240002E0401CBF
:10A5100025F8140035F8141078200AEB4105F021D5
:10A52000FEF75AFC687018F804002870641C032CAD
:10A53000CCDB7079254D20B1022802D0214C0027B8
:10A5400038E0204C002715E0607830B1C10816D003
:10A55000401A60702078401C20706078318D48432C
:10A56000020A207805EB8001B8B20968FEF716FFF1
:10A57000A41C7F1CB08C8742E6DBBDE8F09F401E28
:10A58000E7E7607830B1C10818D0401A60702078D1
:10A59000401C20706078318D4843020A207805EB1A
:10A5A0008001B08C0968C01B401E80B2FEF7F6FE29
:10A5B000A41C7F1CB08C8742E3DBDEE7401EE5E78E
:10A5C0000C0000203A3400205C38002000E800082D
:10A5D0002DE9F05F554A5079DFF854B14FF0000A89
:10A5E000012815D9D07B401CD073D07B08280FD907
:10A5F000534682F80FA0918C0BEB4100801E02E0C5
:10A6000030F8024D4480491E0029F9DC20F8023C54
:10A61000DFF82091454E002409F130074C36904672
:10A6200037F81400B8F82420651C6A4390420BD117
:10A6300059F82410002903DC401C27F8140028E0F6
:10A64000491E49F8241024E00DDD27F814A04F20FE
:10A65000FEF7D0FB3055B8F824004008FEF7CAFBDF
:10A6600049F8240002E0401C27F8140037F81400D1
:10A6700090FBF5F10BEB41056878B8B12878315DB6
:10A680000844C0F346002870F0217820FEF7A4FBB0
:10A690006870641C032CC3DB254C98F80500474602
:10A6A000254E28B1022803D0002539E0305DEAE7C5
:10A6B000002515E0607830B1010916D0401A6070AD
:10A6C0002078401C20706078398D4843020A207839
:10A6D00006EB8001A8B20968FEF760FEA41C6D1CA1
:10A6E000B88C8542E6DBBDE8F09F401EE7E7607866
:10A6F00030B1010918D0401A60702078401C2070D9
:10A700006078398D4843020A207806EB8001B88CC6
:10A710000968401B401E80B2FEF740FEA41C6D1C61
:10A72000B88C8542E3DBDEE7401EE5E70C00002045
:10A730003A3400205C38002000E800082DE9F0479A
:10A74000B04FB149F86BFC8E0278407851F82290F6
:10A7500051F820A0F88E6443C0F10F0578796D435D
:10A7600005287DD2DFE800F0031C355D8700002559
:10A7700005E0A2B2A8B24946FEF710FE6D1CB88CE7
:10A78000B5EB500FF5DBC0F34E0505E0A2B2A8B261
:10A790005146FEF703FE6D1CB88C8542F6DB04E1E2
:10A7A000002605E0AAB2B0B24946FEF7F7FD761CD6
:10A7B000B88CB6EB500FF5DBC0F34E0505E0A2B246
:10A7C000A8B25146FEF7EAFD6D1CB88C8542F6DB57
:10A7D000EBE0002620E0A2B2B0B24946C846FEF740
:10A7E000DDFDB88CA2B206EB500080B24146FEF708
:10A7F000D5FDB88CAAB2C6EB5000401E80B25146BF
:10A80000D046FEF7CBFDB88CAAB2801B401E80B2AA
:10A810004146FEF7C3FD761CB88CB6EB900FDADB31
:10A82000C3E0002622E0A2B2B0B24946C846FEF715
:10A83000B5FDB88CA2B2801B401E80B24146FEF727
:10A84000ADFDB88CAAB206EB500080B25146D0469E
:10A85000FEF7A4FDB88CAAB2C6EB5000401E00E083
:10A8600057E080B24146FEF799FD761CB88CB6EBF6
:10A87000900FD8DB99E0002646E0A2B2B0B249467C
:10A88000C846FEF78BFDB88CA2B2801B401E80B27A
:10A890004146FEF783FDB88CA2B206EB900080B271
:10A8A0004146FEF77BFDB88CA2B2800800EB400069
:10A8B000801B401E80B24146FEF770FDB88CAAB2E4
:10A8C00006EB500080B25146D046FEF767FDB88CCB
:10A8D000AAB2C6EB5000401E80B24146FEF75EFDB4
:10A8E000B88CAAB2C6EB9000401E80B24146FEF77B
:10A8F00055FDB88CAAB2800800EB4000304480B20D
:10A900004146FEF74BFD761CB88CB6EBD00FB4DB9E
:10A910004BE0002645E0A2B2B0B24946FEF73EFD4C
:10A92000B88CAAB2801B401E80B25146D046FEF7BA
:10A9300035FDB88CA2B206EB500080B24946FEF756
:10A940002DFDB88CAAB2C6EB5000401E80B2414625
:10A95000FEF724FDB88CA2B206EB900080B2494607
:10A96000FEF71CFDB88CAAB2C6EB9000401E80B268
:10A970004146FEF713FDB88CA2B2800800EB400000
:10A98000304480B24946FEF709FDB88CAAB280086F
:10A9900000EB4000801B401E80B24146FEF7FEFCEB
:10A9A000761CB88CB6EBD00FB5DB787B0028F88E20
:10A9B00005D070B1F88E401EF886BDE8F087401CC7
:10A9C000F886F88E0F28F8D90F20F88601207873C2
:10A9D000F3E70021F9867973F878072809D0F87829
:10A9E00038713879094900EB400001EB4000F86309
:10A9F000E3E73879401CC0B238710628F1D93971C3
:10AA0000EFE700000C00002000E800086C030020C5
:10AA10002DE9F04106460F46F7F766F8041E0D468D
:10AA200018BF0120284320F00040C0F17F6000F1F2
:10AA3000E040C00F0ED0301C18BF0120384320F07A
:10AA40000040C0F17F6000F1E040C00F04BF012072
:10AA5000FBF7F4FF20462946BDE8F08110B50A480F
:10AA60000A4A00210A4C09E0137800F8013B5378A8
:10AA700000F8013B937800F8013B491CA38C03EBE1
:10AA800043038B42F0DC10BDC92B002000E000081E
:10AA90000C00002070B5154EB07B78B130790007FE
:10AAA000000E5F2801D91030C0B2B17B81F00101E6
:10AAB000B1730F49002401EB800508E07F20F4E723
:10AAC000328D20462968FEF769FC641CE4B2B08C24
:10AAD0008442F5D3F078072807D13079401CC0B202
:10AAE0003071062801D90020307170BD0C000020A3
:10AAF00000E800080D4900B5C88E0828C88E05D2A8
:10AB0000022805D308790007000E04E00A2801D2C4
:10AB1000702000E07F20064A098D52F82000FDF7E2
:10AB200065F810205DF804EBFCF73EBA0C0000203D
:10AB300000E800082DE9F043524A5079032801D279
:10AB40000F2400E00624908C5379B0FBF4F54D48B7
:10AB5000022B4178C06B09D05379052B06D0D38ED8
:10AB6000A34201D209B118E0B9B1067890465279F2
:10AB7000DFF814919AB1012A23D0032A0FD0042AB6
:10AB80001FD0B8F83630A3423CD269B34778FEF7FD
:10AB9000CFFD002609EB870731E04678E6E7FEF7B0
:10ABA000C7FD002709EB860608E007FB04F0B8F8AC
:10ABB000282080B23168FEF7F1FB7F1CAF42F4DB46
:10ABC00036E0FEF7CDFD002709EB860609E0781C8C
:10ABD0006043401EB8F8282080B23168FEF7DEFBE3
:10ABE0007F1CAF42F3DB23E00778D0E706FB04F0DD
:10ABF000B8F8282080B23968FEF7D0FB761CAE4248
:10AC0000F4DB15E031B10778FEF7AAFD002609EB69
:10AC100087070BE04778F7E7701C6043401EB8F8E1
:10AC2000282080B23968FEF7B9FB761CAE42F3DB10
:10AC3000B8F836004146401C80B2A8F836004FF004
:10AC4000FF3202EB440290421ADD0022CA86C87825
:10AC5000072815D10879401CC0B20871062800D910
:10AC60000A710879094B00EB400003EB4000C86310
:10AC70004878401CC0B24870012801D988F80120EA
:10AC8000BDE8F0830C00002000E800086C03002001
:10AC90002DE9F0413549487905280ED2DFE800F06A
:10ACA000030507090B00022408E0032406E004243E
:10ACB00004E0062402E00A2400E00F24888C90FBC4
:10ACC000F4F6C88E401C80B2C88606EBD672B0EB94
:10ACD000620F1ADD0022CA86C878072807D0487894
:10ACE000401CC0B2487001280FD94A701AE0087998
:10ACF000401CC0B20871062800D90A7108791C4AA4
:10AD000000EB400002EB4000C863487850B1C86BCC
:10AD100040787F2800D97F20164A0025884602EB1C
:10AD200080070DE0C86B0078F3E7B8F83600B8F894
:10AD3000282005FB060080B23968FEF72FFB6D1C4A
:10AD4000A542F2DB00250CE0681CB8F83620704301
:10AD5000801A401EB8F8282080B23968FEF71EFB22
:10AD60006D1CA542F0DBBDE8F08100000C00002066
:10AD70006C03002000E800080B4AD18E491C89B200
:10AD8000D186132901D90021D186D38E0649834269
:10AD9000C96B01DD087800E04878044901EB8000C8
:10ADA000118D0068FCF722BF0C00002000E80008AD
:10ADB000074800B54278C16B895C064A02EB810204
:10ADC000018D1068FCF712FF5DF804EB00F026BC63
:10ADD0000C00002000E800082DE9F0476E4E6D4C95
:10ADE000B58C7079012800D96D087079032800D9D5
:10ADF0006D1040F27F10208001274FF07F082DE07A
:10AE000014F8030F401E10F0FF0004F8010902D0EF
:10AE1000B18C884221D3C7EB071090FBF5F0401CA2
:10AE20006070208824F8020C681E874213DB6420BF
:10AE3000FDF7E0FF32280ED2F078062804D007286C
:10AE400004D0F078000104E0702002E05F20FDF7FC
:10AE5000D1FF207001E084F800807F1CAF42CFDB7F
:10AE60004C4C7079B0464D4F012817D0022827D09E
:10AE7000032841D004284FF000060BD186E014F8D7
:10AE8000020BB8F8282007EB8001B0B20968FEF782
:10AE900085FA761CAE42F2DBBDE8F08700260CE0B6
:10AEA00014F8020BB8F8282007EB8001A81B401EFD
:10AEB00080B20968FEF772FA761CAE42F0DBEBE76F
:10AEC000002616E02078B8F8282007EB8001B0B201
:10AED0000968FEF763FA2078B8F8282007EB8001AC
:10AEE000C6EB4500401E80B20968FEF757FAA41C65
:10AEF000761CAE42E6DBCFE7C1460026B84614E03A
:10AF00002178A819B9F8282080B24F4658F82110A6
:10AF1000FEF744FAA81B2178401E3A8D80B258F8FB
:10AF20002110FEF73BFAA41C761CAE42E8DBB3E727
:10AF30002078B8F8282007EB8001B0B20968FEF746
:10AF40002DFA2078B8F8282007EB800106EB4500A1
:10AF500080B20968FEF722FA2078B8F8282007EBBB
:10AF60008001C6EB4500401E80B20968FEF716FA64
:10AF70002078B8F8282007EB8001C6EB8500401E3A
:10AF800080B20968FEF70AFAA41C761CAE42CFDB39
:10AF900082E700003A3400200C00002000E800089E
:10AFA0002DE9F0477C4E7B4DB48C7079012800D997
:10AFB00064087079032800D9641040F27F1028805B
:10AFC00001274FF070084FF07F0947E015F8030F95
:10AFD000401E10F0FF0005F8010902D0B18C884234
:10AFE0003BD328787F281BD0E01B401E00EB80005D
:10AFF000400090FBF4F0401C6870288825F8020C93
:10B00000601E874227DB6420FDF7F4FE322822D23F
:10B01000F07806281CD0072815D0F078000115E03C
:10B0200001206870601E874217DB6420FDF7E2FE96
:10B03000322812D2E01BB18C401E484390FBF4F042
:10B04000401C6870E4E75F20FDF7D4FE287004E040
:10B0500085F8008001E085F800907F1CA742B5DBF1
:10B060004C4D7079B0464D4F012817D0022827D09B
:10B07000032841D004284FF000060BD186E015F8D4
:10B08000020BB8F8282007EB8001B0B20968FEF780
:10B0900085F9761CA642F2DBBDE8F08700260CE0BD
:10B0A00015F8020BB8F8282007EB8001A01B401E02
:10B0B00080B20968FEF772F9761CA642F0DBEBE776
:10B0C000002616E02878B8F8282007EB8001B0B2F7
:10B0D0000968FEF763F92878B8F8282007EB8001A3
:10B0E000C6EB4400401E80B20968FEF757F9AD1C5C
:10B0F000761CA642E6DBCFE7002616E02878B8F8F3
:10B10000282007EB8001A01980B20968FEF746F9F4
:10B110002878B8F8282007EB8001A01B401E80B2D9
:10B120000968FEF73BF9AD1C761CA642E6DBB3E7E7
:10B130002878B8F8282007EB8001B0B20968FEF73C
:10B140002DF92878B8F8282007EB8001C6EB840099
:10B15000401E80B20968FEF721F92878B8F8282047
:10B1600007EB800106EB440080B20968FEF716F990
:10B170002878B8F8282007EB8001C6EB4400401E71
:10B1800080B20968FEF70AF9AD1C761CA642CFDB37
:10B1900082E700003A3400200C00002000E800089C
:10B1A0002DE9F043534C524B6079032101EB5001E0
:10B1B000E2780020504D02EB420205EB4202E263CE
:10B1C000024609E0E56B2D5C401CC0B203F8025B4F
:10B1D000884200D30020521CA58CAA42F2DB0A222E
:10B1E000B2FBF1F301FB1322E38EC2F10A02FF2549
:10B1F0004FF0000C9A422ADDE07B401CC0B2E073A5
:10B20000884204D384F80FC0E28E521CE2860020EC
:10B21000374A03464F1E16E0E67BB04201D1557017
:10B2200001E082F801C06679F60705D010B1401E32
:10B23000C0B206E0F8B204E0401CC0B2884200D3BD
:10B240000020921C5B1CA68CB342E5DB39E0E27B5C
:10B25000521CE273E37B01EB4102B3EB420F03D3D9
:10B2600084F80FC0A4F836C0E27B26460623B2FB62
:10B27000F3F7E1461E4A0023A1F1010C1DE0B8429C
:10B2800006D196F80F805FEAC87801D0557001E0CA
:10B2900082F8019096F805805FEAC87806D010B170
:10B2A000401EC0B207E00CF0FF0004E0401CC0B23A
:10B2B000884200D30020921C5B1CB6F824804345D2
:10B2C000DDDB0B4E00250D4F0CE07078218D4843DF
:10B2D000020A307807EB8001A8B20968FEF75EF831
:10B2E0006D1CB61CA08C8542EFDBBDE8F08300002E
:10B2F0003A3400200C0000206C03002000E8000815
:10B30000134900B5888C0622B0FBF2F0CA8E904239
:10B3100001D9C86B0FE00020C886CA7B521CCA73D3
:10B32000CA7B052A00D9C873C8780A4A00EB4000D6
:10B3300002EB4000C863CA7B098D805C064A52F864
:10B340002000FCF753FC18205DF804EBFBF72CBE43
:10B350000C0000206C03002000E800082DE9F041FB
:10B36000DFF86C801B4DA8F104070024A7F140060C
:10B3700018F80400401E10F0FF0008F804001AD16D
:10B380001548005D08F80400385D401CC0B238550F
:10B39000B18C884201D300203855E007F06B005D86
:10B3A0000FD005EB8003385D328D081A401E80B245
:10B3B0001968FDF7F3FF641CE4B2042CD8D3BDE890
:10B3C000F08105EB8001385D328D0968F1E70000FE
:10B3D0005000002000E80008F0C500081D4900B535
:10B3E000C88E0A281C482AD20A7900EB8210CA8E1D
:10B3F0000068022A10D2CA8E1ABBC0F3850262F31B
:10B400000700C0F30722920862F30F20C0F307423F
:10B41000920862F3174014E0CB8EC2B29B1EDA4052
:10B4200062F30700CB8EC0F307229B1EDA4062F363
:10B430000F20CB8EC0F307429B1EDA40E9E7D0F81D
:10B44000FC01098DFCF7D2FB18205DF804EBFBF73B
:10B45000ABBD00000C00002000E800080C4900B55E
:10B46000C88E042807D208790007000E5F2803D988
:10B470001030C0B200E07F20064A098D52F820004B
:10B48000FCF7B4FB08205DF804EBFBF78DBD000072
:10B490000C00002000E8000810B5104CA17B2046ED
:10B4A000C06BB9B140787F2800D97F200C4901EBEF
:10B4B0008000218D0068FCF799FBE08E401C80B273
:10B4C000E086092805D90020E086A07B20B1002075
:10B4D000A07310BD0078E6E70120F9E70C0000201A
:10B4E00000E800081C4900B5087900015F2800DD6C
:10B4F00010301A4A52F82000CA8ECB8E0A2AC2B2E5
:10B500000CD2DA4062F30700CB8EC0F30722DA4098
:10B5100062F30F20C0F30742CB8E11E0C3F1130397
:10B52000DA4062F30700CB8EC0F30722C3F11303A6
:10B53000DA4062F30F20CB8EC0F30742C3F113034E
:10B54000DA4062F31740098DFCF750FB14205DF8D8
:10B5500004EBFBF729BD00000C00002000E8000808
:10B5600010B5134C20790007000E00F023F8E08E90
:10B57000401C80B2E086262815D90022E286A07BF6
:10B5800090B10020A073E07807280FD00020A17BA5
:10B5900001B10121084206D02079401CC0B22071BF
:10B5A000062800D9227110BD0120EBE70120EEE74B
:10B5B0000C0000205F2801D91030C0B2154B997BD8
:10B5C0000029D98E01D0C1F12601134A01EB4101B6
:10B5D000490652F82000090EC2B2521A00D50022C4
:10B5E0005243120A62F30700C0F30722521A00D531
:10B5F00000225243120A62F30F20C0F30742511A8D
:10B6000000D500214943090A61F31740198DFCF761
:10B61000EDBA00000C00002000E800081249C88EB6
:10B62000401C80B2C8868A8CB0EB520F0BD300222C
:10B63000CA86C878072807D04878401CC0B248702E
:10B64000012800D94A7070470879401CC0B20871BF
:10B65000062800D90A710879044A00EB400002EB81
:10B660004000C863704700000C0000206C030020FD
:10B6700070B5FFF7F3F9144EB07B401CC0B2B07345
:10B68000022801D90020B0730024FF250FE02044D8
:10B6900090FBF5F105FB1100C0B2FBF706F901467E
:10B6A000B07B328D204480B2FDF778FEE41CB08C74
:10B6B000B17B401AA042F08EE9DC401CF086F08E8F
:10B6C000C0B2F08670BD00000C00002000EBC0008E
:10B6D0000649C01C80B2C884054A0021104411707C
:10B6E00000F8011C00F8021CFFF7B8B90C0000209C
:10B6F000C82B002010B521214E48F6F70FFD002879
:10B70000F9D14C4802215738F6F708FD0028F8D146
:10B71000484804214A38F6F701FD0028F8D1454889
:10B720001E212230F6F7FAFC0028F8D141481E21EC
:10B730004130F6F7F3FC0028F8D13E482321603071
:10B74000F6F7ECFC0028F8D13A4824218430F6F7CB
:10B75000E5FC0028F8D137482C21A930F6F7DEFCAB
:10B760000028F8D134213448F6F7D8FC0028F9D164
:10B7700031481E219E38F6F7D1FC0028F8D12E481A
:10B780003A217F38F6F7CAFC0028F8D12A4843212D
:10B790004438F6F7C3FC0028F8D126482E21D630CD
:10B7A000F6F7BCFC0028F8D123482E21CD38F6F757
:10B7B000B5FC0028F8D1204836213530F6F7AEFC2C
:10B7C0000028F8D11C4836216C30F6F7A7FC002879
:10B7D000F8D119481921A330F6F7A0FC0028F8D1B8
:10B7E00015482E21BD30F6F799FC0028F8D11248F3
:10B7F0003F21EC30F6F792FC0028F8D124210F48C5
:10B80000F6F78CFC0028F9D10A4802215738F6F7E0
:10B8100085FC0028F8D109481D212530F6F77EFC6B
:10B820000028F8D1034802215738F6F777FC0028A2
:10B83000F8D110BD43C6000815C8000842C9000869
:10B840003EB504460723002201A9FBF7D9F90028D9
:10B8500014DB04444FF0FF3514F8010B2C280CD1F5
:10B860000523002202A92046FBF7CAF9002805DBC0
:10B87000204410F8011B2C2901D028463EBD7F230F
:10B8800000226946FBF7BCF90028F7DBBDF804008D
:10B89000054B00EB400203EB4202BDF80830BDF857
:10B8A0000010D1543EBD00006C03002008B547F6DF
:10B8B000FF7320226946FBF7A3F900280ADB06483C
:10B8C000418E01F400414186418EBDF800201144B3
:10B8D0004186002008BD00000C000020F0B507469E
:10B8E0001348002501240188124E06E030F8142088
:10B8F000914200D22546641CE4B2727C9442F5D396
:10B900002846FBF713F94043718D000C4843010CA6
:10B91000012905D958204543707CB5FBF0F0C7B22A
:10B92000054850F82700BDE8F040FCF75FB900007B
:10B930003A3400200C00002000E800082DE9F04710
:10B94000244C81460025608DDFF88CA001B228468A
:10B9500022E0224ADFF8888094F817C032F81020DD
:10B9600038F810300AEB0016D31A26F81C3028F8E5
:10B9700010200022134636F913C05B1C02EB2C3258
:10B98000DBB212B2082BF6D3002A03DB954201DAB0
:10B9900015460746401CC0B2627C9042D9D3012DA7
:10B9A0000ADD58204743607C401E97FBF0F000F012
:10B9B000FF090C2D00DAC9100A4A52F82900FCF7D9
:10B9C00015F9E07D401CE075E07D00F00700E075B2
:10B9D000BDE8F0870C000020323600203A34002009
:10B9E000F001002000E800082DE9FC4F0021084686
:10B9F000F54CDFF8D8B3F64D0E461BE03BF81020AF
:10BA00006F7A5B46B2EBC71F05D96F7AA2EBC712FC
:10BA100023F8102001E023F8106033F8107034F898
:10BA20001020974201D223F810203BF81020401C30
:10BA30001144C0B26A7C9042E0D3E54800244079CA
:10BA4000DFF890A301280AF5C07509D0022860D05C
:10BA5000032876D0002975D00026DFF8748390E1A2
:10BA6000E1B30026DFF8688333E0582006FB00F2DC
:10BA7000487C0027401E92FBF0F080B201903BF81A
:10BA800016008A8C5043C010000C009014E00199FD
:10BA9000528D0AEB8109A0B2D9F80010FDF77EFCA7
:10BAA000B8F82400B8F82A20001B401E80B2D9F84C
:10BAB0000010FDF773FC641C384600997F1C884217
:10BAC00005DAB8F824004246B4EB500FDFDB761CF1
:10BAD000F6B298F8110041468642C6D3BC4F002604
:10BAE000B88CC4EB500810E0BA79A0B2B949D1F8CB
:10BAF000C011FDF753FCB88CBA79001B401E80B210
:10BB0000296CFDF74BFC641C761C4645ECDBBDE85C
:10BB1000FC8FE9B34FF00008AD4E4DE0582108FB13
:10BB200001F0717C4FF00009491E90FBF1F080B2EA
:10BB300001903BF81800B18C48430011000C0090B4
:10BB40002CE06FE022E1019A04EB90000AEB8207FF
:10BB5000728D80B23968FDF721FCB08C728DC4EB18
:10BB60009000401E80B23968FDF718FCB08C728DD1
:10BB7000800800EB4000204480B23968FDF70EFCDD
:10BB8000B08C800800EB4000001B401E80B200E03B
:10BB900015E0728D3968FDF701FC641C4946009878
:10BBA00009F10109814203DAB08CB4EB900FCADBD2
:10BBB00008F1010000F0FF08717C8845AED3844E87
:10BBC0000027B08CC4EB900829E0B08CB27904EB6C
:10BBD000900080B27F49D1F8C011FDF7DFFBB08C37
:10BBE000B279C4EB9000401E80B2296CFDF7D6FB01
:10BBF000B08CB279800800EB4000204480B2296C00
:10BC0000FDF7CCFBB08CB279800800EB4000001B44
:10BC1000401E80B2296CFDF7C1FB641C7F1C4745A8
:10BC2000D3DB74E7F1B34FF00008694E44E05821CC
:10BC300008FB01F0717C4FF00009491E90FBF1F008
:10BC400080B201903BF81800B18C48430011000C01
:10BC5000009021E00199728D0AEB8107A0B239684A
:10BC6000FDF79CFBB08C728DC4EB5000401E80B27F
:10BC70003968FDF793FBB08C728D04EB500080B2F5
:10BC80003968FDF78BFBB08C728D001B401E80B2B3
:10BC90003968FDF783FB641C4946009809F10109E6
:10BCA000814200E00BE003DAB08CB4EB900FD1DB03
:10BCB00008F1010000F0FF08717C8845B7D3444EBD
:10BCC0000027B08CC4EB900821E0B279A0B24149C2
:10BCD000D1F8C011FDF762FBB08CB279C4EB500013
:10BCE000401E80B2296CFDF759FBB08CB27904EB91
:10BCF000500080B2296CFDF751FBB08CB279001B6B
:10BD0000401E80B2296CFDF749FB641C7F1C47452F
:10BD1000DBDBFCE6582006FB00F2487C0027401ED7
:10BD200092FBF0F080B201903BF816008A8C5043F1
:10BD3000C010000C009017E0019B04EB5000528DE6
:10BD40000AEB830980B2D9F80010FDF727FBB8F899
:10BD50002400B8F82A20C4EB5000401E80B2D9F865
:10BD60000010FDF71BFB641C384600997F1C8842BD
:10BD700005DAB8F824004246B4EB500FDCDB761C41
:10BD8000F6B298F8110041468642C3D3104F002600
:10BD9000B88CC4EB500814E0B88CBA7904EB5000AE
:10BDA00080B20C49D1F8C011FDF7F8FAB88CBA7915
:10BDB000C4EB5000401E80B2296CFDF7EFFA641C02
:10BDC000761C4645E8DBA2E63A340020F00100206C
:10BDD0000C00002000E800082DE9F04F0024DFF8F7
:10BDE00094B1DFF89481BEE02046FAF79FFE40430D
:10BDF000060CB8F82A0098F8111046435820604302
:10BE0000491E90FBF1F087B298F8050030B1012887
:10BE100019D002284FF000057DD15BE000250BEB27
:10BE20008707360C09E0407C324605FB004080B2B3
:10BE30003968FDF7B3FA6D1CEDB298F8131040465F
:10BE40008D42F0D38DE000251BE0320C497C9246F8
:10BE50000BEB870905FB014188B2D9F80010FDF70B
:10BE60009DFA98F8111005FB0142B8F82410891AC0
:10BE7000491E88B25246D9F80010FDF78FFA6D1CA2
:10BE8000EDB298F813004146B5EB500FDDD368E0F2
:10BE9000B8F8240004EB500198F811000BEB870967
:10BEA00005FB0010320C80B29246D9F80010FDF765
:10BEB00075FA98F81100524605FB0041B8F82400C5
:10BEC000C1EB5000401E80B2D9F80010FDF766FAB1
:10BED0006D1CEDB298F81310B5EB510FD8D340E0BC
:10BEE000320C497C92460BEB870905FB014188B275
:10BEF000D9F80010FDF752FA98F8111005FB01422D
:10BF0000B8F82410891A491E88B25246D9F8001090
:10BF1000FDF744FA00E01EE0B8F8240004EB5001FD
:10BF200098F81100524605FB001080B2D9F80010B5
:10BF3000FDF734FA98F81100524605FB0041B8F8B5
:10BF40002400C1EB5000401E80B2D9F80010FDF76C
:10BF500025FA6D1CEDB298F813004146B5EB900F31
:10BF6000BED3641CE4B298F811008442FFF43CAFE5
:10BF7000BDE8F08F00E800080C000020F0B40025B8
:10BF80002B462A46104E114F07E036F812409C42CD
:10BF900001D923461546521CD2B27C7CA242F4D36E
:10BFA0004BB136F815208A4205D958204543787C94
:10BFB000B5FBF0F0C0B2064901EB8000798D006856
:10BFC000F0BCFBF713BE00003A3400200C00002048
:10BFD00000E800082DE9FC4F00208146DFF820B280
:10BFE00004E1FAF7A3FD4043040CB8F82A004443E7
:10BFF000582009FB00F198F81100401E91FBF0F069
:10C0000085B298F8130009FB00F698F8050005289A
:10C0100073D2DFE800F003152B4D730000270BEB04
:10C020008505240C07E0F01980B222462968FDF747
:10C03000B5F97F1CFFB298F813008742F3D3D1E023
:10C0400000270BEB8505240C0BE0B8F82400F11950
:10C05000401A401E80B222462968FDF79FF97F1CD6
:10C06000FFB298F813108F42EFD3BBE070080026A0
:10C07000009017E000980BEB8507220C00EB060AF6
:10C0800090461FFA8AF03968FDF788F95D49424603
:10C09000898CA1EB0A00401E80B23968FDF77EF959
:10C0A000761CF6B25748C07CB6EB500FE2D399E04D
:10C0B000770800261BE053480BEB8508220C808C88
:10C0C000924607EB5000304480B2D8F80010FDF7DC
:10C0D00065F94C48B9195246808CC1EB5000401E9E
:10C0E00080B2D8F80010FDF759F9761CF6B2454B2E
:10C0F000D87CB6EB500FDED374E034E04FEA960AFA
:10C1000000262AE0220C0BEB85070AEB06080092BA
:10C110001FFA88F03968FDF741F93A49009A898C8D
:10C12000A1EB0800401E80B23968FDF737F93549A8
:10C13000009A898C0AEB5100304480B23968FDF7CF
:10C140002DF93049009A898CC8EB5100401E80B20D
:10C150003968FDF723F9761CF6B22A48C07CB6EBA5
:10C16000900FCFD33EE04FEA960A002635E0220C2E
:10C170000092B8F824100BEB85070AEB91003044CD
:10C1800080B23968FDF70AF90AEB06000190B8F8A9
:10C190002410009AC0EB9100401E80B23968FDF770
:10C1A000FDF8B8F82400009A800800EB400101EB8C
:10C1B0000A00304480B23968FDF7F0F8B8F824007E
:10C1C000009A800800EB40010198081A401E80B2D6
:10C1D0003968FDF7E3F8761CF6B298F81300B6EB71
:10C1E000900FC4D309F10100C0B28146DFF814807A
:10C1F00098F811108945FFF4F4AEBDE8FC8F0000FB
:10C2000000E800080C0000202DE9FC4F00208046CB
:10C21000DFF810B2FAF78AFC4043050C8248418DE2
:10C2200058224D4308FB02F10522B1FBF2F6017DD5
:10C2300008FB01F44179052975D2DFE801F0031606
:10C240002D4F7500002781460BEB86062D0C07E06D
:10C25000E01980B22A463168FDF7A0F87F1CFFB2D2
:10C2600099F814008742F3D3D3E0002781460BEB03
:10C2700086062D0C0BE0B9F82400E119401A401E87
:10C2800080B22A463168FDF789F87F1CFFB299F821
:10C2900014108F42EFD3BCE061080024009117E036
:10C2A00000980BEB86072A0C00EB040A91461FFA54
:10C2B0008AF03968FDF772F85B494A46898CA1EB30
:10C2C0000A00401E80B23968FDF768F8641CE4B2C9
:10C2D0005548007DB4EB500FE2D39AE06708002484
:10C2E0001BE051480BEB86092A0C808C924607EB29
:10C2F0005000204480B2D9F80010FDF74FF84A48AA
:10C3000039195246808CC1EB5000401E80B2D9F8DA
:10C310000010FDF743F8641CE4B2434B187DB4EB06
:10C32000500FDED375E034E04FEA940A00242AE08F
:10C330002A0C0BEB86070AEB040900921FFA89F01E
:10C340003968FDF72BF83849009A898CA1EB090070
:10C35000401E80B23968FDF721F83349009A898C74
:10C360000AEB5100204480B23968FDF717F82E49D6
:10C37000009A898CC9EB5100401E80B23968FDF7E4
:10C380000DF8641CE4B22848007DB4EB900FCFD3C5
:10C390003FE04FEA94090024824635E02A0C0092DF
:10C3A000BAF824100BEB860709EB9100204480B209
:10C3B0003968FCF7F3FF09EB04000190BAF8241088
:10C3C000009AC0EB9100401E80B23968FCF7E6FF8E
:10C3D000BAF82400009A800800EB400101EB090044
:10C3E000204480B23968FCF7D9FFBAF82400009ADB
:10C3F000800800EB40010198081A401E80B239689D
:10C40000FCF7CCFF641CE4B29AF81400B4EB900F74
:10C41000C4D308F10100C0B280460628FFF4FAAE8A
:10C42000BDE8FC8F00E800080C0000202DE9F84F63
:10C43000002108464F4D504B04E035F81020401CB9
:10C440001144C0B25A7C9042F7D3587CDFF82CA13B
:10C45000B1FBF0F40020064629E0597C6E22091A4F
:10C46000491E51435A7C521E91FBF2F1503189B260
:10C4700061434FF4007202EBD11135F810208A426B
:10C4800003D9FA222AF810200FE03AF81010524689
:10C49000FA2902D922F8106005E0092903D90A39DE
:10C4A0002AF8101001E02AF81060401CC0B2597C34
:10C4B0008842D2D30025DFF8C8B0994652E03AF856
:10C4C0001510428D5143C1F3CF1100915821427C88
:10C4D0006943B1FBF2F1CFB2C17C6943C1F34706B6
:10C4E00041794FF00004C90735D10BEB870711E004
:10C4F00030198046009A3968FCF750FFB9F82410CB
:10C50000009AA1EB0800401E80B23968FCF746FF94
:10C51000641CE4B299F81300B4EB500FE8D31FE0A9
:10C52000B9F824000BEB870806EB5000204480B2DA
:10C53000009AD8F80010FCF731FFB9F8240031193F
:10C54000C1EB5000401E80B2009AD8F80010FCF7F2
:10C5500025FF641CE4B299F81300B4EB500FDFD34D
:10C560006D1CEDB299F8111048468D42A7D3BDE875
:10C57000F88F00003A3400200C000020F001002069
:10C5800000E80008F0B4002423462146DFF84CC040
:10C59000134E144F0DE03CF8112036F81150AA420A
:10C5A00003D99A4201D913460C4626F81120491C9A
:10C5B000C9B27A7C9142EED3B3F5007F06D95820F8
:10C5C0004443787C401E94FBF0F0C0B2064901EB76
:10C5D0008000798D0068F0BCFBF708BB3A3400207E
:10C5E000F00100200C00002000E800080D0A000007
:10C5F000030304044F4B0D0A0041540D0A0050720E
:10C60000696E7420706C6179206C6973743A0D0ADC
:10C61000004E0970726F670973756270726F6709F7
:10C6200074656D706F096469720D0A005072696EED
:10C63000742070726F6772616D20636F6C6F723AF5
:10C640000D0A0053544D333220434D5520636F6E15
:10C6500074726F6C6C657220415420436F6D6D6114
:10C660006E640D0A0041542B5353202D20536176E4
:10C67000652053657474696E677320636F6E6669B5
:10C68000670D0A0041542B5350202D2053617665CD
:10C6900020506C61794C69737420636F6E666967B2
:10C6A0000D0A0041542B5343202D20536176652001
:10C6B00070726F6772616D20436F6C6F7220636F71
:10C6C0006E6669670D0A0041542B5050202D205092
:10C6D00072696E74696E6720506C61796C697374ED
:10C6E0002070726F6772616D730D0A0041542B5098
:10C6F00043202D205072696E74696E6720636F6CE1
:10C700006F72207573656420696E2074686520708F
:10C71000726F6772616D0D0A0041542B44302E2EEA
:10C720003739202D2044656C657465207468652058
:10C7300070726F6772616D2066726F6D20506C61F0
:10C74000794C6973740D0A0041542B4441202D200B
:10C7500044656C65746520616C6C2074686520703C
:10C76000726F6772616D2066726F6D20506C6179B7
:10C770004C6973740D0A0041542B4C33302E2E3209
:10C780003430202D20536574204C6564204E756D27
:10C790006265720D0A0041542B41302E2E32392C25
:10C7A000302E2E372C302E2E352C302E2E3234308B
:10C7B000202D20416464207468652070726F677258
:10C7C000616D20746F20506C61794C6973740D0A2F
:10C7D0000041542B49302E2E37392C302E2E323931
:10C7E0002C302E2E372C302E2E352C302E2E32344F
:10C7F00030202D20496E7365727420746865207036
:10C80000726F6772616D20746F20506C61794C6932
:10C8100073740D0A0041542B4E302E2E32392C30B9
:10C820002E2E372C302E2E352C302E2E323430201A
:10C830002D2053657420612064796E616D696320D9
:10C8400070726F6772616D0D0A0041542B42302E79
:10C850002E323536202D2053657420746865206291
:10C8600072696768746E65737320666F722064798D
:10C870006E616D69632070726F6772616D730D0A0E
:10C880000041542B4D302E2E323536202D2053654D
:10C890007420746865206272696768746E6573736A
:10C8A00020666F72206D75736963616C2070726FA2
:10C8B0006772616D730D0A0041542B5431302E2E76
:10C8C000323430202D205365742074656D706F0DE7
:10C8D0000A0041542B57305B315D202D2030202D34
:10C8E0002064697361626C6520434C41502C203197
:10C8F000202D20656E61626C6520434C41500D0A0D
:10C900000041542B43302E2E372C302E2E352C3018
:10C910002E2E313132202D205772697465207375A7
:10C920006270726F6772616D2C636F6C6F72206ED4
:10C93000756D6265722C6E657720636F6C6F720D1A
:10C940000A0041542B5A302E2E3332373630202DE8
:10C95000205365742070726F6772616D2072756EFE
:10C9600074696D650D0A0053616D706C653A204104
:10C97000542B4C3630202D20536574203630206CDB
:10C9800065640D0A004572726F7220636F6D6D6190
:10C990006E642E20456E7465723A2041542B4820F7
:10C9A0002D20746F2076696577207468652068652E
:10C9B0006C702E0D0A004572726F723A20746865B1
:10C9C0007265206973206E6F207365742076616CC8
:10C9D00075650D0A004572726F723A207365742096
:10C9E00076616C7565206973207665727920736D48
:10C9F000616C6C0D0A004572726F723A2073657437
:10CA00002076616C75652069732076657279206285
:10CA100069670D0A004572726F723A206E6F206D61
:10CA2000756C7469706C652062616E64776964749A
:10CA3000680D0A004572726F723A20746865206C46
:10CA40006F6F702062756666657220697320667507
:10CA50006C6C2C206265666F7265207772697469F0
:10CA60006E672C2072656D6F7665206F6E65206F26
:10CA700066207468652070726F6772616D730D0A4D
:10CA80000041542B454E41424C45494E443D300DEA
:10CA90000A00000000000000000001020304060775
:10CAA000080900000000010203040000000000006B
:10CAB000000000000000F03F000000000000F83F10
:10CAC00000000000000000000000004003B8E23F4A
:10CAD000000000000000000006D0CF43EBFD4C3EFC
:10CAE000033333333333E33FFFAB6FDBB66DDB3FF1
:10CAF0004D268F515555D53F01411DA96074D13F39
:10CB000065DBC9934A86CD3FEF4E454A287ECA3F32
:10CB10003E5555555555C53F93BDBE166CC166BFB4
:10CB20002CDE25AF6A56113FF16BD2C541BDBBBEAD
:10CB3000D0A4BE726937663E00000000000000000D
:10CB400060CB000800000020CC0100008A1B000818
:10CB50004CCC0008CC010020744A00002C6A00086C
:10CB600032019210321E120A7320083C1405080B81
:10CB70002A09166112F01373085A01021183800703
:10CB8000136C0342204F0303040498390C511939E4
:10CB900013B1591B08E1041AED0413155A1B08417F
:10CBA000041A910C1ABD041704030904120114029B
:10CBB00002021640830440571D020102035A13BDAE
:10CBC000201B08B7041AB3041AE104113CA24A045A
:10CBD0004F120632022A40B81C0902432F111CC012
:10CBE00032091B1B01020B1305241D100105249C97
:10CBF0001008042402020524061701070582030811
:10CC00001C1009046529C51D07050102432C0705F1
:10CC100081070938442A40072A8107112B09074454
:10CC20000A2204440A16FF44136D571408DB561CED
:10CC3000084958EC311A17101A99101AAD04C11A84
:0CCC400055181A49041A61041A3D04C179
:020000040800F2
:10E000009249249249269249349249369249A492DF
:10E0100049A69249B49249B6924D24924D26924D0A
:10E0200034924D36924DA4924DA6924DB4924DB677
:10E030009269249269269269349269369269A4920F
:10E0400069A69269B49269B6926D24926D26926D1A
:10E0500034926D36926DA4926DA6926DB4926DB6A7
:10E060009349249349269349349349369349A49379
:10E0700049A69349B49349B6934D24934D26934DA5
:10E0800034934D36934DA4934DA6934DB4934DB612
:10E090009369249369269369349369369369A493A9
:10E0A00069A69369B49369B6936D24936D26936DB5
:10E0B00034936D36936DA4936DA6936DB4936DB642
:10E0C0009A49249A49269A49349A49369A49A49AEF
:10E0D00049A69A49B49A49B69A4D249A4D269A4D22
:10E0E000349A4D369A4DA49A4DA69A4DB49A4DB68F
:10E0F0009A69249A69269A69349A69369A69A49A1F
:10E1000069A69A69B49A69B69A6D249A6D269A6D31
:10E11000349A6D369A6DA49A6DA69A6DB49A6DB6BE
:10E120009B49249B49269B49349B49369B49A49B88
:10E1300049A69B49B49B49B69B4D249B4D269B4DBC
:10E14000349B4D369B4DA49B4DA69B4DB49B4DB629
:10E150009B69249B69269B69349B69369B69A49BB8
:10E1600069A69B69B49B69B69B6D249B6D269B6DCC
:10E17000349B6D369B6DA49B6DA69B6DB49B6DB659
:10E18000D24924D24926D24934D24936D249A4D2DE
:10E1900049A6D249B4D249B6D24D24D24D26D24D49
:10E1A00034D24D36D24DA4D24DA6D24DB4D24DB6B6
:10E1B000D26924D26926D26934D26936D269A4D20E
:10E1C00069A6D269B4D269B6D26D24D26D26D26D59
:10E1D00034D26D36D26DA4D26DA6D26DB4D26DB6E6
:10E1E000D34924D34926D34934D34936D349A4D378
:10E1F00049A6D349B4D349B6D34D24D34D26D34DE4
:10E2000034D34D36D34DA4D34DA6D34DB4D34DB650
:10E21000D36924D36926D36934D36936D369A4D3A7
:10E2200069A6D369B4D369B6D36D24D36D26D36DF3
:10E2300034D36D36D36DA4D36DA6D36DB4D36DB680
:10E24000DA4924DA4926DA4934DA4936DA49A4DAED
:10E2500049A6DA49B4DA49B6DA4D24DA4D26DA4D60
:10E2600034DA4D36DA4DA4DA4DA6DA4DB4DA4DB6CD
:10E27000DA6924DA6926DA6934DA6936DA69A4DA1D
:10E2800069A6DA69B4DA69B6DA6D24DA6D26DA6D70
:10E2900034DA6D36DA6DA4DA6DA6DA6DB4DA6DB6FD
:10E2A000DB4924DB4926DB4934DB4936DB49A4DB87
:10E2B00049A6DB49B4DB49B6DB4D24DB4D26DB4DFB
:10E2C00034DB4D36DB4DA4DB4DA6DB4DB4DB4DB668
:10E2D000DB6924DB6926DB6934DB6936DB69A4DBB7
:10E2E00069A6DB69B4DB69B6DB6D24DB6D26DB6D0B
:10E2F00034DB6D36DB6DA4DB6DA6DB6DB4DB6DB698
:020000040800F2
:10E80000FF000000FF100000FF200000FF300000AC
:10E81000FF400000FF500000FF600000FF7000009C
:10E82000FF800000FF900000FFA00000FFB000008C
:10E83000FFC00000FFD00000FFE00000FFF000007C
:10E84000FFFF0000F0FF0000E0FF0000D0FF00002D
:10E85000C0FF0000B0FF0000A0FF000090FF00001C
:10E8600080FF000070FF000060FF000050FF00000C
:10E8700040FF000030FF000020FF000010FF0000FC
:10E8800000FF000000FF100000FF200000FF30002C
:10E8900000FF400000FF500000FF600000FF70001C
:10E8A00000FF800000FF900000FFA00000FFB0000C
:10E8B00000FFC00000FFD00000FFE00000FFF000FC
:10E8C00000FFFF0000F0FF0000E0FF0000D0FF00AD
:10E8D00000C0FF0000B0FF0000A0FF000090FF009C
:10E8E0000080FF000070FF000060FF000050FF008C
:10E8F0000040FF000030FF000020FF000010FF007C
:10E900000000FF001000FF002000FF003000FF00AB
:10E910004000FF005000FF006000FF007000FF009B
:10E920008000FF009000FF00A000FF00B000FF008B
:10E93000C000FF00D000FF00E000FF00F000FF007B
:10E94000FF00FF00FF00F000FF00E000FF00D0002C
:10E95000FF00C000FF00B000FF00A000FF0090001B
:10E96000FF008000FF007000FF006000FF0050000B
:10E97000FF004000FF003000FF002000FF001000FB
:10E98000FF000000FF100000FF200000FF3000002B
:10E99000FF400000FF500000FF600000FF7000001B
:10E9A000FF800000FF900000FFA00000FFB000000B
:10E9B000FFC00000FFD00000FFE00000FFF00000FB
:10E9C000FFFFFF00EEEEEE00DDDDDD00CCCCCC0085
:10E9D000BBBBBB00AAAAAA009999990088888800A5
:10E9E00077777700666666005555550044444400C5
:10E9F00033333300222222001111110000000000E5
:020000040800F2
:10EC000005081040D20000000000000000000000D5
:10EC100000000000000000000000000000000000F4
:10EC20000508103060FC000000000000000000003B
:10EC300000000000000000000000000000000000D4
:10EC4000030406090C10182850F000000000000012
:10EC500000000000000000000000000000000000B4
:10EC600002030405060708090A0C12182850F000D0
:10EC70000000000000000000000000000000000094
:10EC80000202030304050607080A0C0E12182840A6
:10EC90006478000000000000000000000000000098
:10ECA0000202020303040405060708090B0D1119EB
:10ECB000233C6496000000000000000000000000FB
:10ECC00002020203030304040505060607070808F9
:10ECD00009090A0A0B0C0D0E0F10182850A000008D
:020000040800F2
:10F40000001040500A2010204030143620301030B8
:10F41000084830405010285F405020503212007091
:10F420000030041E704030100C447020004028143E
:020000040800F2
:10F500001F1F1F1F1F1F1F1F1F1F1F1F1F1F1F1F0B
:10F510001F1F1F1F1F1F1F1F1F1F1F1F1F1F000039
:10F520001F1F1F1F1F1F1F1F1F1F1F1F1F1F1F1FEB
:10F530001F1F1F1F1F1F1F1F1F1F1F1F1F1F000019
:10F540001F1F1F1F1F1F1F1F1F1F1F1F1F1F1F1FCB
:10F550001F1F1F1F1F1F1F1F1F1F1F1F1F1F0000F9
:10F560001F1F1F1F1F1F1F1F1F1F1F1F1F1F1F1FAB
:10F570001F1F1F1F1F1F1F1F1F1F1F1F1F1F0000D9
:10F580001F1F1F1F1F1F1F1F1F1F1F1F1F1F1F1F8B
:10F590001F1F1F1F1F1F1F1F1F1F1F1F1F1F0000B9
:10F5A0001F1F1F1F1F1F1F1F1F1F1F1F1F1F1F1F6B
:10F5B0001F1F1F1F1F1F1F1F1F1F1F1F1F1F000099
:10F5C0001F1F1F1F1F1F1F1F1F1F1F1F1F1F1F1F4B
:10F5D0001F1F1F1F1F1F1F1F1F1F1F1F1F1F000079
:10F5E0001F1F1F1F1F1F1F1F1F1F1F1F1F1F1F1F2B
:10F5F0001F1F1F1F1F1F1F1F1F1F1F1F1F1F000059
:04000005080000ED02
:00000001FF
